:020000040001F9
:10900000C0400020C1930100C9930100CB9301002F
:10901000CD930100CF930100D19301000000000027
:10902000000000000000000000000000D3930100D9
:10903000D593010000000000D7930100D9930100EF
:109040009DB40100DB930100DB930100DB93010081
:10905000DB93010000000000D5B2010041B5010022
:10906000DB930100DB930100DB930100DB93010044
:10907000DB930100F5B40100DB930100DB930100F9
:10908000DB9301001DB50100DB930100DB930100C0
:1090900089B60100DB9301008DB60100DB9301006E
:1090A000DB930100DB9301000000000000000000E2
:1090B000DB930100DB9301000000000000000000D2
:1090C00000000000000000000000000000000000A0
:1090D0000000000000000000000000000000000090
:1090E0000000000000000000000000000000000080
:1090F0000000000000000000000000000000000070
:10910000000000000000000000000000000000005F
:10911000000000000000000000000000000000004F
:10912000000000000000000000000000000000003F
:10913000000000000000000000000000000000002F
:10914000000000000000000000000000000000001F
:10915000000000000000000000000000000000000F
:1091600000000000000000000000000000000000FF
:1091700000000000000000000000000000000000EF
:1091800000000000000000000000000000000000DF
:1091900000000000000000000000000000000000CF
:1091A00000000000000000000000000000000000BF
:1091B00000000000000000000000000000000000AF
:1091C000000000000000000000000000000000009F
:1091D000000000000000000000000000000000008F
:1091E000000000000000000000000000000000007F
:1091F000000000000000000000000000000000006F
:10920000DFF80CD000F0F0FF00480047AD0102008D
:10921000C040002030B450E8012F93B2C4892344E9
:109220008489A34228BF1B1B0489A34202BFBFF34A
:109230002F8F002007E0C3EA020340E80134002C2E
:10924000E9D14FF001000A6030BC704750E8012FAF
:10925000C2EA024240E801210029F7D1704730B448
:1092600050E8022F1FFAA2F3C488A34202BFBFF343
:109270002F8F00200DE0C48923448489A34228BF96
:109280001B1BC2EA034340E80234002CE8D14FF034
:1092900001000A6030BC704750E8022FC2EA224247
:1092A00040E802210029F7D17047034653E8022F16
:1092B000D988B2EB324F4FF0000017BF92B241EAAB
:1092C000014142EA014104E05A68B2EB324F08BF63
:1092D000012043E80212002AE8D1704730B4044666
:1092E00054E8000F0D4644E80053002BF8D11560F8
:1092F00030BC704730B4044654E8000F40EA010522
:1093000044E80053002BF7D1156030BC704730B4EF
:10931000044654E8000F00EA010544E80053002B1E
:10932000F7D1156030BC704730B4044654E8000FE4
:1093300080EA010544E80053002BF7D1156030BCEA
:10934000704730B4044654E8000F00EB010544E8D0
:109350000053002BF7D1156030BC704730B4044681
:1093600054E8000FA0EB010544E80053002BF7D1AF
:10937000156030BC704770B404464FF0000054E8EC
:10938000006F0D68AE4207BF44E80023012044E8A7
:1093900000630E60002B1CBF0020F0E770BC70471C
:1093A00030B4044654E8000F88422CBF451A0546E5
:1093B00044E80053002BF5D1156030BC7047000025
:1093C0000648804706480047FEE7FEE7FEE7FEE75F
:1093D000FEE7FEE7FEE7FEE7FEE7FEE791B60100E7
:1093E000019201002DE9F00791E8F807B2E80210B8
:1093F0005B1854EB0C04B2E802104D4156EB0C061E
:10940000B2E802104F4158EB0C08B2E8021059EBD9
:1094100001095AEB0C0A4FF0260261EB010122EA26
:1094200001015B1854F1000455F1000556F10006E6
:1094300057F1000758F1000859F100095AF1000AE4
:1094400061EB010122EA01010B4480E8F807BDE865
:10945000F00770472DE9F00791E8F807B2E802102D
:109460005B1A74EB0C04B2E802108D4176EB0C062B
:10947000B2E802108F4178EB0C08B2E8021079EBE9
:1094800001097AEB0C0A4FF0260261EB010102EAB6
:1094900001015B1A74F1000475F1000576F1000614
:1094A00077F1000778F1000879F100097AF1000AF4
:1094B00061EB010102EA0101A3EB010380E8F80777
:1094C000BDE8F00770470A462DE9F04F92E8F00F2B
:1094D0002DE9F30F87B091E839000999A0FB0178D5
:1094E0004FF00009E3FB01894FF0000AE4FB019A09
:1094F0004FF0000BE5FB01AB0D994FF0000CE0FBCA
:1095000001BC4FF0000EE3FB01CE4FF00002E4FB84
:1095100001E24FF00006E5FB012600970A994FF0A3
:109520000007E0FB018719EB07094FF0000747EB45
:109530000707E3FB01971AEB070A4FF0000747EB19
:109540000707E4FB01A71BEB070B4FF0000747EBF6
:109550000707E5FB01B70E991CEB070C4FF000075E
:1095600047EB0707E0FB01C71EEB070E4FF00007B4
:1095700047EB0707E3FB01E7D2194FF0000747EB82
:109580000707E4FB0127F6194FF0000747EB070731
:10959000E5FB0167CDF804800B994FF00008E0FB74
:1095A00001981AEB080A4FF0000848EB0808E3FBA3
:1095B00001A81BEB080B4FF0000848EB0808E4FB80
:1095C00001B81CEB080C4FF0000848EB0808E5FB5D
:1095D00001C80F991EEB080E4FF0000848EB080871
:1095E000E0FB01E812EB08024FF0000848EB080826
:1095F000E3FB012816EB08064FF0000848EB0808CB
:10960000E4FB016817EB08074FF0000848EB080877
:10961000E5FB0178CDF808900C994FF00009E0FBCC
:1096200001A91BEB090B4FF0000949EB0909E3FB0A
:1096300001B91CEB090C4FF0000949EB0909E4FBE7
:1096400001C91EEB090E4FF0000949EB0909E5FBC2
:1096500001E9109912EB09024FF0000949EB0909E1
:10966000E0FB012916EB09064FF0000949EB090957
:10967000E3FB016917EB09074FF0000949EB090902
:10968000E4FB017918EB09084FF0000949EB0909DF
:10969000E5FB0189CDF80CA0089901F1100191E8D2
:1096A000390009994FF0000AE0FB01BA1CEB0A0CE3
:1096B0004FF0000A4AEB0A0AE3FB01CA1EEB0A0E4E
:1096C0004FF0000A4AEB0A0AE4FB01EA12EB0A0235
:1096D0004FF0000A4AEB0A0AE5FB012A0D9916EB46
:1096E0000A064FF0000A4AEB0A0AE0FB016A17EB90
:1096F0000A074FF0000A4AEB0A0AE3FB017A18EB6B
:109700000A084FF0000A4AEB0A0AE4FB018A19EB47
:109710000A094FF0000A4AEB0A0AE5FB019ACDF864
:1097200010B00A994FF0000BE0FB01CB1EEB0B0EC3
:109730004FF0000B4BEB0B0BE3FB01EB12EB0B02BF
:109740004FF0000B4BEB0B0BE4FB012B16EB0B0666
:109750004FF0000B4BEB0B0BE5FB016B0E9917EB7E
:109760000B074FF0000B4BEB0B0BE0FB017B18EBF7
:109770000B084FF0000B4BEB0B0BE3FB018B19EBD2
:109780000B094FF0000B4BEB0B0BE4FB019B1AEBAF
:109790000B0A4FF0000B4BEB0B0BE5FB01ABCDF8CD
:1097A00014C00B994FF0000CE0FB01EC12EB0C0223
:1097B0004FF0000C4CEB0C0CE3FB012C16EB0C06F1
:1097C0004FF0000C4CEB0C0CE4FB016C17EB0C079E
:1097D0004FF0000C4CEB0C0CE5FB017C0F9918EBE7
:1097E0000C084FF0000C4CEB0C0CE0FB018C19EB5F
:1097F0000C094FF0000C4CEB0C0CE3FB019C1AEB3A
:109800000C0A4FF0000C4CEB0C0CE4FB01AC1BEB16
:109810000C0B4FF0000C4CEB0C0CE5FB01BCCDF835
:1098200018E00C994FF0000EE0FB012E16EB0E062F
:109830004FF0000E4EEB0E0EE3FB016E17EB0E0722
:109840004FF0000E4EEB0E0EE4FB017E18EB0E08FF
:109850004FF0000E4EEB0E0EE5FB018E109919EB4A
:109860000E094FF0000E4EEB0E0EE0FB019E1AEBC0
:109870000E0A4FF0000E4EEB0E0EE3FB01AE1BEB9B
:109880000E0B4FF0000E4EEB0E0EE4FB01BE1CEB78
:109890000E0C4FF0000E4EEB0E0EE5FB01CE4FF01E
:1098A0002601DDE900344FF00000E6FB013024180A
:1098B0004FF0000040EB0000E7FB0140DDE90256FD
:1098C0002D184FF0000040EB0000E8FB0150361867
:1098D0004FF0000040EB0000E9FB0160DDE9048986
:1098E00018EB00084FF0000040EB0000EAFB01809D
:1098F00019EB00094FF0000040EB0000EBFB01907A
:10990000DDF818A01AEB000A4FF0000040EB000051
:10991000ECFB01A012184FF0000040EB0000EEFB42
:10992000012000FB01F01B1854F1000455F1000563
:1099300056F1000658F1000759F100085AF10009E4
:1099400052F1000A60EB000021EA0000034407988E
:1099500080E8F80711B0BDE8F08F2DE9F00791E835
:10996000F0174EF6A1514FEA4101A4FB01234FF03D
:109970000004E5FB01344FF00005E6FB01454FF024
:109980000006E7FB01564FF00007E8FB01674FF0C8
:109990000008E9FB01784FF00009EAFB01894FF06C
:1099A000000AECFB019A4FF026010AFB01FA12EBC8
:1099B0000A0253F1000354F1000455F1000556F179
:1099C000000657F1000758F1000859F100096AEB49
:1099D0000A0A21EA0A010A4480E8FC03BDE8F0070C
:1099E00070472DE9F00390E8F8134FEAEC7202F0AB
:1099F00013022CF0004C02F11301591854F100012C
:109A000055F1000156F1000157F1000158F1000134
:109A100059F100015CF100014FEAE17101F013011D
:109A200011445B1854F1000455F1000556F100068D
:109A300057F1000758F1000859F100094CF1000CEA
:109A40002CF0004C80E8F813BDE8F003704700BF2D
:109A500070B491E87800B2E802105B1854EB0C0483
:109A6000B2E802104D4156EB0C0680E878008041C8
:109A7000013070BC70472DE9F00791E8F807B2E8B3
:109A800002105B1854EB0C04B2E802104D4156EB87
:109A90000C06B2E802104F4158EB0C08B2E8021075
:109AA00059EB01095AEB0C0A80E8F80780410130B4
:109AB000BDE8F00770472DE9F00791E8F807B2E834
:109AC00002105B1A74EB0C04B2E802108D4176EBC5
:109AD0000C06B2E802108F4178EB0C08B2E80210D5
:109AE00079EB01097AEB0C0A80E8F80780414042E3
:109AF000BDE8F00770472DE9F007524290E8780082
:109B0000B1E880071740DB1918EA020854EB080493
:109B100019EA020955EB09051AEA020A56EB0A0688
:109B200078C090E87800B1E8800717407B4118EAD8
:109B3000020854EB080419EA020955EB09051AEA70
:109B4000020A56EB0A0678C080410130BDE8F007F2
:109B500070472DE9F007524290E87800B1E880079D
:109B60001740DB1B18EA020874EB080419EA020923
:109B700075EB09051AEA020A76EB0A0678C090E846
:109B80007800B1E880071740BB4118EA020874EB7F
:109B9000080419EA020975EB09051AEA020A76EBCC
:109BA0000A0678C080414042BDE8F007704790E85F
:109BB000300091E8C000A31B1340E41AF618EB1B19
:109BC0001340ED1AFF1830C0C0C17047F0B55242C3
:109BD000FFF7EDFFFFF7EBFFFFF7E9FFFFF7E7FF09
:109BE000F0BD2DE9F0073AC91668A1FB069A4FF0BF
:109BF000000CE3FB06AC4FF00007E4FB06C74FF098
:109C00000008E5FB067840F8049B56684FF0000911
:109C1000E1FB06A91CEB090C4FF0000949EB09090F
:109C2000E3FB06C917EB09074FF0000949EB0909E7
:109C3000E4FB067918EB09084FF0000949EB090924
:109C4000E5FB068940F804AB96684FF0000AE1FB9B
:109C500006CA17EB0A074FF0000A4AEB0A0AE3FBB1
:109C6000067A18EB0A084FF0000A4AEB0A0AE4FBEE
:109C7000068A19EB0A094FF0000A4AEB0A0AE5FBCB
:109C8000069A40F804CBD6684FF0000CE1FB067C46
:109C900018EB0C084FF0000C4CEB0C0CE3FB068CA3
:109CA00019EB0C094FF0000C4CEB0C0CE4FB069C80
:109CB0001AEB0C0A4FF0000C4CEB0C0CE5FB06AC5D
:109CC00080E88017BDE8F00770470A462DE9F04F9D
:109CD00092E8F00F2DE9F30F87B091E83900099968
:109CE000A0FB01784FF00009E3FB01894FF0000A67
:109CF000E4FB019A4FF0000BE5FB01AB0D994FF02F
:109D0000000CE0FB01BC4FF0000EE3FB01CE4FF076
:109D10000002E4FB01E24FF00006E5FB012600979C
:109D20000A994FF00007E0FB018719EB07094FF094
:109D3000000747EB0707E3FB01971AEB070A4FF011
:109D4000000747EB0707E4FB01A71BEB070B4FF0EE
:109D5000000747EB0707E5FB01B70E991CEB070C63
:109D60004FF0000747EB0707E0FB01C71EEB070EAC
:109D70004FF0000747EB0707E3FB01E7D2194FF06D
:109D8000000747EB0707E4FB0127F6194FF0000730
:109D900047EB0707E5FB0167CDF804800B994FF00F
:109DA0000008E0FB01981AEB080A4FF0000848EBA6
:109DB0000808E3FB01A81BEB080B4FF0000848EB79
:109DC0000808E4FB01B81CEB080C4FF0000848EB56
:109DD0000808E5FB01C80F991EEB080E4FF00008BC
:109DE00048EB0808E0FB01E812EB08024FF000081E
:109DF00048EB0808E3FB012816EB08064FF00008C3
:109E000048EB0808E4FB016817EB08074FF000086F
:109E100048EB0808E5FB0178CDF808900C994FF065
:109E20000009E0FB01A91BEB090B4FF0000949EB0E
:109E30000909E3FB01B91CEB090C4FF0000949EBE0
:109E40000909E4FB01C91EEB090E4FF0000949EBBB
:109E50000909E5FB01E9109912EB09024FF000092D
:109E600049EB0909E0FB012916EB09064FF000094F
:109E700049EB0909E3FB016917EB09074FF00009FA
:109E800049EB0909E4FB017918EB09084FF00009D7
:109E900049EB0909E5FB0189CDF80CA0089901F10E
:109EA000100191E8390009994FF0000AE0FB01BA6E
:109EB0001CEB0A0C4FF0000A4AEB0A0AE3FB01CA4A
:109EC0001EEB0A0E4FF0000A4AEB0A0AE4FB01EA15
:109ED00012EB0A024FF0000A4AEB0A0AE5FB012ADC
:109EE0000D9916EB0A064FF0000A4AEB0A0AE0FB4E
:109EF000016A17EB0A074FF0000A4AEB0A0AE3FB74
:109F0000017A18EB0A084FF0000A4AEB0A0AE4FB50
:109F1000018A19EB0A094FF0000A4AEB0A0AE5FB2D
:109F2000019ACDF810B00A994FF0000BE0FB01CB7D
:109F30001EEB0B0E4FF0000B4BEB0B0BE3FB01EB9F
:109F400012EB0B024FF0000B4BEB0B0BE4FB012B66
:109F500016EB0B064FF0000B4BEB0B0BE5FB016B0D
:109F60000E9917EB0B074FF0000B4BEB0B0BE0FBC5
:109F7000017B18EB0B084FF0000B4BEB0B0BE3FBDB
:109F8000018B19EB0B094FF0000B4BEB0B0BE4FBB8
:109F9000019B1AEB0B0A4FF0000B4BEB0B0BE5FB95
:109FA00001ABCDF814C00B994FF0000CE0FB01ECB5
:109FB00012EB0C024FF0000C4CEB0C0CE3FB012CF1
:109FC00016EB0C064FF0000C4CEB0C0CE4FB016C98
:109FD00017EB0C074FF0000C4CEB0C0CE5FB017C75
:109FE0000F9918EB0C084FF0000C4CEB0C0CE0FB3D
:109FF000018C19EB0C094FF0000C4CEB0C0CE3FB43
:10A00000019C1AEB0C0A4FF0000C4CEB0C0CE4FB1F
:10A0100001AC1BEB0C0B4FF0000C4CEB0C0CE5FBFC
:10A0200001BCCDF818E00C994FF0000EE0FB012EBA
:10A0300016EB0E064FF0000E4EEB0E0EE3FB016E1C
:10A0400017EB0E074FF0000E4EEB0E0EE4FB017EF9
:10A0500018EB0E084FF0000E4EEB0E0EE5FB018ED6
:10A06000109919EB0E094FF0000E4EEB0E0EE0FBAF
:10A07000019E1AEB0E0A4FF0000E4EEB0E0EE3FBA4
:10A0800001AE1BEB0E0B4FF0000E4EEB0E0EE4FB81
:10A0900001BE1CEB0E0C4FF0000E4EEB0E0EE5FB5E
:10A0A00001CE079800F11C0181E8C45FBDE8F80308
:10A0B00080E8F8030AB0BDE8F08F00BF2DE9F05F3B
:10A0C0000546002092469B46884606468146402427
:10A0D0001BE0284641464746224600F075F85346A5
:10A0E0005A46C01A914110D311461846224600F034
:10A0F00016F82D1A67EB01084F4622460120002171
:10A1000000F00DF817EB00094E41201EA4F10104E8
:10A11000DFDC484631462A464346BDE8F09F202A08
:10A1200004DB203A00FA02F1002070479140C2F1AE
:10A13000200320FA03F319439040704740EA0103DB
:10A140009B0703D009E008C9121F08C0042AFAD2ED
:10A1500003E011F8013B00F8013B521EF9D27047B1
:10A16000D2B201E000F8012B491EFBD27047002259
:10A17000F6E710B513460A4604461946FFF7F0FF06
:10A18000204610BD421C10F8011B0029FBD1801A8B
:10A19000704730B504460020034600E05B1C934244
:10A1A00003D2E05CCD5C401BF8D030BD10B5484315
:10A1B000044606F075F8002805D00021002C02D0D6
:10A1C000641E0155FAE710BD202A04DB203A21FA6B
:10A1D00002F00021704721FA02F3D040C2F12002C0
:10A1E0009140084319467047064C074D06E0E06869
:10A1F00040F0010394E8070098471034AC42F6D3CE
:10A20000FFF702F8906C0200B06C020070B58C1879
:10A2100010F8015B15F0070301D110F8013B2A117A
:10A2200006D110F8012B03E010F8016B01F8016B67
:10A230005B1EF9D12B0705D40023521E0DD401F863
:10A24000013BFAE710F8013BCB1A921C03E013F82C
:10A25000015B01F8015B521EF9D5A142D8D3002061
:10A2600070BD00002DE9F047CC7F0D78C0B00B46E3
:10A2700025F0070504F03F0493F8028049788DF833
:10A28000405044F040041D7F93F803C0D3F804E02D
:10A290009F68D3F810A0DE688DF841108DF85F40FC
:10A2A00011469C695A698DF842808DF85C5093F88C
:10A2B0001D809B7F8DF843C081466D466846CDF872
:10A2C00044E01297CDF850A0159216948DF85D8059
:10A2D0008DF85E30139600F00FFB0FCD18AC0FC455
:10A2E00095E80F0084E80F006846012100F018FB94
:10A2F00018AD08A8002100F013FB0FCD20AC0FC44F
:10A3000095E80F0084E80F0028A8012100F008FB61
:10A3100018AF0DF140084FF0060A002417F8016D40
:10A3200046FA0AF505F001056C40224620A9684668
:10A33000FFF74CFC224628A908A8FFF747FC08AA0B
:10A34000694630A8FFF74EF808AA10466946FFF79D
:10A3500081F828AA20A938A8FFF744F828AA1046AF
:10A3600020A9FFF777F838A9084608AAFFF7ACF844
:10A3700028A9084630AAFFF7A7F838AA28A920A8D4
:10A38000FFF730F828A938AA0846FFF763F820A994
:10A390000846FFF798F828A90846FFF794F828A977
:10A3A00018AA0846FFF790F830A90846FFF78BF87F
:10A3B00008A938A8FFF787F838AA30A96846FFF738
:10A3C00083F830A938AA0846FFF744F830A908A84E
:10A3D000FFF7C3FA08A9084638AAFFF703F808A947
:10A3E0000AF1FF3A30AA0846FFF76EF8BAF1FF3FCC
:10A3F0002C4695D147454FF0070A8FD108A908464A
:10A40000012200F097FA08AA69466846FFF75CF84F
:10A410006946484600F09CFB40B0BDE8F08700BFAD
:10A42000014AFFF71FBF00BF706B020038B50C4632
:10A43000054600F0A5FB204600F0A4FC04F1A801AD
:10A440002046402200F048FD29462046202200F008
:10A4500043FD21462846BDE8384000F091BB00BFCF
:10A46000402A2DE9F84316460C46054600F20982BB
:10A47000002A00F03382671E05F16702002100E028
:10A48000014617F8013F481C83F03603B04202F83A
:10A49000013FF5D3402808BF05F1680700F0A3800D
:10A4A00001F1690E8B1C05EB0E01402BC1F100017F
:10A4B000C0F1400201F0030188BF0122914228BF90
:10A4C0001146062A904600F2CE8105F1680705EB99
:10A4D000000C3621012A8CF8681000F0F18105EBA0
:10A4E0000309022A03F1010C89F868101DD005EB5D
:10A4F0000C09032A03F1020C89F8681015D005EB4A
:10A500000C09042A03F1030C89F868100DD005EB3F
:10A510000C09062A03F1040C89F8681005D105EB33
:10A520000C0903F1050C89F86810424558D0402BFE
:10A53000A8EB0208C0F13F00A8F1040388BF002087
:10A540009B08801A013302284FEA830935D97244E7
:10A550004FF03630012B05EB0201A8502AD0022B18
:10A56000486027D0032B886024D0042BC86021D0FA
:10A57000052B08611ED0062B48611BD0072B886174
:10A5800018D0082BC86115D0092B086212D00A2BED
:10A5900048620FD00B2B88620CD00C2BC86209D0FC
:10A5A0000D2B086306D00E2B486303D00F2B886356
:10A5B00000D0C863C845CC4412D005EB0C020CF1A6
:10A5C00001033621402B82F8681009D0EA180CF1FB
:10A5D0000203402B82F8681002D02B4483F86810E5
:10A5E000002E00F06F81221D05F1A80305F1AC01DA
:10A5F000A14288BF9A4200F25381062E40F2508158
:10A60000331F21689B08013381F05C31012B4FEA35
:10A610008302C5F8A81066D06168022B81F05C3116
:10A62000C5F8AC105FD0A168032B81F05C31C5F890
:10A63000B01058D0E168042B81F05C31C5F8B4103B
:10A6400051D02169052B81F05C31C5F8B8104AD092
:10A650006169062B81F05C31C5F8BC1043D0A1695B
:10A66000072B81F05C31C5F8C0103CD0E169082BA4
:10A6700081F05C31C5F8C41035D0216A092B81F016
:10A680005C31C5F8C8102ED0616A0A2B81F05C31AC
:10A69000C5F8CC1027D0A16A0B2B81F05C31C5F82E
:10A6A000D01020D0E16A0C2B81F05C31C5F8D410B9
:10A6B00019D0216B0D2B81F05C31C5F8D81012D068
:10A6C000616B0E2B81F05C31C5F8DC100BD0A16BF7
:10A6D000102B81F05C31C5F8E01004D1E16B81F002
:10A6E0005C31C5F8E410B24218D014F82300A91860
:10A6F000531C80F05C00B34281F8A8000ED2E05CED
:10A70000E918931CB34280F05C0281F8A82005D2BE
:10A71000E25C2B4482F05C0283F8A820402E00F01B
:10A72000988006F1A8042A19711C4029C2F1000280
:10A73000C6F1400302F0030288BF01239A4228BFFA
:10A740001A46062B9E4600F29780A8195C22012B20
:10A7500080F8A82000F0B28005EB010C022B01F17B
:10A7600001008CF8A8201CD005EB000C032B01F194
:10A7700002008CF8A82014D005EB000C042B01F18A
:10A7800003008CF8A8200CD005EB000C062B01F17F
:10A7900004008CF8A82004D105EB000C481D8CF8AF
:10A7A000A820734555D04029AEEB030EC6F13F06F5
:10A7B000AEF1040288BF00269208F61A0132022E7A
:10A7C0004FEA820C35D92344012A4FF05C3405EB63
:10A7D0000301EC502AD0022A4C6027D0032A8C6057
:10A7E00024D0042ACC6021D0052A0C611ED0062A70
:10A7F0004C611BD0072A8C6118D0082ACC6115D077
:10A80000092A0C6212D00A2A4C620FD00B2A8C62E1
:10A810000CD00C2ACC6209D00D2A0C6306D00E2A6B
:10A820004C6303D00F2A8C6300D0CC63E6456044B0
:10A830000FD02918431C5C22402B81F8A82008D097
:10A840002B440230402883F8A82002D0284480F806
:10A85000A820284600F096FA394628464022BDE84E
:10A86000F84300F039BB84460A4605F168076046A4
:10A87000002A3FF45CAE2AE613463046002B92D005
:10A8800063E700F07FFA32462146284605F1E804E6
:10A8900000F022FB2046294600F072F92026EAE566
:10A8A000711E214405F1A702013C14F8013F83F019
:10A8B0005C038C4202F8013FF7D12FE7084670E7AE
:10A8C0009C4632E66B4203F00303304601214FF011
:10A8D000400EA824002B3FF466AF36E700F168076E
:10A8E0007A4202F00302B4464FF0680E01234FF0A3
:10A8F0004008BCE700F0F0BA0B6803604B684360A7
:10A900008B688360CB68C3600B6903614B694361EB
:10A910008B698361CB6923F00043C361704700BF3B
:10A92000002380E80A008360C360036143618361A0
:10A93000C3617047F0B5A1B00546684617460E469C
:10A94000FEF7C1FD694618A8FEF7BDFD18A9084627
:10A95000FEF7B9FD324618A908A8FEF7B5FD6A460C
:10A9600008A96846FEF7B0FD694618A8FEF7ABFDDA
:10A9700008AA104618A9FEF7A7FD08A918A8FEF70F
:10A98000A2FD18A90846FEF79EFD18A90846FEF785
:10A990009AFD18A90846FEF796FD18A90846FEF785
:10A9A00092FD08AA18A91046FEF78EFD022408A9F8
:10A9B00018A8FEF788FD18A90846FEF784FD18A917
:10A9C0000846FEF780FD18A90846FEF77CFD18A989
:10A9D0000846FEF778FD013C18A9E9D110A808AA9D
:10A9E000FEF772FD042410A918A8FEF76CFD18A943
:10A9F0000846FEF768FD18A90846FEF764FD18A989
:10AA00000846FEF760FD18A90846FEF75CFD013C0C
:10AA100018A9E9D110AA0846FEF756FD022418A984
:10AA20000846FEF750FD18A90846FEF74CFD18A988
:10AA30000846FEF748FD18A90846FEF744FD18A988
:10AA40000846FEF740FD013CE9D118A908AA10A864
:10AA5000FEF73AFD0A2410A918A8FEF734FD18A93C
:10AA60000846FEF730FD18A90846FEF72CFD18A988
:10AA70000846FEF728FD18A90846FEF724FD013C0C
:10AA800018A9E9D110AA08A8FEF71EFD142408A9E8
:10AA900018A8FEF718FD18A90846FEF714FD18A916
:10AAA0000846FEF710FD18A90846FEF70CFD18A988
:10AAB0000846FEF708FD013C18A9E9D108AA084696
:10AAC000FEF702FD0A2418A90846FEF7FCFC18A9A7
:10AAD0000846FEF7F8FC18A90846FEF7F4FC18A98A
:10AAE0000846FEF7F0FC18A90846FEF7ECFC013C0E
:10AAF000E9D118A9084610AAFEF7E6FC18A90846ED
:10AB000067B9FEF7E0FC18A90846FEF7DCFC324600
:10AB100018A92846FEF7D8FC21B0F0BDFEF7D3FCFB
:10AB200018A90846FEF7CFFC18A90846FEF7CBFC8B
:10AB300018A90846FEF7C7FC18A90846FEF7C3FC8B
:10AB40006A4618A92846FEF7BFFC21B0F0BD00BF39
:10AB500038B50C4605460846FEF743FF23682B60D0
:10AB600063686B60A368AB60E368EB6023692B618B
:10AB700063696B61A369AB61E369EB6138BD00BFD9
:10AB8000F8B50A6E0C46531C11448026382B054636
:10AB900081F8206000F2BE8004F1200603F120005D
:10ABA00022185242C3F13B0102F003028A4228BF3D
:10ABB0000A46062900F2E1800A46E7184FF0000E27
:10ABC000012A87F820E003F1010724D004EB070CE9
:10ABD000022A03F102078CF820E01CD004EB070CDA
:10ABE000032A03F103078CF820E014D004EB070CD0
:10ABF000042A03F104078CF820E00CD004EB070CC6
:10AC0000062A03F105078CF820E004D104EB070CB9
:10AC10009F1D8CF820E091424ED0A1EB020EAEF1C8
:10AC20000401C3F13A0389089B1A0131022B4FEA50
:10AC3000810C31D910440023012904EB0002235078
:10AC400027D00229536024D00329936021D00429FE
:10AC5000D3601ED0052913611BD00629536118D07B
:10AC60000729936115D00829D36112D009291362ED
:10AC70000FD00A2953620CD00B29936209D00C29FA
:10AC8000D36206D00D29136303D00E29536300D07D
:10AC90009363E64567440FD0E2197B1C00213B2BF0
:10ACA00082F8201008D0E218BB1C3B2B82F8201041
:10ACB00002D0234483F82010636E4FEA537E580B72
:10ACC0005A095F0DDB0084F85D0084F85F3031467F
:10ACD00084F85BE084F85C7084F85E20204600F025
:10ACE0005DFA23681BBA2B6063681BBA6B60A368AC
:10ACF0001BBAAB60E3681BBAEB6023691BBA2B611C
:10AD000063691BBA6B61A3691BBAAB61E3691BBAC8
:10AD1000EB61F8BD3F2B25D82344901C002140282F
:10AD200083F820101ED02044D31C402B80F8201024
:10AD300018D0E018131D402B80F8201012D0E01816
:10AD4000531D402B80F820100CD0E018931D402B91
:10AD500080F8201006D02344382A83F8201001D12F
:10AD600084F85F1004F120063146204600F016FA00
:10AD70003A2803467FF612AF9EE71F46002A3FF4AB
:10AD80004CAF1AE7F0B40D4A0260A2F162620C4BBC
:10AD90000C4F0D4E0D4D0E4C0E494360A2F5112285
:10ADA0000023A2F64E128760C6600561446181618E
:10ADB000C26103664366F0BC704700BF67E6096A7C
:10ADC00085AE67BB72F36E3C3AF54FA57F520E51CC
:10ADD0008C68059BABD9831F2DE9F04F824602F1A9
:10ADE000100090E8014283B0A1F1040B0AF1400485
:10ADF000D1680091D369D2F80880019492E80210DA
:10AE0000774602E08C46304629465AF8046B5BF8D8
:10AE1000044FD7614FEAF02587EA090E85EAB0159D
:10AE2000264485EA70650EEA000E8EEA070E354468
:10AE300075441D444FEA7134009BC2F8189041EAF2
:10AE40000C0606EA080684EAB10401EA0C0E2B445B
:10AE500046EA0E0684EAB154344450611E4613613A
:10AE60003B464F4681460198C2F80C8025448245F6
:10AE7000CDF80080C2F808C051601560E046C1D12D
:10AE800003B0BDE8F08F00BFF0B50022061F1546E5
:10AE9000931E013202F00F0103F00F03073D50F83B
:10AEA00021E050F8237005F00F054FEABE4450F83A
:10AEB0002530756884EAFE144FEAF7412B4484EA92
:10AEC000DE0481EA7741234481EA97210B44102A6A
:10AED00046F8043FDBD1F0BDF8B5436E0646006E80
:10AEE000134414460D467366C8B13F2800F29380A0
:10AEF000002A00F0848000F11F03334401E0002C9D
:10AF00007DD0013015F8012B03F8012F402804F102
:10AF1000FF34F4D106F12001304600F03FF9002C57
:10AF20006DD022462946304600F07CF8231A2B4487
:10AF3000002864D0221D121A2A4406F1200106F1CD
:10AF40002407BB4238BF91425BD3082859D9021F5E
:10AF5000196831629208013259687162022A4FEA17
:10AF6000820135D09C68B462032A31D0DC68F46277
:10AF7000042A2DD01C693463052A29D05C697463C6
:10AF8000062A25D09C69B463072A21D0DC69F463C2
:10AF9000082A1DD01C6A3464092A19D05C6A7464BA
:10AFA0000A2A15D09C6AB4640B2A11D0DC6AF464B6
:10AFB0000C2A0DD01C6B34650D2A09D05C6B7465AE
:10AFC0000E2A05D09C6BB4650F2A01D0DC6BF465AA
:10AFD000884203EB010512D013F8222074184B1C91
:10AFE000984284F820200AD9F2188B1C984269787C
:10AFF00082F8201003D93344AA7883F820203066E1
:10B00000F8BD2C4406F11F0213F8011B02F8011FC2
:10B01000A342F9D1F3E740283FF47CAF002C80D164
:10B02000EDE700BF2DE9F04F9BB03F2A1646019295
:10B0300040F2AB8005460C46D0F81090D0F8148052
:10B04000D0F818C0009690E80E04C06927686668BA
:10B05000D4F808E0D4F810B002910392E168A26A33
:10B060000493CDF814A0E36AD4F814A0CDF8189096
:10B07000CDF81C80D4F81890D4F81C80CDF820C0EE
:10B080000990D4F820C0606A3FBA36BA9EFA8EFEA4
:10B0900009BA9CFA8CFC00BA12BA1BBA9BFA8BFB59
:10B0A0009AFA8AFA99FA89F998FA88F80A970B961F
:10B0B000CDF830E00D91139014921593CDF838B07F
:10B0C000CDF83CA0CDF84090CDF84480CDF848C0F4
:10B0D000304ED4F830C0D4F834E0A76BE36B9CFA60
:10B0E0008CFC9EFA8EFE1BBA3FBA02AA0AA9304611
:10B0F000CDF858C0CDF85CE018971993FFF76CFEB7
:10B10000403440360AA8FFF7BFFE304602AA0AA91B
:10B11000FFF762FE204B9E42F3D1009BA8682F6888
:10B1200002996E68039A403B0093049B0344E868CD
:10B13000AB60864605980EEB000A2869C5F80CA09E
:10B14000864606980EEB00096869C5F81090864699
:10B15000079839440EEB0008AF690898296032441B
:10B1600007EB000CEE6909986A603044009EC5F850
:10B1700014803F2EC5F818C0E8613FF667AF019B09
:10B1800003F03F001BB0BDE8F08F10461BB0BDE8D8
:10B19000F08F00BF906B0200506C02002DE9F0416F
:10B1A0008E68CD680C698A69CB69D1F800E04F6878
:10B1B00098B08046486936BA2DBA24BA00BA12BA95
:10B1C0001BBA0A960B95D8F80060D8F804500C9476
:10B1D0009EFA8EFED8F808400D903FBAD8F80C00C1
:10B1E0000E920F93D8F81020D8F8143000960195DD
:10B1F000D8F81860D8F81C50CDF820E009970294D0
:10B2000003900492059306960795486B0A6BD1F854
:10B2100020E04F6A8E6ACD6A8C6BCB6B00BA11BA94
:10B2200015902B4814919EFA8EFE2DBA24BA1BBAA3
:10B230003FBA36BA6A4608A913951694CDF840E08D
:10B240000446119712961793FFF7C6FD04F1C00547
:10B25000403408A8FFF718FE20466A4608A9FFF701
:10B26000BBFDAC42F4D1D8F80410019ED8F8000020
:10B27000009FD8F80850D8F80C30039C029A31444B
:10B280003844049EC8F80410D8F81010C8F800001C
:10B290002A442344D8F81800069CD8F81450059F77
:10B2A000C8F808200E44079AD8F81C10C8F80C30CB
:10B2B00020443D441144C8F818000020C8F810602C
:10B2C000C8F81450C8F81C1018B0BDE8F08100BFD1
:10B2D000906B02002DE9F04700268AB0DFF850910C
:10B2E000B0464FF48075012437460696284607F08D
:10B2F0000DF838B1D9F80403204203D0284606F0EF
:10B30000FBFF26432D1D64007F1CADB2082FEDD33B
:10B310004FF4BE74204606F0F9FF48B1204606F00F
:10B32000EBFF46F0004606AA0121002006F0D0FF00
:10B33000404D16F0FF0F15D00127002437420DD0E5
:10B3400009EB8401D1F81005D1F81015C0F30420E1
:10B3500055F82420C1F3014102B190477F00641CDD
:10B36000082CEBD3002E5FDA4FF0FF30CDF81080C1
:10B3700054E0281910F8507F90F9000027F0C00819
:10B38000401C3BD007A9404605F002FF10B34FEA2E
:10B390009719404602F0D0F955F820701FB1B9F165
:10B3A000030F03D006E0B9F1030F27D104A94046EB
:10B3B00005F0F6FE4FF0A04101EB8800D0F8000741
:10B3C00006A9C0F3014A404605F0E2FE18B1BAF101
:10B3D000020F03D012E0BAF1030F0FD1B9F1030F3E
:10B3E00008D1BAF1020F1DD00221404606F053FFEA
:10B3F000761CF6B217B149464046B847641C042C87
:10B40000B7D3002E10D06A460121002006F060FF5D
:10B4100006990098884207D0069004980026344682
:10B420000790A6E70321E0E70AB0BDE8F087000037
:10B4300000600040DC21002000F01F02012191404B
:10B440004009800000F1E020C0F88012704700F051
:10B450001F02012191404009800000F1E020C0F866
:10B460000011704700F01F02012191404009800047
:10B4700000F1E020C0F8001270474907090E0028CB
:10B4800006DA00F00F0000F1E02080F8141D70478C
:10B4900000F1E02080F800147047000070B54FF410
:10B4A0008076304606F0D2F8114CB50560B13046D2
:10B4B00006F0D3F80120C5F80803607920B901200F
:10B4C00060712168002088474FF48276304606F08C
:10B4D000BDF800280AD0304606F0BFF80220C5F8B3
:10B4E00008032168BDE870400120084770BD0000D6
:10B4F000641C0020064882B00021016000680090B2
:10B50000044800680449C0B2496802B00847000016
:10B5100000D1004008D500406C1C002007480021E5
:10B52000C0F84011C0F84411C0F84811C0F84C11DF
:10B53000C0F80011C0F8041108F098BC00100140D8
:10B540002DE9FE434FF48278404607F009F84C4F4E
:10B5500000254C4C012600B3404607F009F894F84A
:10B560002E0010B194F82F10D1B18DF80050616801
:10B5700001912189ADF80810E26832B1218B618315
:10B5800062602181E56010B102E0257400E03E6058
:10B5900021686846884784F82F5094F82E0060B3DD
:10B5A0004FF48077384606F0DBFF30B3384606F0BC
:10B5B000DFFF628B94F82D108A420AD9A2EB0100BA
:10B5C00080B260832289A2EB0000626802EB400037
:10B5D00005E007D1E06828B184F82F60658306F0A4
:10B5E000ADFF04E08A4202D184F82F6065834046B3
:10B5F00006F0BEFF2248001D06604FF488773846EB
:10B6000006F0AEFF48B1384606F0B2FF25740220BE
:10B610008DF800002168684688474FF48A773846DD
:10B6200006F09EFF28B1384606F0A2FF2574BDE85B
:10B63000FE834FF000484FF48C7967691DE000BF2E
:10B64000B7FA87F028FA00F109EB80058F43284606
:10B6500006F086FF88B1284606F08AFFA5F58C75AE
:10B66000E8088DF8040045F38000401C8DF8006068
:10B670008DF80500216868468847002FE0D1D6E79D
:10B68000007000403822002008F03EBB07F02EB8C2
:10B69000F0B5A848A74B012600781B1D1A1D4FF0D6
:10B6A000805106280BD11C78240708D11478C4F3E4
:10B6B0000314032C06D0042C04D0052C02D0062839
:10B6C00007D011E0B1F824439B4DC4F304242C604F
:10B6D00002E01C78240707D11478C4F30314032C68
:10B6E00002D1974D954C6C67D1F83051D1F8444256
:10B6F000944FC4F342343C6006280CD11C782407D4
:10B7000009D11478C4F30314032C04D18E4C276898
:10B7100027F0807727604FF080470024C7F80C415E
:10B72000C7F81041874F3F1F3C60062807D11F789C
:10B730003F0704D11778C7F30317032F02D0062859
:10B7400008D01FE0DFF8FCC103270CF1640CCCF833
:10B75000007007E01F783F0714D11778C7F303176D
:10B76000032F0FD1DFF8E4C10527CCF80070774F25
:10B7700078373E60754F08373C600CF1040C3F276A
:10B78000CCF80070724F3F68DFF8C8C1CCF8007089
:10B790006F4F3F1D3F680CF1040CCCF800706C4FEC
:10B7A00008373F680CF1040CCCF80070684F0C3778
:10B7B0003F680CF1040CCCF80070654F10373F68FF
:10B7C0000CF1040CCCF80070614F14373F680CF199
:10B7D000040CCCF800705E4F18373F68DFF874C176
:10B7E0000CF1200CCCF80070594F1C373F680CF15D
:10B7F000040CCCF80070564F20373F680CF1040C55
:10B80000CCF80070524F24373F680CF1040CCCF890
:10B8100000704F4F28373F680CF1040CCCF80070D3
:10B820004B4F2C373F680CF1040CCCF80070484F9C
:10B8300030373F68DFF81CC10CF1400CCCF80070C9
:10B84000434F34373F680CF1040CCCF80070404F84
:10B8500038373F680CF1040CCCF800703C4F3C3793
:10B860003F680CF1040CCCF80070394F40373F684A
:10B870000CF1040CCCF80070DFF8DCC0FB27CCF82E
:10B880000070062813D11F783F0710D11778C7F32F
:10B890000317032F03D0042F01D0052F07D1D1F8B0
:10B8A0005872DFF8B8C007F04F07CCF800702C488A
:10B8B0000268D20702D06FF001020260062D08D1A3
:10B8C000D1F83401062804D12648016841F480618A
:10B8D00001604FF01021D1F80002002803DBD1F8FD
:10B8E0000402002822DA204A166020480368002B50
:10B8F000FCD01523C1F800320568002DFCD0C1F83A
:10B90000043201680029FCD0146001680029FCD0D1
:10B91000BFF34F8F0C48F0380168154A01F4E0611D
:10B9200011430160BFF34F8F00BFFDE7124911487B
:10B930000860F0BDE00F00F0403501400DF0ADBAF9
:10B9400000C007403C050040FCED00E01056004000
:10B950000404001020C5004018F50040E40E00402B
:10B96000000400403C17004004E5014000E40140B1
:10B970000400FA050090D003AC1D002002E008C8C6
:10B98000121F08C1002AFAD170477047002001E059
:10B9900001C1121F002AFBD170470000012120289D
:10B9A00003DA81400548014003E0402802DA2038EC
:10B9B000814009B10120704700207047FC06FFBD9F
:10B9C000082806D228B1012803D0042801D001207C
:10B9D000704700207047000070B58CB0044600200E
:10B9E00001900290089009900A90069007900390A9
:10B9F000049005906088ADF80C0060680490208881
:10BA000009AA06A903F07CFE0646A07B10B1022815
:10BA100004D005E026B130460CB070BD0A2E2ED001
:10BA200028B11B4D012813D0022828D12CE001A9F0
:10BA300006A803F06DFE0028EED1A2890299A06845
:10BA4000FEF77CFB06A803F01BFE0028E4D116E0FD
:10BA5000A289D4E90101FEF771FBA08903A9C01CEA
:10BA6000800805902088ADF80E000A2E06A808D0A0
:10BA700003F072FE0028CFD16868401C6860002087
:10BA8000CAE703F070FEF5E706A803F019FEF1E738
:10BA9000EC1C002002680B685A40026042684B6848
:10BAA0005A40426082688B685A408260C268C968A6
:10BAB0004A40C2607047800701D0002070470120D3
:10BAC0007047C3688B4206D811440069491E814201
:10BAD00001D8012070470020704710B538B1012807
:10BAE00001D002280AD1BDE8104004F0E1B80020DE
:10BAF00004F0DEF8BDE8104003F082B910BD00008C
:10BB000010B503F04FFA90F8400110B1002000F09A
:10BB10002BF80E480178002917D040884FF4FA72AC
:10BB2000410CC003801841F1000152000023FEF7D0
:10BB3000C5FA014606480022006800F0A1FA002874
:10BB400003D0BDE8104000F0ADB910BDDC1C0020F2
:10BB5000104702000348407808B102F079B802F0BB
:10BB6000EDBA0000BC1C002038B52849044601EBA2
:10BB7000840250788DF8010011F8240000B10120F2
:10BB8000234D8DF800002878D8B191F828000128BD
:10BB900017D9401EA04214D950884FF4FA72410CB4
:10BBA000C003801841F1000152000023FEF786FA1D
:10BBB00001461848621C406800F062FA08B100F0C3
:10BBC00071F914B96868401C686003F0EBF990F8EB
:10BBD0004D1189B19DF8011090F84C01814203D0BC
:10BBE0009DF80000012807D168680521B0FBF1F23B
:10BBF00001FB1200002807D1A9686846002903D07C
:10BC00002A78002A00D0884738BD00002024002070
:10BC1000DC1C00201047020010B5044603F088FB2E
:10BC20000A492246A1F11004E06872DF08B100F071
:10BC300039F9E0680021007873DF112805D0002869
:10BC400003D0BDE8104000F02DB910BDCC1C002081
:10BC5000064810B5C068007874DF082802D008B123
:10BC600000F020F9BDE8104002F02EBBBC1C002003
:10BC7000F0B587B0044603F095F9224E0546F0680A
:10BC8000007874DF43F20407082804D0B84202D0D9
:10BC900008B100F007F9207810B1012812D023E094
:10BCA0006078002105EB801090F90120012077DFFA
:10BCB000B84202D008B100F0F5F8124A60781032AC
:10BCC00000210FE095F84C01002105EB801090F960
:10BCD0000120012077DF08B100F0E4F8094A60781C
:10BCE0001032012102F082F9002004F055F9727837
:10BCF0000121684603F024FF6846FFF78DFF07B077
:10BD0000F0BD0000BC1C002010B501220221002063
:10BD100000F07CFF08B1072810D107220221012082
:10BD200000F074FF08B1072808D100210A22084654
:10BD300000F06CFF08B1072800D1002010BD000002
:10BD40002DE9F0470E4602C89708491C4FEA8108C2
:10BD50000546002407E000BF06EB840007F08BFBDC
:10BD600045F82400641CBC42F6D34FF001090026BC
:10BD700026E000BF05EB8400BE4250F8040C03D15E
:10BD800009F10109002605E026B1062F10D9042E7D
:10BD90000BD00DE04FEA30600B4907F00DFF0B4A66
:10BDA00012F8091080EA016002E0074907F004FF79
:10BDB000E11B55F82110414045F82410641C761C05
:10BDC0004445D7D3BDE8F087EE440200EE450200BB
:10BDD000022000F07DBE000070B50024064D06E094
:10BDE0006868012110F8340006F032FD641C2878E0
:10BDF0008442F5D3002070BD781C0020F8B51546AC
:10BE00000C460646052A01D20720F8BD06F01CFEA6
:10BE100018B906F0E1FD0028F7D1124900224E6062
:10BE20000C708D60C1E90422C1E906220E4D0DE0BF
:10BE300006EBC4002968009181788DF80110007824
:10BE40000A4A694606F056FD0028DED1641EE4B2B7
:10BE5000EED2BDE8F84004480021054A001D00F07C
:10BE6000BDB80000781C0020E04402002DFC010059
:10BE700021DE010072B609480068C00700D000BE8C
:10BE8000BFF34F8F0548E4380168054A01F4E061CB
:10BE900011430160BFF34F8F00BFFDE7F0ED00E0FD
:10BEA0000400FA050EB500210091CDE901106A46A3
:10BEB00044F20100FFF7DEFF0EBD00002DE9F84F50
:10BEC000254C8146924660880E46814241D8002723
:10BED0004FF6FF788DF80070684600F025F922785B
:10BEE0006078A188884201DA401C00E00020C0B2DE
:10BEF000904204D19DF8000000F03AF927E06578FF
:10BF00006078884201DA401C00E0002060709DF8F3
:10BF1000000000F02DF9454519D0A068B9F1000FD7
:10BF200040F835A00DD066B16188E068324605FB67
:10BF300001004946FEF702F9A06800EBC5008680C3
:10BF400002E000EBC50087800020BDE8F88F0420E8
:10BF5000FBE70920F9E70000981C002010B50E4C03
:10BF600003E0401C00E000202070207861788142CE
:10BF700010D022786188E068A36802FB010003EB1F
:10BF8000C20153F83220898890472078A1888842DE
:10BF9000E9DAE6E710BD0000981C002030B5CB00C0
:10BFA00008339DB293074FF0000401D0072030BD45
:10BFB000044B9A602A44DA605C701C705880998047
:10BFC000002030BD981C0020401A20F07F407047B0
:10BFD000014800687047000004150140074B9B783A
:10BFE00023B12AB120B10068037C1BB1082070473F
:10BFF000072070474174426100207047882200206A
:10C0000070B5012670044FF0E0210024C1F88001D2
:10C01000174D4010C5F84803C5F808036E602F207F
:10C0200006F00EFCAE60134D2F20AC6006F008FC4D
:10C030001148AC700B210470447081706C602C70DE
:10C040006C701420FFF7F8F907211420FFF715FA98
:10C050001420FFF7FCF90948046007211120FFF7BD
:10C060000CFA0648001F0068A860002070BD0000A0
:10C0700000100140A81C0020882200200815014063
:10C080002DE9FC47DFF8789099F8023073B368B374
:10C09000052902D20720BDE8FC87436933B3437CFE
:10C0A000012B25D0002704460025884616468DF82A
:10C0B0000050684600F038F801A807F091FFC8B1B9
:10C0C000012101700F4944600968C0E90218C0E904
:10C0D00004769DF8040089F801009DF8000000F046
:10C0E00047F81420FFF7BEF92846D4E70820D2E726
:10C0F0000F46D8E704259DF8000000F039F8F3E773
:10C1000088220020041501400649897839B130B1F0
:10C11000416921B100210174022107F083BE08208A
:10C12000704700008822002030B5EFF3108172B60E
:10C130000D4A9468012324B10370002900D162B62E
:10C1400030BD93604FF0E023D3F88051074C254079
:10C150001560C3F88041D3F8844154605A17C3F87E
:10C16000842100220270E8E794230020FC06FFBD32
:10C170000B498A68002A11D000280FD1EFF31080F4
:10C1800072B60B684FF0E022C2F800314B68C2F87B
:10C19000043100228A60002800D162B67047000096
:10C1A000942300202DE9F04788B00D46DDE91561A4
:10C1B000DDE91397DDE9108CDDF848A0002409B112
:10C1C000102904D948F2625008B0BDE8F087083061
:10C1D000012D03D085B148F21750F5E7CDE905618F
:10C1E00002AD014685E88C00CDE9008C4B465246F5
:10C1F0000E4801F0D6F916E0CDE904610697CDE9C5
:10C200000223CDE9008C01464B465246074801F017
:10C210006FF920B1012804D048F2165403E000243D
:10C2200001E048F260542046CEE70000FC460200E0
:10C2300010B543685A88802A07D0C02A05D0B2F5C5
:10C24000807F02D048F2185010BD1B78022B02D01C
:10C2500048F2035010BDD208083000F0FCFE002068
:10C2600010BD10B5083000F0EFFE002010BD70B515
:10C270001446049D2A68A24202D248F2145070BDAE
:10C28000220708D042681278032A04D0022A02D07A
:10C2900048F2115070BD224600F052F80028F9D142
:10C2A0002C6070BD70B5044640680D46002641887C
:10C2B000802907D0C02905D0B1F5807F02D048F28F
:10C2C000185070BD0078042806D0052804D048F224
:10C2D00003562572304670BD012D03D015B148F2CA
:10C2E000175070BD0020207204F10C0004F029FCEE
:10C2F000EFE710B542681378042B04D0052B02D069
:10C3000048F2035010BD037A0C305288012B02D042
:10C3100004F01CFC01E004F07FFCBDE8104007F0D5
:10C32000F5B910B541680978042904D0052902D06F
:10C3300048F2035010BD0C3004F0F8FB002010BD93
:10C340002DE9F04744682478042C05D0052C03D04F
:10C3500048F20250BDE8F0870446002588461F4693
:10C360001646100710D06FF0210007E07B1908EB8C
:10C370000502217A484604F003F818B1BDE8F047F9
:10C3800007F0C4B9103501E004F10C09B542EDD352
:10C390000020DFE72DE9FC470025178806461580B9
:10C3A00090F82D001446894630B13A462146484659
:10C3B00000F0E6F8051E09D1B0784FF00C0A18B36A
:10C3C0002088C846001DB84202D95046BDE8FC8707
:10C3D000684679DF0028F9D12088032108F8001089
:10C3E00020881921401C80B2208008F80010208885
:10C3F000401C80B2208000EB0801BDF8000007F06F
:10C4000079FD218808442080F0780222C8B1218873
:10C4100096F9033001F1030C4846BC45D5D8425487
:10C4200021884FF0010C491C89B2218000F801C01D
:10C430002188491C89B2218009F801302088401CDC
:10C4400020807068B8B1218890F9003001F1030CA8
:10C450004846BC45B9D8425421880A22491C89B2B1
:10C46000218042542188491C89B2218009F8013079
:10C470002088401C2080308950B1CDE900474B46D0
:10C480000622022106F1080007F0C2FD051E9DD11B
:10C49000308A50B1CDE900474B460722032106F10F
:10C4A000100007F0B5FD051E90D1308B50B1CDE9DD
:10C4B00000474B461522142106F1180007F0A8FD8D
:10C4C000051E83D1306A30B13B462246494601F011
:10C4D00056FB051EDBD1706A30B13B462246494609
:10C4E00003F014FF051ED2D196F82C0038B13B465C
:10C4F00022464946304607F02FFA051EC7D130784C
:10C5000038B13B4622464946304604F067FD051ED9
:10C51000BDD128465AE7000070B5040012D001468C
:10C520001C221448FDF70AFE1248134D05602068CE
:10C5300050B17ADF002806D1206801682960406880
:10C54000686005E00E2070BD0B487BDF0028FAD143
:10C5500008484FF6FF711438084A20F8041B0549B3
:10C56000343901600021FFF739FD0028EBD00320AA
:10C5700070BD00002C1F0020381C00205D3F020011
:10C580007CB5054608880C460930904201D90C203C
:10C590007CBD68466DDF0028FAD1218808206854E8
:10C5A00020881B21401C80B2208029542088401CF8
:10C5B00080B220802844DDF801100160BDF805102C
:10C5C00081802088801D80B220809DF8001049085D
:10C5D00000D0012129542088401C208000207CBDEF
:10C5E00070B51DA08AB0D0E90056047A0F216846C4
:10C5F000FDF7BDFD00208DF8000005218DF801102C
:10C600008DF8021002218DF803100F21ADF80410EF
:10C61000CDF80650CDF80A604FF47A71ADF81010DD
:10C620008DF813008DF812008DF8140001208DF89C
:10C6300015000C4807908DF80E400B480890CDF877
:10C6400018D006A9094804F039FE002801D0FFF7E8
:10C6500029FC0AB070BD0000D8ECF0F4F8FC00032F
:10C660000400000025E50100DDE40100882F002022
:10C6700008B50188132919D009DC102925D101201A
:10C6800000F040FABDE80840022000F033BA21294A
:10C6900012D0522919D1002380881A461946B1DFD9
:10C6A000002812D0BDE80840FFF7FCBB00238088BB
:10C6B0001A4685217FDFF3E70021009180886946D3
:10C6C0008FDF002801D0FFF7EDFB08BD10B51A4C35
:10C6D0000188606810290ED011292BD1401E60609E
:10C6E00028D1FFF711FB002824D02168002921D090
:10C6F000BDE810400847D0B900210122084600F0EB
:10C7000085FA08B107280FD107220221012000F085
:10C710007DFA08B1072807D104220221002000F089
:10C7200075FA20B1072802D0216801B188476068F6
:10C73000401C606010BD0000301C00202DE9F04757
:10C7400001883B4E40F2F3194FF6FF7510291BD0BC
:10C7500011293ED0122954D0502946D1C188F289DE
:10C76000841D914241D1618902293ED1868830469B
:10C7700003F098FB050038D004F10C0000F0DEF85F
:10C78000A8B3294630464EE0C17B8788044601297C
:10C790002BD1A846284603F085FB050017D02F8033
:10C7A00000202872234843464A460168C5F80A100B
:10C7B0004068C5F80E0004F1100105F10A0003F00D
:10C7C000FBFB6872F08900280FD129462AE004207B
:10C7D00013E0808803F066FB040006D06068FFF772
:10C7E00093FC08B107F098F82580BDE8F087FFE7D3
:10C7F0006868FFF789FC0028F7D0BDE8F04707F02C
:10C800008BB887880646384603F04CFB0400ECD012
:10C810002B464A4606F1080104F10A0003F0CCFB5E
:10C82000607221463846BDE8F04701F0EDB90000DE
:10C830002C1F0020381C00202DE9F04F074685886A
:10C8400002883D48012197B08346102A09D0112A59
:10C8500049D01A2A6CD1387AB1EB101F45D2012287
:10C8600044E0354C083CA068C0430B9061680BA8BD
:10C8700004F072FC0B990CA801F062F92C220CA9AF
:10C880006846FDF75BFC0026E946A04610E000BFC5
:10C8900009EB46005FF00004B0F804A008EB840048
:10C8A0005146001D04F02FFC641C1D2CF6D3761C91
:10C8B0000098B042ECD8142D05D317B00420BDE881
:10C8C000F04FFFF7EFBA2946584604F032FC2946EC
:10C8D00008F1040004F02DFCF87B012828D016484C
:10C8E0002946001D15E029461AE000220221B1EB7D
:10C8F000101F01D2012600E000260F49083901F17E
:10C900001000041D294682B104F013FC36B12946FB
:10C91000204617B0BDE8F04F04F00BBC2946204676
:10C9200017B0BDE8F04F04F0EEBB04F0ECFBF5E708
:10C9300017B0BDE8F08F0000501F0020007800F015
:10C94000010070472DE9F04FADF5477D14460E46C6
:10C950008246B2F5C07F05D96FF037000DF5477DEF
:10C96000BDE8F08F4FF4D0716846FDF700FC68A871
:10C9700004F0E7F8200E8DF81000200C8DF811005F
:10C98000200A8DF8120030208DF8170006AD8DF8C2
:10C990001340224631462846FDF7D0FB802028551B
:10C9A00004F119050020BEA90854401C2028FBDB17
:10C9B0004FF4807B5A4668A804F02EF90026B14651
:10C9C0006F46CDF8B892CDF8BC92CDF8C0922C4607
:10C9D0000DF52E78CDF8C49215E0002041463B5C61
:10C9E0000A5C5A400A54401C1028F8DB1037102CFF
:10C9F00001D3102000E02046241AAEAB1A460121D4
:10CA000068A803F0BDFC002CE7D1B2A83044102286
:10CA1000AEA9FDF793FB9DF803001036401C8DF87E
:10CA20000300302ECCDB5A46B2A968A804F0F4F813
:10CA3000BAAD56462B461A46012168A803F0A0FC61
:10CA4000102229463046FDF779FB10341036302C81
:10CA5000F0DB68A804F06AF800207FE741094A4249
:10CA600000EB421010B5044A0124844052F82130F2
:10CA7000234342F8213010BD7C1D00202DE9FC41EC
:10CA80000646C0074FF000050ED0104F00240122CB
:10CA9000385D009500231146019505F0D8FB641C14
:10CAA000042CF4D300F046F8B0070DD5074E00244F
:10CAB000361D0022305D032300951146019505F0D7
:10CAC000C6FB641C042CF4D3BDE8FC81DA430200ED
:10CAD00007490B5C4FF0A041D1F804250120984094
:10CAE00020EA0203C1F808351040C1F80C05704770
:10CAF000DA4302000249085C012105F0DDBB0000B9
:10CB0000DA4302000249085C002105F0D5BB0000B1
:10CB1000DA4302000649095C4FF0A040D0F8040552
:10CB2000C84010F0010000D0012080F001007047E3
:10CB3000DA43020010B500242046FFF7DBFF641C37
:10CB4000042CF9D310BD10B500242046FFF7DAFFFE
:10CB5000641C042CF9D310BD10B50246064B4FF0EF
:10CB6000FF3000215C5C944201D1084610BD491C95
:10CB70000429F7D310BD0000DE4302002DE9F04781
:10CB80000D468146FFF7E8FF0446042836D2DFF859
:10CB900074801B481C4EA8F10C0725B3012D0ED044
:10CBA000022D2BD104EB440030444578002D25D0D4
:10CBB000B968002922D02846BDE8F047084704EBB1
:10CBC0004401755C0E44717849B10E4A4FF400413E
:10CBD000093A8068FFF754FA08B987F80390B178EA
:10CBE00008F80410E2E78068FFF78EFA04EB4401CE
:10CBF000314418F804008D78A842D7D0BDE8F087FA
:10CC0000E44302002C1C0020CC1E002070B5002341
:10CC1000042810D20D4D00EB4004012A02D1012955
:10CC20000CD00022094E00EB4000304461B10129D4
:10CC300006D0022906D00723184670BD0E30C2B2B6
:10CC40002A55F9E74270F7E78270F5E7CC1E00201D
:10CC500070B506461E480024C0E90161B00720D522
:10CC60000025012211462846FFF7D0FF6D1C04461F
:10CC7000042D02D2002CF4D013E094B940F2666285
:10CC800004211448FFF7BAF804000AD1FFF7A4F80A
:10CC9000040006D10F48104A0021001FFFF79EF93B
:10CCA0000446F00712D00120FFF7E8FE74B90948E6
:10CCB0000A4A00210C38FFF791F9040006D1054813
:10CCC000074A01210838FFF789F90446204670BD5C
:10CCD000201C0020F0430200ABCE0100390002000E
:10CCE000D1BD01002DE9F05F6A4C05460026607851
:10CCF000B34618B184F801B003F086F9664F4FF4DB
:10CD00007A694FF4C87A4FF00108182D62D2DFE833
:10CD100005F0AC0C0C31404D62676B746B74BE7DDA
:10CD20007D7D7D7DACAFB2B5BEBE0020FFF7F2FECB
:10CD300000284FF0000008D0FFF7DCFE022D02D1E2
:10CD40004FF4E16008E0484606E0FFF7DBFE022D05
:10CD500001D1C82000E05046410CC0034FF4FA72E4
:10CD6000801841F10001257052000023FDF7A6F95B
:10CD700001462AE00020FFF7CDFE00284FF000001A
:10CD800004D0FFF7B7FE4FF44870E5E7FFF7BAFEAF
:10CD9000DFE70020FFF7BEFE00284FF0000002D0C2
:10CDA000FFF7A8FECFE7FFF7ADFED4E70020FFF7BF
:10CDB000B1FE00284FF0000002D0FFF79BFE01E01B
:10CDC000FFF7A0FE257041F69A1100223868FFF7A0
:10CDD00057F9064646E00020FFF77AFE257008E086
:10CDE000002051E025703DE084F801800120FFF72C
:10CDF0006FFE002240F6CD41E8E784F80180012073
:10CE0000FFF766FE00224FF48041DFE77868FFF706
:10CE10007BF90646D5F1110000D02EB10220FFF7B4
:10CE200069FE84F802B01DE0012816D980B2C8213D
:10CE30004843C117C90341EA5041C0034FF4FA7295
:10CE4000801841F1000152000023FDF737F9014637
:10CE500000227868FFF714F906460220FFF752FE19
:10CE600084F802803046BDE8F09F03F0CDF8B9E7C2
:10CE700003F0CAF8B4E703F0C7F804E003F0C4F81D
:10CE80000020FFF73FFE0120FFF73CFEAAE7FFF777
:10CE90005AFEA7E7201C0020E4430200012903D129
:10CEA0000D2801D104F008BA704700780221FFF77D
:10CEB00065BE00007FB50546006816460C460A2888
:10CEC00005D00C2803D00E2801D0AFF3008008460F
:10CED00006F0D1FA0090201D06F0CDFA019004F181
:10CEE000080006F0C8FA029004F10C0006F0C3FA3C
:10CEF0000390286805EB0014241D21466846FEF7C0
:10CF0000C9FD2D6819E000BF02F0EFFF684603F08D
:10CF100029F821466846FEF7BDFD009802F0CCFFD7
:10CF20000090019802F0C8FF0190029802F0C4FF3F
:10CF30000290039802F0C0FF0390103C6D1E6846FB
:10CF4000E2D102F0D2FF684603F00CF821466846B1
:10CF5000FEF7A0FD3146009807F0FCF8311D01985E
:10CF600007F0F8F806F10801029807F0F3F806F167
:10CF70000C01039807F0EEF87FBD00002DE9FF419A
:10CF80000546006816460C460A2805D00C2803D032
:10CF90000E2801D0AFF30080084606F06CFA00902E
:10CFA000201D06F068FA019004F1080006F063FA0B
:10CFB000029004F10C0006F05EFA0390281D04466E
:10CFC00001466846FEF766FD012710341BE000BFEE
:10CFD00006F0D8FD684606F043FD009803F0F0FF28
:10CFE0000090019803F0ECFF0190029803F0E8FF35
:10CFF0000290039803F0E4FF039021466846FEF791
:10D0000049FD10347F1C2868B8426846E0D806F015
:10D01000B9FD684606F024FD21466846FEF73AFD54
:10D020003146009807F096F8311D019807F092F804
:10D0300006F10801029807F08DF806F10C0103983B
:10D0400007F088F8BDE8FF8110B50446F421FDF72C
:10D050008EF8207810BD70B50E4615460446F421B2
:10D06000FDF785F8102D05D0182D05D0202D05D001
:10D07000AFF300800A2002E00C2000E00E202060C8
:10D080002A4631462046BDE87040FEF759BE2DE9DC
:10D09000FF5F9046DDE90E7B0E4682464FF00009A9
:10D0A00020E03568A8EB0504BC4200D93C46B9F144
:10D0B000000F05D10AEB05002146039AFDF750F851
:10D0C0001DB9444501D14FF001092919414505D148
:10D0D00051465A4610989047002001E0306820449D
:10D0E0003F1B3060002FDCD1BDE8FF9F2DE9FF4FD3
:10D0F00083B01746DDE91354129EDDF840B089462F
:10D100008246002E31D04FF00108012E1DD0022E94
:10D1100006ABCDF800802BD0CDE90154504600F08D
:10D1200037F89DF844105846594526D0B61E00964B
:10D13000CDE9015403463A4649465046FFF7A7FF5A
:10D1400011AB3A46CDF8008009E09DF818009DF833
:10D15000441006AB48408DF81800CDF80080CDE9AA
:10D1600001544946504600F013F807B0BDE8F08F6F
:10D17000CDE9015400F00CF8E2E7761E0096CDE907
:10D18000015403463A4649465046FFF780FFECE714
:10D190007FB50DF1200C9CE87000CDE90045CDE98C
:10D1A000025600F001F87FBD2DE9F05F5FEA00094B
:10D1B0000AA8164690E8100C0F461D464ED0396856
:10D1C000B1424BD205B99CBB5FEA0A0046D00D982C
:10D1D00070B351B34CB3701AA04200D320468046BE
:10D1E00001EB090042461946FCF7A8FF396845449F
:10D1F00001EB0800A4EB08043860B04215D10D988B
:10D20000494624B152469047002038600DE05A4606
:10D21000F9E7386860B90D98B442294601D15A46F9
:10D2200000E0524690473544A41BB442F1D217E0C7
:10D2300014E03968701AA04200D32046804601EB02
:10D24000090042462946FCF779FF3968454401EB5D
:10D250000800A4EB08043860B04201D3AFF30080AB
:10D26000002CE6D1BDE8F09F2DE9F05F5FEA000AEF
:10D270000AA8914690E8C0080D461C4609D02968C6
:10D28000494506D204B927B95FEA0B0001D00D98D1
:10D2900030BBAFF30080286830B951465A460D982C
:10D2A00090474846C5F80090A9EB0001B84200D36A
:10D2B00038460AEB01033246002108E014F801C0A9
:10D2C00013F801808CEA080C02F801C0491C84465E
:10D2D0008142F3D329683F1A091A16186444296059
:10D2E000002FD8D1BDE8F09F2DE9FF470446006824
:10D2F0001E461746884604F10809056812E02B46C9
:10D300004A464146684607F05DF8D4E900104A46AF
:10D310004B68694698472A4649463846FCF70EFF4F
:10D32000A8442F44761EEAD2BDE8FF87E0E8021247
:10D330000A681946FCF702BF70B50446086888B051
:10D3400016460D46102801D0AFF300802821204654
:10D3500003F02EFE04A8296803F02AFE04AA6B68D5
:10D36000114630469847694604A800F087F9694697
:10D37000084600F05FF904F10801684600F093F9EF
:10D380006946084600F056F904F11801684600F0B5
:10D390008AF9C4E9005608B070BD10B50B46816D1E
:10D3A00041B101680A6800F13001BDE8104018463B
:10D3B000FCF7C4BEAFF3008010B50446FFF7BCFF16
:10D3C0002046BDE81040AFF300807FB5002504463D
:10D3D0000095019502950395D4E900126B4628301B
:10D3E000FFF7A4FF102104F1400003F0E1FD2565E3
:10D3F0006565A5657FBD00002DE9F0410446006824
:10D4000086B00F46066822480025DBB1216D8B18D7
:10D410001B0702D0002312B104E00123FBE709B986
:10D42000616D39B15FF00001D4F858C0BCF1000F54
:10D430002AD101E00121F7E752EA010C24D003B11F
:10D4400021B301251249CDE90204CDE900213B4673
:10D4500004F1500104F14000324688460746FFF7C8
:10D46000A3FE002D0DD0206D01AB311A094A00201A
:10D4700083E8170000908023324641463846FFF784
:10D4800035FE06B0BDE8F081AFF300800248D9E771
:10D490006FD90100D5D90100C3D901001FB5074CD0
:10D4A000CDE90240CDE9002302680B4600F12801D6
:10D4B00012681830FFF7D8FE1FBD000071DD0100B3
:10D4C0002DE9F0410D461F46164604463421FCF76F
:10D4D0004EFE0020E06229682163A062C4E9005684
:10D4E000394604F108002A68BDE8F041FCF726BE81
:10D4F0002DE9FF4FB9B08146DDE94A84DDE9487680
:10D50000DDE946BA014601A83A9AFFF755FF25AD75
:10D5100033463A46002101A8009500F0F9F929AEFA
:10D5200053465A46012101A8009600F0F1F92DAFAB
:10D530000097DDE93B23022101A800F0E9F91CB1C5
:10D54000D9F80000A04201D2AFF30080002031AA38
:10D5500006E0295C3B5C5940335C59401154401C47
:10D56000A042F6D311464046002205E010F8015BC8
:10D5700011F8013B6B401A43641EF7D21AB1012027
:10D580003DB0BDE8F08F25AB494618A83A9AFFF7A1
:10D5900097FFDDE93B1318A84C9AFFF77FFF0020A7
:10D5A000EEE72DE9FF4FB1B00E46DDE94095DDE92C
:10D5B0003EBA0A468046014601A8449FFFF7FCFE9A
:10D5C00025AC2B464A46002101A8009400F0A0F9A2
:10D5D00029AD53465A46012101A8009500F098F95B
:10D5E00025AB3246414618A8FFF76AFFDDE9331341
:10D5F00018A8429AFFF752FF2DAE0096022101A80B
:10D60000349B429A00F084F9D8F80000B84201D265
:10D61000AFF30080002007E0215C325C51402A5CBF
:10D620005140439A1154401CB842F5D335B0BDE87F
:10D63000F08F000038B50C460FA100220968009158
:10D64000C16842EA4102E260CA0F816842EA4102CF
:10D65000A260CA0F416842EA410262600068C90FD5
:10D6600041EA40012160C00F0222694606F03CF900
:10D67000E1684840E06038BD0087000070B50C46A6
:10D68000054605F0FFFE2060281D05F0FBFE6060EA
:10D6900005F1080005F0F6FEA06005F10C0005F0AC
:10D6A000F1FEE06070BD70B504460D46006806F0FE
:10D6B00059FD291D606806F055FD05F10801A068B7
:10D6C00006F050FD05F10C01E068BDE8704006F081
:10D6D00049BD000005494FF0FF32082841F82020DD
:10D6E00002D3084480F8482070470000DC21002065
:10D6F000F0B54FF0FF3512B10023082601E00823F2
:10D700000C260C4C05E000BF54F823707F1C04D09D
:10D710005B1CB342F8D32846F0BD26185DB286F8EC
:10D72000305044F82310002AF5D1E11881F8480060
:10D73000F1E70000DC2100200249084490F93000A4
:10D7400070470000DC210020F0B591B01E4617465E
:10D750000D4604001FD0F5B1EFB1E6B11C2101A8C0
:10D76000FCF705FD142109A8FCF701FD0020089035
:10D770000090A078C00711D09DF8040040F002008E
:10D780008DF804009DF8000020F00F00401C20F0F0
:10D79000F000103006E00E2011B0F0BD9DF8000042
:10D7A00020F0FF008DF80000A07880079DF80100B0
:10D7B00020F00F000CD5401C20F0F00010308DF848
:10D7C00001009DF8040040F008008DF8040003E01B
:10D7D00020F0F0008DF8010028788DF822002088D4
:10D7E000ADF82000A078334641099DF8020009AA4F
:10D7F00061F342008DF80200A178890861F3C3004B
:10D800008DF80200A178C90861F304108DF80200B8
:10D81000A178090961F300008DF8020008A80990B9
:10D82000CDF828D0E078ADF82C000D972079ADF830
:10D830003000688801A9AADF01000BD1074A064B16
:10D840003588107823F8205003EB800324885C800F
:10D85000401C107008469FE700200020401C00205C
:10D860003EB5194C08B1012060706088A0F57F4179
:10D87000FF3925D16078002822D0002060709DF803
:10D88000000020F0FE008DF8000002A830DF01E06B
:10D8900002A830DF9DF808000628F9D306210DF113
:10D8A000010031DF207874DF68466CDF0828FBD088
:10D8B00008B1FEF7F7FA00F027FC10B100F030FCD9
:10D8C0003EBD00F03BFC3EBD801D002070B5084C05
:10D8D000050009D010342168002907D008682060AD
:10D8E000496828468847F6E70834F4E770BD000029
:10D8F00078210020054A012120B1012805D191702D
:10D90000FFF7E4BF51700020FAE77047782100204C
:10D910002DE9FF4707460068DDF830901D46046892
:10D9200090460E46ACB121466846FCF720FC0DEB54
:10D93000040000F8016C3846FFF747FD5DB1002395
:10D94000224669463846FFF757FD01232A464146DD
:10D9500004E0AFF300800123224669463846FFF712
:10D960004BFD49463846FFF718FDBDE8FF871FB558
:10D97000044601236A462830FFF7B6FC2168606D33
:10D980000968084460651FBDF0B5044689B0236886
:10D9900068461D68002304E0CE5CD75C7E40C65418
:10D9A0005B1CAB42F8D30146012304AA04F1280012
:10D9B000FFF79AFC2168606D09680844606509B04A
:10D9C000F0BD10B5044600F10802FFF7DDFF0120AD
:10D9D000A06510BD10B5044600F11802FFF7D4FF92
:10D9E0000120A06510BD00002DE9F05F24484168CA
:10D9F000002942D0DFF88CB00E688146DBF8004089
:10DA000087688078E11B21F07F45ED1CB0B9DFF815
:10DA100078804FF48030C8F84403C8F8040311201C
:10DA2000FDF70AFD1120FDF712FD4FF0010AC8F8BD
:10DA300000A02F2004F004FF89F802A0B54200D214
:10DA40003546104BE8193C3320F07F401860DBF876
:10DA500000105A46091B21F07F41001B20F07F4037
:10DA6000C91C814209D9106818602F2004F0E8FE13
:10DA7000BDE8F05F1120FDF7F5BCBDE8F09F0000A8
:10DA8000A81C002004150140001001402DE9F041C0
:10DA900016461278174C0D460746202A03D194F8F3
:10DAA0004D01002817D100233946124801F044FBEC
:10DAB00004EB8714317884F82610A17404F1140063
:10DAC00059B1102909D0202905D1801E01F064FC2C
:10DAD0000E2084F82700BDE8F0816A1E711CFCF757
:10DAE0002DFB0021384605F07BFF6D1C84F8275084
:10DAF000F1E70000B02B002070B50C460978491EF4
:10DB0000C9B20023C55C954216D18B4204D30DE007
:10DB1000C2185278C2545B1C8B42F9D3C1F1050381
:10DB20000844AB221946FCF71BFB01E0AB21C154B2
:10DB30002078401E207070BD5B1C052BE2D370BDA9
:10DB400073B58CB00646002000900D9880B100247B
:10DB50006D4621460DA803F0E1FA30B1009805EBBF
:10DB6000400084800098401C0090641C142CF0D36A
:10DB70002C2269463046FCF7E1FA0EB070BD2DE963
:10DB8000F04117880646B81D14460D46984202D942
:10DB90000C20BDE8F0813188072206290AD34FF412
:10DBA000486C4FF6FF73614501D9994202D17088E4
:10DBB000062801D21046ECE7604501D99842F9D118
:10DBC000994203D0984201D08142F3D80520E8550C
:10DBD00020881221401C80B2208029542088401CBB
:10DBE00080B220804119308806F084F921880844E9
:10DBF00080B220804119708806F07CF921880844A1
:10DC000020800020C5E7000038B54A7A0F4B62B18A
:10DC100000220A725969002906D001228DF80020DD
:10DC2000ADF802006846884738BD0A7A62B19B6841
:10DC30004C68024619462046FEF722FA0028F3D027
:10DC4000BDE8384005F068BE5B68F1E72C1F002096
:10DC500010B5174896B0174C00681590A0788DF84D
:10DC600056003C216846FCF782FA02208DF800003D
:10DC700000208DF802000120ADF8100015A80590D5
:10DC800004F110000C4981601F2181810146684622
:10DC900000F0A8F9627800210FA801F051FF0FA849
:10DCA000FDF7BAFF012002F077F916B010BD0000B1
:10DCB00008470200BC1C0020BF23002030B10068D0
:10DCC0000549884205D048F20250704748F2015099
:10DCD00070470020704700004145414430B1006862
:10DCE0000549884205D048F20250704748F2015079
:10DCF0007047002070470000634145532DE9F04113
:10DD00008CB00E4604466F4630213846FCF72FFA99
:10DD1000002504F120081020211811F8012D521CB3
:10DD200012F0FF020A7002D1401E0028F4DC3B46CC
:10DD300022460121404602F023FB10351037302DDA
:10DD4000E9DB00206946335C0A5C5A400A54401CF7
:10DD50003028F8DB4FF48072404602F05DFF08ADDA
:10DD600095E80F0084E80F000CB00020BDE8F081BA
:10DD700070B50446D4E9002053680A4604F108014E
:10DD80000D469847E06A4119206B01E0002806D053
:10DD9000401E0A5C521C12F0FF020A54F6D070BDFD
:10DDA0007FB50C4610B1012004B070BD207900266B
:10DDB00038B141F61D5501281BD0022826D00F206E
:10DDC000F2E70220207102960396E068019069460E
:10DDD00001A805F001FC50B102988188E18000881B
:10DDE0002081BDF80010029805F074FCDCE70A20E1
:10DDF000DAE70A4B6A460021A01D05F0A9FB38B1FD
:10DE0000064918398E61CE610A28CDD12846CBE764
:10DE100002488188019805F05DFCF5E7601D00204F
:10DE20002DE9F0470025DFF88C803CE06068002198
:10DE300000EBC506012032789146FCF770F9D4E971
:10DE4000062300EA020701EA030C57EA0C0728D070
:10DE500082438B434846C4E9062304F0B3FD32787D
:10DE60008246914601200021FCF759F9D4E90423A8
:10DE700000EA020401EA03074A4650460021FCF783
:10DE80004EF944404F403C430BD17078012801D0FB
:10DE9000012100E00021726881EA0A010AB14846C6
:10DEA00090476D1CEDB298F8000044468542BDD302
:10DEB000BDE8F087781C002070B5054600EB4500F2
:10DEC000C0EB451186B01C48102200EB81040023F2
:10DED000059244F8403F05AE6360A360E36094F8A8
:10DEE0002C00E072A16AC1408140080E2073080C2A
:10DEF0006073080AA07304F80F1F601CA4F10F01DF
:10DF0000CDE90031CDE90220A4F11F0304960122DE
:10DF10000A490B484F3C03F014FC08B1FDF7C2FF5F
:10DF2000D4E91401074AC4E918010121926828467E
:10DF3000904706B070BD0000CC250020B44402001C
:10DF400060280020241D00200E4910B50A784C7866
:10DF50000023A24212D0521CD2B20A70022A00D16F
:10DF60000B70084A0B780C3252F823200260886844
:10DF7000104420F07F408860012010BD0360002025
:10DF800010BD0000A81C002010B50846114603F083
:10DF9000EDFF002010BD00002DE9F843104D0F46A5
:10DFA00080461E4691466946286803F080F80400C2
:10DFB00014D01C21FCF7DBF801202071C4F8149068
:10DFC000380BC4F80080C4E902606946286803F091
:10DFD0008FF805F02BFA0020BDE8F8830420FBE75A
:10DFE000504802000A46002101F0D8BB2DE9FC414F
:10DFF0000546002016460F460090019000F0D2FF23
:10E0000004462FB1284600F09BFF94F84C5107E0DE
:10E0100004EB851090F82600202801D101F0CEF8FD
:10E0200004EB851000F11201019190F82700ADF882
:10E03000000032466946002001F0B0FBBDE8FC81DB
:10E0400070B5084C049DA0700020A1602070637022
:10E05000A280E56001F074F9BDE87040024800F06C
:10E0600075B80000BC1C002071BC0100014880880C
:10E0700070470000BC1C002010B5044600F092FF61
:10E0800090F8411139B190F84D1121B190F840014B
:10E090004FF4487103E090F840014FF4FA7110FB1F
:10E0A00001F080B2844200D80446044844F620615E
:10E0B0008C42848000D9818010BD0000BC1C0020EF
:10E0C00010B502880F49102A10D0112A14D0262A20
:10E0D00017D1007A012814D10878002811D1022024
:10E0E00001F05AFFBDE81040FDF734BD0120087073
:10E0F000BDE8104000F022B800200870FDF7A8FD30
:10E10000F0E710BDBC1C00200148407870470000BB
:10E11000BC1C00200149487070470000BC1C002056
:10E12000054810B50078002805D1FDF791FDBDE840
:10E130001040FFF78DBD10BDBC1C00200148808839
:10E1400000F072B8BC1C002000F0C4B803490022E3
:10E150000A7088602A210248FCF709B8DC1C0020FC
:10E16000202400202DE9F04F30B1027C002132B193
:10E17000027A22B1012303E00E20BDE8F08F0023D4
:10E18000827842B1D21A0488002594FBF2F21FFA79
:10E1900082F9AB4637E00720EFE74268525D13B1E2
:10E1A000447C94422ED0446904EB8106491C727071
:10E1B00086F800B0A6F80290C9B21BB3077A002413
:10E1C000D0F80CA016E000BF1AF804C090469445A1
:10E1D0000FD144694FF4967C04EB81040127A6F823
:10E1E00002C084F801802770E14506D9A9F596722E
:10E1F00005E0641CBC42E7D304E04FF4FA72491C0A
:10E200006280C9B26D1C8278AA42C6D8426982F87F
:10E210002810406929B16FF0010303EB810120F858
:10E2200001B00020A9E7000030B587B0044600F037
:10E23000B9FE234D0121297090F8400100283DD0FE
:10E24000610CE0034FF4FA72801841F100016C8018
:10E2500052000023FBF732FF01461A4800220068F3
:10E26000FDF70EFF08B1FDF71DFE00F09BFE1549FE
:10E270000446182208316846FBF760FF6888ADF84D
:10E28000000094F840018DF8020004F5A17001909F
:10E2900094F841018DF8080004F24710039094F8B7
:10E2A0004D018DF8100094F84C018DF8110068466E
:10E2B000FFF758FF002801D0FDF7F4FD07B030BD8F
:10E2C000DC1C002010470200014900200870704744
:10E2D000DC1C002010B50A4A00210A48FDF77EFE2A
:10E2E00008B1FDF7DFFD0748074A0021001DFDF7D3
:10E2F00075FE002803D0BDE81040FDF7D3BD10BD6A
:10E3000001BB01001047020069BB010010B50028E5
:10E3100015D00B494988018004F010FD00280ED16A
:10E320000121074804F012FC08B1FDF7BBFD04F021
:10E330000DFD002803D0BDE81040FDF7B3BD10BDB2
:10E34000E81C00200EB51049104804F0AFFC08B1DD
:10E35000FDF7A8FD0D4A121D07CA8DE807006946A2
:10E36000002004F045FC08B1FDF79CFD01210848A0
:10E3700004F0ECFB08B1FDF795FD04F0E7FC002884
:10E3800001D0FDF78FFD0EBD793702003047020046
:10E39000E81C00201FB5074CD4E90423E46903946A
:10E3A0000092CDE901308DF80E106846FDF714FBA0
:10E3B00004B010BD404702001FB5074CD4E90C2340
:10E3C000E46B03940092CDE901308DF80E1068469D
:10E3D000FDF702FB04B010BD404702001FB5074C1B
:10E3E000D4E90023E46803940092CDE901308DF86C
:10E3F0000E106846FDF7F0FA04B010BD4047020069
:10E400001FB5052802D3072004B010BD0A4C236AAB
:10E41000E46A0093094B039433F81030ADF80030F0
:10E42000064B0C3353F82000CDE901018DF80E2086
:10E430006846FDF7D1FAE7E740470200F41C0020E8
:10E4400010B541F2373001F067F8002802D1024AD6
:10E450000121117010BD0000EC1C0020094810B50E
:10E46000012141604FF6FF71418000210170064893
:10E4700001F07EF9002803D1BDE8104001F096B804
:10E4800010BD0000EC1C0020BDF4010001484068F4
:10E4900070470000EC1C002002880D49102A14D09F
:10E4A000112A14D14FF6FF704880087800280ED04A
:10E4B000BFF34F8F07480168074A01F4E061114339
:10E4C0000160BFF34F8F00BFFDE780884880704731
:10E4D000EC1C00200CED00E00400FA0538B5104BF0
:10E4E000154647F207541A7882B1A14203D101219F
:10E4F00000F0F4F804E000925B782A4600F076F829
:10E5000000280BD0BDE83840FDF7CCBCA14202D1B9
:10E5100000F058F8F4E700F03BF8F1E738BD0000F0
:10E52000201D00202DE9FC411C46114B089D47F29F
:10E5300007561F786FB1B14213D05B78CDE9005315
:10E54000234600F023F900280FD0BDE8FC41FDF779
:10E55000A9BCB14205D113462A46214600F0E8F88D
:10E56000F1E7002100F0BAF8EDE7BDE8FC8100001A
:10E57000201D002040B1054900224A700A704A1C43
:10E58000C0E91C21002070470E207047201D00208C
:10E5900007B582B078B1A1F5EA420C3A06D0921DD7
:10E5A0000BD0012100F09AF805B000BD01218DF8D3
:10E5B00000106A4602E00E20F6E704AA012104F0EA
:10E5C000B3FFF1E71FB504000ED0684600F01AFB58
:10E5D000002807D1684600F0D9FB6A461021204682
:10E5E00004F0A2FF04B010BD0E20FBE7F0B58DB023
:10E5F0001C4616460F4605000FD000F0D3FC02461D
:10E600006FF4EA4038440C2864D2DFE800F00909CE
:10E61000232D33210909445C633E0E200DB0F0BD6B
:10E62000242104A8FBF7A3FD2B4802AA3146006869
:10E63000029004A80390B5F86400ADDF0028EDD186
:10E64000BDF80800039AC1B2284604F06DFFE5E763
:10E6500012AA17E0FFF70AFD010241EA1020ADF807
:10E6600000006A460221EFE702EB841201212846EE
:10E67000521C23E002EB841292F8280008B12932E0
:10E6800000E0521C0121284618E001208DF800000E
:10E690006A460146D8E702EB841292F82A0018B1C4
:10E6A00092F82600302806D00DB02846BDE8F0408C
:10E6B000012100F013B810212846921C0DB0BDE8CE
:10E6C000F04004F031BF0DB021462846BDE8F040CF
:10E6D00004F0DFBE0720A1E7804702001FB500223B
:10E6E000009201920292039230B141B101218DF862
:10E6F00000104FF4817107E00E2004B010BD02211C
:10E700008DF8001040F20311ADF80410694600F0D6
:10E7100001F8F2E740B139B1B0F86400A0F57F42EA
:10E72000FF3A03D0B0DF70470E20704708207047D3
:10E7300070B586B0144606000CD059B10025059579
:10E740000095029503950495ADF800400191102CB9
:10E7500003D00CE00E2006B070BDB6F864006A4627
:10E760001946ACDF60B140F20310ADF80C0001981F
:10E770000590ADF8124002A9304605F0E0F8EAE74E
:10E78000ADF80C50019800F027FBF0E72DE9FF41B0
:10E790001C46DDE90A53070017D0B4B10020A1F5EB
:10E7A000EA41019002390090029006460390ADF8CC
:10E7B000040040F20D120B2975D2DFE801F00A11B6
:10E7C000171D2374747438676F000E2004B0BDE801
:10E7D000F0812078042866D9ADF80420002562E095
:10E7E0002088010241EA102080B24CE094F9001028
:10E7F000184600F03DFC56E094F90010184600F071
:10E80000C9FC50E0012D02D0112D05D006E0217881
:10E81000D9B3022947D001E0217809B1207004E082
:10E82000601C00F0ABF90028D0D101253BE0142D8D
:10E8300000D9012615F0FF001AD0012801D1217856
:10E84000B1B1217831B1102907D0202909D0302960
:10E850000FD109E011280BD00BE0001F0F2807D9BA
:10E8600007E0012804D004E0222801D0122800D1BA
:10E870000022ADF8042042B9E9B22246184600F061
:10E8800095FBFFF7F3FBFFF7F7FB0CE020780B2875
:10E8900009D1FFF7D5FD002898D104E0207800B118
:10E8A0000120FFF737FCADF80A5003940EB10020A9
:10E8B0008CE76946384605F042F887E72DE9F043D2
:10E8C000CDB0894680461746202141A8FBF74FFC72
:10E8D000202508EB48023C484026C2EB481200EBDA
:10E8E0008204CDE94A560121499584F8701084F8D4
:10E8F0006C704FF47F40A0662B464A462FA93348E0
:10E9000003F04CF808B1FDF7CDFA314B2F491F4603
:10E91000A3F128022F4803F01FF808B1FDF7C2FA4F
:10E920004AA800902A492B4827AB2FAA2839001D56
:10E9300003F068F808B1FDF7B5FA202227A941A82D
:10E94000FBF727FC10B90320FDF7ACFA49AA39A957
:10E95000384603F03DF808B1FDF7A4FA20224946F5
:10E9600017A8FBF7EBFB202239A91FA8FBF7E6FB52
:10E970000020CDE903600590069027A9CDE9001598
:10E9800017A802904BAB07AA1349144803F068F884
:10E9900008B1FDF787FA07AD95E80F0084E80F008E
:10E9A000404605F06DF94046FFF786FA094C032111
:10E9B0000C3C4046A2689047A2680221404690471E
:10E9C0004DB0BDE8F0830000CC250020804402005B
:10E9D00038280020301D00208C44020084290020AB
:10E9E00000EB4001C1EB4010024901EB8000806E5A
:10E9F00070470000CC25002000EB4002C2EB401025
:10EA0000034A02EB8000026E0A60406E4860704765
:10EA1000CC25002000EB4001C1EB4010024901EB86
:10EA200080007421FBF7A3BBCC25002070B5054600
:10EA300000EB4500C0EB45140D4800EB8404204674
:10EA400084F86C10A26610221946FBF777FB0120B0
:10EA5000084A84F8700002219268284690472846A8
:10EA600005F00EF92846BDE87040FFF725BA000012
:10EA7000CC250020241D002070B50D46014601EB79
:10EA80004102C2EB4111134A86B0102002EB81060D
:10EA9000A2F1200105905CCE81E85C00CDE9011077
:10EAA000002001F11004009005AACDE90342A1F174
:10EAB00010030122084903F5317002F042FE08B14B
:10EAC000FDF7F0F9102221462846FBF737FB06B088
:10EAD00070BD0000CC250020B44402007FB50400C6
:10EAE0002ED01F4D00212846FFF778FC0A2829D098
:10EAF00008B1FDF7D7F91B48502184601A48FBF78D
:10EB000036FB174A00204FF47F41303200EB4003C0
:10EB1000C3EB401302EB8303401C99660528F5D331
:10EB20004FF400410F4800F0D5FB08B1FDF7BAF9EA
:10EB300003F0AEF808B1FDF7B5F9002004B070BDE0
:10EB40000720FBE709A10FC98DE80F0010226946D5
:10EB50002846FBF7F3FA01212846FFF73FFCC7E7F9
:10EB60009C250020241D002010280020FFFFFFFF0F
:10EB7000FFFFFFFFFFFFFFFFFFFFFFFF10B58AB0A2
:10EB800000211022CDE908120591069109AB05ACD0
:10EB900007910091CDE90343CDE90102094B0A46F3
:10EBA000094903F5317002F0CCFD002808D1A446D4
:10EBB00004489CE81E0080E81E000121FFF70EFCBF
:10EBC0000AB010BD9C250020B44402000B4600EBA7
:10EBD0004001C1EB40100349102201EB80011846AF
:10EBE000FBF7ACBACC25002008B5202000906A467F
:10EBF000034802F0EDFE002801D0FDF753F908BDEF
:10EC000038280020102103F079B9000000EB400102
:10EC1000C1EB4010024901EB800090F86C00704796
:10EC2000CC25002070B5044600EB4400C0EB441630
:10EC3000154886B0102300EB86000125059380F867
:10EC4000705080F86C204FF47F42826605AACDE9AF
:10EC5000030200208DE80B000B4B0246303B0B49B2
:10EC600003F5317002F06DFD08B1FDF71BF9204688
:10EC700005F006F82046FFF71FF9054A0221204655
:10EC80009268904706B070BDCC250020B4440200C5
:10EC9000241D0020F0B595B000240E460C940D9470
:10ECA0000E94D1F802100C91D6F806100D91D6F8FA
:10ECB0000A100E9100EB4001C1EB4011304815469F
:10ECC00000EB81010DF13C0E91E80D100A940B94BC
:10ECD0008EE80D10886E91F86C100C27C8408840A3
:10ECE000010E8DF82810010C8DF82910010A8DF8FD
:10ECF0002A108DF82B00022113A8139403F0FEF8BC
:10ED000008B1FDF7CFF8BDF84C00ADF82C000FAA04
:10ED10001C491D48149402F0E7FC08B1FDF7C2F845
:10ED2000022014A9CDE9051007AA0094CDE90372C9
:10ED30000CA8CDE9014006230AAA0121124802F0DD
:10ED400094FC08B1FDF7AEF80F4802F0EDFC08B1F5
:10ED5000FDF7A8F830782870012068700798C5F88A
:10ED600002000898C5F806000998C5F80A00BDF821
:10ED70004C00E881BDF85000288215B0F0BD0000BD
:10ED8000CC250020A4440200B42A002030B501465E
:10ED900087B010240E48224605460594FBF7CEF9AD
:10EDA0000B4805A910300294CDE903010020084B5F
:10EDB000CDE90005103B0122064903F5317002F050
:10EDC000C0FC002801D0FDF76DF807B030BD000091
:10EDD000AC250020B444020010B510220649FBF710
:10EDE000D8F9002806D1054A002108469268BDE8F6
:10EDF0001040104710BD0000BC250020241D00203D
:10EE00002DE9F047DFF8A89099F8000000F03CFAEF
:10EE100007004BD0274C002505EB4500C0EB451003
:10EE200004EB800090F8701001B3816E3944816664
:10EE3000E8B2804600EB4001C1EB481004EB8006CD
:10EE4000B6F868000004000C02D1404604F018FF38
:10EE500096F86C000221401EB26E8140B2FBF1F0C8
:10EE600001FB102010B94046FFF726F86D1C052D58
:10EE7000D2D3D9F80400104938444E46C9F80400EA
:10EE8000884213D35FF0000505EB4500C0EB451049
:10EE900004EB800090F8700018B1B268E8B2042169
:10EEA00090476D1C052DEFD300207060BDE8F08702
:10EEB000241D0020CC2500208051010070B505469E
:10EEC0001348302600EB85140A2084F8266084F865
:10EED000270004F114012846FFF78EFDA67494F96B
:10EEE0000110284604F07CFD0A4C207840B1012333
:10EEF00030222946064800F01FF90020207070BD1E
:10EF00002946BDE8704000233022014800F014B9C2
:10EF1000B02B0020381D002013B50C46684604F0C5
:10EF2000DBFD002C09D005489DF80010102200EBF5
:10EF300081102146801CFBF701F91CBDB02B00207D
:10EF400030B5054689B0164800F0D6F8002821D023
:10EF5000134C002194F841011FE0621892F84731E8
:10EF6000AB4219D105A800F017FA6A4605A9284650
:10EF7000FFF790FE94F84C01122204EB80106946D2
:10EF80001230FBF7DBF894F84C11122004EB8111DE
:10EF900081F8270009B030BD491C8842DDD8F9E767
:10EFA000B02B002000487047B02B0020F7B5154665
:10EFB0000C46684604F090FD15B90E20FCF772FF70
:10EFC00044B1012C01D1287820B129782748302973
:10EFD00006D009E09DF80010244800F05FF8FEBD5F
:10EFE000222C12D0122C10D09DF8001000EB8110B2
:10EFF00090F82A0010B11D4800F050F82A4621462A
:10F000009DF80000FEF742FDFEBD9DF8001000EBEC
:10F01000811090F82A0010B1144800F03FF89DF8D4
:10F02000006027462C463146104800F037F810B1F2
:10F030003046FFF7EFFC2078302802D00820FCF79C
:10F0400031FF222F05D0122F0AD00720FCF72AFF0C
:10F05000FEBD94F82120611C3046FFF72FFCFEBD59
:10F06000627C611C3046FFF7DDFDFEBDB02B002049
:10F0700013B50C46684604F02FFD07499DF80000C3
:10F0800001EB80114C7091F82810002902D1214623
:10F0900004F0A6FC1CBD0000B02B00202DE9F041BF
:10F0A0000E4600EB8615044695F82A000027E0B1CD
:10F0B00094F84D01B84628B194F84C11B14201D1F1
:10F0C00084F84D8104F5A0713246881CFEF714FDCA
:10F0D00095F82600302806D104F241113246881DE9
:10F0E000FEF70AFD012785F82A8028464021FBF714
:10F0F0003EF83846BDE8F08190F8411121B190F812
:10F100004D0108B1012070470020704770B50025FF
:10F11000044680F84D51AB22052100F5A170FBF7A4
:10F120001FF8AB22052104F24710FBF719F884F809
:10F13000415184F8405170BD70B50125202A03D19A
:10F1400080F84D5180F84C1100EB81145B1E94F84F
:10F150002A601E4200F2471315D184F82A5090F815
:10F1600040515C1F295590F84041641C80F8404193
:10F17000302A07D190F84121D15490F84111491C0F
:10F1800080F8411170BD302AFCD194F82620302A35
:10F19000F0D170BD13B50C46684604F09DFC0649DD
:10F1A0009DF80000012201EB801101F8282F4C701E
:10F1B000214604F015FC1CBDB02B0020064890F839
:10F1C0004D11002906D090F84C1100EB811012303F
:10F1D00000F0E2B870470000B02B002070B5054683
:10F1E000104800EB851494F82A00C0B194F826006A
:10F1F00030280DD12846FFF7F3FBE0622846FFF7E1
:10F2000005FD84F82B0004F130012846FFF7DEFCF1
:10F21000214601222846BDE87040FFF7F1B80222DE
:10F220000021F7E7B02B00207CB5002504460095AF
:10F2300013480195FFF76AFF1248002105706846E0
:10F24000FFF7BAF80A2807D008B1FCF72BFE002414
:10F250006D46285D68B10FE0402221460848FAF764
:10F260006DFF94F82620012300210548FFF764FF75
:10F270007CBDE0B200F06EFF641C052CE9D37CBDC0
:10F28000B02B0020381D00202DE9F0410446FCF78A
:10F290009FFE0F4E054656F8240010B90820FCF7D3
:10F2A00001FE0B4F2846103F57F82410FCF78CFE48
:10F2B00056F82410814208D8B5FBF1F2B0FBF1F00A
:10F2C0004A4347F82420BDE8F0810020FBE7000016
:10F2D000202D002010B568B1094B1A78042A0BD0F4
:10F2E0005C785CB10270074840F82210521C1A701A
:10F2F000002010BD0E2010BD082010BD802010BDC4
:10F30000391D0020202D00200749084A00200870E0
:10F31000106050609060D060106150619061D06169
:10F320000120487070470000391D0020102D00207A
:10F3300002488168491C8160704700003C1D002024
:10F3400010B50E211248FAF712FF11482021017062
:10F35000002141700F48816004F0EEFD04F032FEA0
:10F3600004F0DEFD40F6CD410A48FFF7B3FF08B1D7
:10F37000FCF798FD07484FF4A021401CFFF7AAFFB7
:10F38000002803D0BDE81040FCF78CBD10BD000084
:10F39000302D00203C1D002010B5044604F0CCFDAB
:10F3A0000A49886802BA0A48C0F806204878FFF778
:10F3B0006BFF18B104F0B4FD04F004FE2046BDE874
:10F3C00010400E220249FAF7B9BE00003C1D002091
:10F3D000302D002010B503780022072B06D2DFE87D
:10F3E00003F005040610202930000A7010BD012327
:10F3F0000B7003898B818388CB81C06888600A7415
:10F4000010BD02220A7002898A818288CA81C2687C
:10F410008A60807D062802D00020087410BD01207B
:10F42000FBE703220A70C2888A810289CA81C06808
:10F43000886010BD04230B70C0888881CA818A60EF
:10F4400010BD0520087010BD70B5064D064600249D
:10F4500055F8241009B130468847641C042CF7D3B2
:10F4600070BD00005C2D002030B50446006887B0F8
:10F470000D46806800281FD018216846FAF777FEED
:10F480000195A0680590207910B1012810D107E0FE
:10F4900001208DF8000020690290E068039005E0EB
:10F4A00002208DF80000E06800030290606904907B
:10F4B000206881686846884707B030BD10B500787D
:10F4C000134C062823D2DFE800F0031C1C050510AE
:10F4D00000201BE000210F4A0846FCF7EFFC002843
:10F4E00015D0BDE81040FCF7DDBC207848B160883D
:10F4F000A0F57F41FF3904D0132176DF08B1FCF776
:10F50000D1FC6068002802D06068401E606010BDB9
:10F51000EC1C002099F5010038B504460E4800782F
:10F52000A8B1A4F57F40FF380FD0684603F07CFEF9
:10F5300078B10521017001210171C480684603F092
:10F5400081FE03F065FF002038BD042038BD022095
:10F5500038BD082038BD0000681D00200C4808B5E3
:10F56000007888B1684603F05FFE78B1062101702B
:10F57000684603F067FE0748017809B10121C174AC
:10F5800003F046FF002008BD022008BD082008BD8A
:10F59000681D0020542F002010B5FFF7DFFF024840
:10F5A0004168491C416010BDEC1C0020F0B587B0DB
:10F5B00014216846FAF7DBFD2C4C207818B1684618
:10F5C000FFF742FF4FE0201D01F0BDFDC0BB4FF033
:10F5D00010204169000400694A1C02D100EB400080
:10F5E0000101234800220161A1F52041C1602149A8
:10F5F00002F083FD002821D120481C234FF49A7289
:10F600001D49006801F040FD03F068FD050014D0BD
:10F61000022D12D000270126062D12D005A803F0D6
:10F6200003FE88B106700C2D18D2DFE805F0170F25
:10F63000170F17161716171113110B2007B0F0BD6F
:10F6400011E026706760BAE70820F7E7077105E068
:10F65000032100E00221017100E0067105A803F01A
:10F66000F1FD03F0D5FE0020E8E70000681D002052
:10F67000B81D0020604802006C2D00208847020061
:10F6800038B5040014D0694603F0A6FFA0B1BDF858
:10F69000000000EB8001094800EB8100C16849B11E
:10F6A000A17A39B1C168491EC1600020A07238BD7D
:10F6B000052038BD062038BD0A2038BDA02E002008
:10F6C00038B504460D48007888B194B1684603F017
:10F6D000ABFD80B104210170002101712168C1607E
:10F6E000684603F0AFFD03F093FE002038BD022012
:10F6F00038BD052038BD082038BD0000681D002039
:10F7000007B513460A466946002003F021FF0EBDE7
:10F71000F8B50D46040018D0BDB1694603F05CFF92
:10F72000A8B1BDF800000B4900EB800001EB8000A0
:10F7300001210C30666801F009FD2E6060680C3014
:10F7400068600120A0720020F8BD0520F8BD0A20E5
:10F75000F8BD0000A02E002018B10323002204F001
:10F7600009BD052070470223002204F003BD0000FC
:10F77000084910B50A69042A0AD0074A096942F8FB
:10F78000210004480121103001F0E0FC002010BDF0
:10F790000C2010BD481D00205C2D0020F0B5074650
:10F7A000204893B01546006812904FF6AA600E00EC
:10F7B0004FF00004ADF83C0004D0D6E90001CDE9DB
:10F7C000100101E0109411943C216846FAF7CFFC37
:10F7D0008DF8004006208DF803000120ADF81000E0
:10F7E00012A805900FA80A900EB1012000E0002099
:10F7F0008DF82C002A1D68462968FCF7CBFD08B15E
:10F80000FCF750FB5FB105F10C023846A968FCF724
:10F81000C1FD002801D0FCF745FB13B0F0BDAC6082
:10F82000AC81FAE70C47020010B5002821D0114B3B
:10F830000022001F196803E0814203D80A46496884
:10F840000029F9D152B11368841A9C4204D100688E
:10F8500018441060104602E0506000E0186039B1B2
:10F8600002680B1A934203D10B681A44026049687C
:10F87000416010BDB01D0020406803F0F5BC0000E1
:10F8800000B519A387B00FCB0DF1040C8CE80F0065
:10F890009DF8000020F00F00401C20F0F000103018
:10F8A0008DF8000001A8FAF76DFC82B201A9684644
:10F8B0007CDF08B1FCF7F6FA0020059006902821BD
:10F8C000ADF81800ADF814104FF4C8704821ADF829
:10F8D0001A00ADF8161005A87ADF002801D0FCF751
:10F8E000E1FA07B000BD00006E524635785F45640E
:10F8F000647973746F6E650070B508B1012070BDD6
:10F90000194C0025E07C08B1E57401E000F0A0F896
:10F910002078082826D2DFE800F02504080C1025FE
:10F920001420BDE8704000F021B8BDE8704000F040
:10F930007DB8BDE8704000F05FB8BDE8704000F0F1
:10F940003BB86088084900EB8000B43901EB8000C7
:10F950004068BDE8704003F0A1BB6560BDE8704041
:10F9600003F0AABB0F2070BD542F00201149F0B442
:10F970008A1C00200346A1F1B4050C18A67A4EB1EA
:10F98000A37200EB800405EB8404E66816B9247CBE
:10F99000012C0AD0401C80B20928EED30B704B809A
:10F9A0004B60F0BC41F61D5070471080F0BC00F079
:10F9B0003DB80000542F00200C48418801EB810223
:10F9C000A0F1B40101EB8201CA6852B105210170B6
:10F9D000074802218180016800230122054802F0C6
:10F9E00065BB042202704968F6E70000542F00202E
:10F9F000701D0020B81D002038B50A4908480324AE
:10FA00000B684268898803EB810153880470DB1C12
:10FA100000201B0400909B0B034802F0E5FB38BD5F
:10FA2000542F0020701D0020B81D0020074910B57C
:10FA30004888091D03F020FE18B1BDE81040FFF70B
:10FA4000DBBFBDE81040FFF7B7BF0000542F002018
:10FA5000F0B51F481F490125067802248B88A0F1C4
:10FA6000B402082E19D2DFE806F00418181B222F62
:10FA70002F170189491C01810021418080F8131052
:10FA800001EB810312F8233043B100234418491CD1
:10FA900089B2A3720929F3D30570F0BD0123F5E7FC
:10FAA00042685288D21C1A448A800470F0BD46888D
:10FAB0000D6806EB860602EB860256680E605560FE
:10FAC00013818C80062100E007210170F0BD000049
:10FAD000542F0020701D00202DE9F0410D46060036
:10FAE000174609D05DB1144C1449A068884209D06A
:10FAF00048F20250BDE8F08148F21350FAE748F2AC
:10FB00001450F7E713462A463146606802F06EF952
:10FB1000A0F505417139EDD100221146104602F0E1
:10FB2000A3F90028E6D13B462A4631466068BDE885
:10FB3000F04102F05BB90000501C00206572E54BFB
:10FB400070B50E46154604461821FAF710FB002E34
:10FB500002D04FF0050001E04FF0010020704FF09F
:10FB600000006060207503D04FF48040A06003E087
:10FB70004FF47A70A06015B14FF0000001E041F23F
:10FB80007070A0814FF00100607570BDF0B50D4C34
:10FB90000246002004F11C0504F138034AB154F870
:10FBA0002060964205D353F8206055F82070BE427D
:10FBB00007D153F820608E4203D8401C0728EDD3AC
:10FBC0000020F0BDA047020010B501460020FFF75D
:10FBD000DDFF024951F8200010BD0000A0470200DF
:10FBE00010B559B1094B002233F82240844207D1A5
:10FBF00003EB820040880880002010BD0E2010BD5D
:10FC0000521CD2B20D2AEFD3052010BD00200020D7
:10FC10004FF0013101EAD01101EBC10101EB4101CB
:10FC200000F07F3081EA4000704700002DE9F0418C
:10FC30008046024601200021FAF771FA1A4F054664
:10FC40000E467868FCF760FA00280CD1174CD4E90E
:10FC5000062110462A4001EA06031A4305D0A843AC
:10FC6000B143C4E90601BDE8F081404602F0AAFEB6
:10FC700030B1D4E9040128433143C4E9040105E06B
:10FC8000D4E90410A943B043C4E90410D4E906013F
:10FC900028433143C4E90601A1687868BDE8F04112
:10FCA0000022FCF7EDB90000E0440200781C0020BF
:10FCB00002494968002900D008477047801D00208C
:10FCC000428800EB82020C328A4201D9022070473E
:10FCD0008188A1F57F42FF3A03D0008808B1002057
:10FCE000704701207047884204D20068401C01D050
:10FCF00001207047002070472DE9FF4FCD6883B089
:10FD00005819401EB0FBF5F7DDF840B099468A4619
:10FD10004FF00008FF2F04D948F2145007B0BDE897
:10FD2000F08F002634463BE0601C8DF80000DDE9D2
:10FD300013235146039801F06BFF0028EED134B134
:10FD40002A461299039801F08BFF0028E6D1BBF1F7
:10FD5000000006D00146119A039801F081FF0028A7
:10FD6000DCD101226946039801F07AFF0028D5D141
:10FD700001AA01951299039801F02EFFB0F1000835
:10FD8000CCD19DF80000B84201D02A4601E0A9EB91
:10FD90000602059812993044FAF7D0F92E44641CF3
:10FDA000BC42C1D34046B9E710B50A4941600A4890
:10FDB00001F0C9F958B902F0ABFC07491C238C22A9
:10FDC000087404488C39001F006801F05DF90020B8
:10FDD00010BD0000544802009C3000202DE9F04185
:10FDE0002D4F002518B17D600120BDE8F081087914
:10FDF000012258B1294E01280CD0274C4FF002089F
:10FE00000834022821D0032842D128E00A7103F0E7
:10FE100053F93BE05FF0000000EB800116F8211081
:10FE2000022908D0401C80B20928F5D33A707D60C1
:10FE300041F61D50D9E700EB800006F8205006EB94
:10FE40008000406803F02AF920E00D71A4F80480D6
:10FE5000002301221248216802F028F916E00D71F2
:10FE6000206803F01BF90D492368B431498801EB80
:10FE7000810206EB8201D1F804C0C4F800C04B60D7
:10FE8000A3880B81A4F8048006F822500028ACD087
:10FE90007D600E20A9E70000681D0020A02E002034
:10FEA000B81D00200146034802888A4200D0002085
:10FEB00070470000181F002070B50546FFF7A8FE28
:10FEC0000446FFF7A5FE0646FFF7A2FE80EA0502FC
:10FED00086EA0201654084EA02004D4085EA30600E
:10FEE00080EA314080EA322070BDF0B50368C26814
:10FEF00003F07F41C2F3074441EA04448168C3F33D
:10FF00000746C1F3072544EA05274468E5B22F43B5
:10FF100004F07F4545EA0645C2F3072645EA062672
:10FF2000CDB22E4301F07F45C4F3074C45EA0C45A2
:10FF3000C3F3072C45EA0C2502F0FF0C02F07F42C8
:10FF4000C1F3074142EA0141C4F3072241EA022119
:10FF5000DAB245EA0C051143C0E90251C0E9007666
:10FF6000F0BD000010B5044600680A4903F024FE05
:10FF700020600849606803F01FFE60600549A068C2
:10FF800003F01AFEA0600349E06803F015FEE0608C
:10FF900010BD0000F945020002498968002900D01F
:10FFA00008477047BC1C00200248007A002800D097
:10FFB000012070479C300020F0B58488A518944239
:10FFC00000D82246A41AC288D6189A4200D81346EE
:10FFD000D21A4B880788BB420CD34088834209D889
:10FFE0008888A04206D3A84204D8C888904201D38A
:10FFF000B04201D90020F0BD0120F0BD800701D042
:020000040002F8
:1000000000207047012070470A4810B5807860B121
:10001000002401E0022C06D02046FCF76BFD641C96
:10002000042CF7D310BD0324F6E7BDE81040FCF71D
:1000300081BD0000201C002003480179C90702D0BF
:100040000078FCF74FBE7047201C0020172101806C
:100050004180002101714171704700002DE9F04796
:10006000394E002780463D46DFF8E090D6F804A0E0
:1000700057E003D00446D0F81C8035E099F8002002
:1000800002EB4201521CD2B289F8002009EBC101F7
:1000900099F80230091D9A4201D189F80050486848
:1000A0000A780446012A12D0022A02D0032A3BD140
:1000B00008E003F087FE00B10127257434E00574E1
:1000C000C06900E070680028F9D170602CE0207CE5
:1000D00050BB88686060C868A0600869E0604869D3
:1000E000A061F07800B165606268B168184B501A81
:1000F00020F07F40984202D2A168084406E0881AA6
:10010000A16820F07F40814202D9081A206000E0F7
:10011000256065600120A56020742046E56103F03C
:1001200033FEB8F10000A4D199F8001099F801004D
:100130008142A3D117B97168514502D00120BDE8B1
:10014000F0870020FBE70000A81C00208822002088
:10015000FFFF7F0070B505461248002200EB8511B5
:100160000C462846FEF74CF90A281AD008B1FBF7CE
:1001700099FE94F82620302A06D02946BDE8704022
:1001800001230848FEF7D8BF0749012004F13003D6
:10019000087094F82B102846E26ABDE87040FEF71C
:1001A00045BC70BDB02B0020381D002088B0FBF787
:1001B00027FF08B1FBF776FE00210120FCF748FD80
:1001C00008B1FBF76FFE40F6CD4201213148FBF745
:1001D00015FE08B1FBF766FEFBF7FEFD08B1FBF765
:1001E00061FE2D4A0A210820FBF7D8FE08B1FBF773
:1001F00059FE02F0E5F808B1FBF754FE02F02EFAC2
:1002000008B1FBF74FFE00246846009402F0BAF9EB
:1002100008B1FBF747FE019401208DF80500029418
:10022000039401A94020009A69DF08B1FBF73AFE68
:10023000684602F0B1F908B1FBF734FEFFF720FB86
:1002400015480021B03001F069F908B1FBF72AFE2A
:100250001C216846F9F78BFF4FF42030CDE90040B0
:100260004FF47020029003208DF80C00ADF80E4082
:100270008DF810406846FCF74FF908B1FBF712FE05
:10028000064800F097FF00BFFBF768FE02F0ACF8ED
:10029000FAE70000181C0020CC1D0020552E02009B
:1002A000F0B50B30154D20F007010024144A0FE083
:1002B00003688B420BD38B4205D95E1A43184768FB
:1002C000C3E9006700E04368136002C004E0021D58
:1002D00010680028ECD12046002802D1286808B117
:1002E0000020F0BD064A07481060074A121A22F0A3
:1002F0000702C0E9002401202860D7E7B41D0020D0
:10030000B01D0020C4300020C038002070B5144655
:1003100082880E4605462088111D0144921C994290
:1003200001D8FE2A01D90C2070BD521C32542088FD
:10033000FF21401C80B2208031542088401C80B2B4
:1003400020808119288803F0D5FD2188084480B2D7
:100350002080AA8842B1A96841B13044F9F7EEFE85
:100360002088A98808442080002070BD072070BD27
:100370004840411E8143C1F3C0104042C0B27047A3
:1003800010B5144601291A46214603D000F006F89C
:10039000002010BD00F0E6F9FAE700002DE9F84F63
:1003A000CC7843680D684E6864F31F6510CB8F6886
:1003B0006C40CD7991F80FC065F31F6620CB0068C3
:1003C0007540CE7ADFF890E366F31F6753F8086B49
:1003D0000EF5806B7E40CF6853F8041C6CF31F67EA
:1003E00079404FF0FF3707EB600A0BF58060CDE0F6
:1003F00004F0FF0C53F8049B5EF82C70C6F3074C16
:1004000089EA0709C1F3072750F82CC05BF8277069
:10041000984687EA0C0789EA0709D04F4FEA156C1E
:1004200057F82C7005F0FF0C89EA07091F685EF881
:100430002C30C1F3074C5F40C4F3072350F82CC0A5
:100440005BF8233083EA0C035F40C44B4FEA166C21
:1004500053F82C305F4008F104030093D8F804C02F
:1004600006F0FF085EF82830C4F307488CEA030C56
:10047000C5F3072350F828805BF8233083EA08038C
:100480008CEA030CB54B4FEA116853F828308CEA1C
:10049000030C009B1B1D0093D3F80080CBB25EF8C9
:1004A0002310C5F3074388EA0108C6F3072150F873
:1004B00023305BF8211009F0FF05594088EA010854
:1004C000A649230E51F82310009B88EA01085EF824
:1004D00025105C68CCF307454C40C8F3072150F861
:1004E00025505BF8211069404C409C493D0E03F1BA
:1004F000080651F825109D68FBB24C405EF82310A9
:10050000C8F307434D40C9F3072150F823305BF887
:100510002110AAF1010A59404D4090494FEA1C634D
:1005200051F82310331D00930CF0FF034D40766803
:100530005EF82310C9F307434E40C7F3072150F874
:1005400023305BF82110C7F3074759404E408349D9
:100550004FEA186308F0FF0851F82310009B4E4043
:100560001B1D009319685EF8283050F82770594019
:10057000CCF307235BF823307B405940774B4FEA9D
:10058000196753F827305940009B1B1DBAF1000F23
:100590003FF72EAFDFF8C0C104F0FF0880CB5CF856
:1005A00028C0C6F3074887EA0C07C1F3072C864624
:1005B0005BF82CC050F828009A468CEA000C87EAB9
:1005C0000C0766484FEA156CD3F8008050F82C00F1
:1005D000EBB24740604806F0FF0C50F82300C1F32F
:1005E000074388EA0008C4F307205EF823305BF86D
:1005F0002000584088EA00085848330E50F823007D
:10060000554B88EA00095AF8040F53F82C3001F0D2
:10061000FF085840C5F30723C5F307455BF823C01F
:10062000C4F307435EF825505EF823308CEA030CD0
:1006300080EA0C00494B4FEA116C474953F82C30C3
:1006400058400AF1040351F8281053F804CB8CEAFF
:10065000010CC6F307215BF8211069408CEA010CFC
:100660003E49240E51F8241010CB8CEA010C3C4971
:1006700051FA87F52D78C0F307466C40CCF3072577
:100680008E5D4D5D2D0285EA06456C4001EB1965D6
:100690002D7884EA056420CB51FA89F63678CCF3BC
:1006A00007487540C7F3072611F808808E5D9A4603
:1006B000360286EA0846754001EB10661B683678FC
:1006C00085EA066551FA80F63678C7F30748734025
:1006D000C9F3072611F808808E5D360286EA0846BF
:1006E000734001EB1C66367883EA066651FA8CFC8F
:1006F0009CF800C0DAF80430C0F3072083EA0C034A
:10070000C9F3074C085C11F80CC0000280EA0C40E9
:10071000434001EB1760210A007814705170210CDE
:100720009170210ED1701571290A5171290C9171A6
:10073000290ED1711672310A5172310C9172310E3B
:1007400083EA0060D1721073010A5173010C917336
:10075000000ED073BDE8F88F485B020048670200C6
:10076000485A02002DE9F84FCC7843680D684E686E
:1007700064F31F6510CB8F686C40CD7991F80FC082
:1007800065F31F6620CB00687540CE7ADFF890E3F2
:1007900066F31F6753F8086B0EF5806B7E40CF68D9
:1007A00053F8041C6CF31F6779404FF0FF3707EBD9
:1007B000600A0BF58060CDE004F0FF0C53F8049B59
:1007C0005EF82C70C6F3074C89EA0709C5F30727C2
:1007D00050F82CC05BF82770984687EA0C0789EA26
:1007E0000709D04F4FEA116C57F82C7005F0FF0C39
:1007F00089EA07091F685EF82C30C1F3074C5F4097
:10080000C6F3072350F82CC05BF8233083EA0C03AF
:100810005F40C44B4FEA146C53F82C305F4008F132
:1008200004030093D8F804C006F0FF085EF82830EF
:10083000C4F307488CEA030CC1F3072350F828805F
:100840005BF8233083EA08038CEA030CB54B4FEACC
:10085000156853F828308CEA030C009B1B1D00938D
:10086000D3F80080CBB25EF82310C5F3074388EAC3
:100870000108C4F3072150F823305BF8211009F078
:10088000FF05594088EA0108A649330E51F82310A4
:10089000009B88EA01085EF825105C68CCF30745E8
:1008A0004C40C7F3072150F825505BF821106940F0
:1008B0004C409C494FEA186503F1080651F8251091
:1008C0009D68FBB24C405EF82310C8F307434D40CF
:1008D000CCF3072150F823305BF82110AAF1010A6C
:1008E00059404D408F494FEA196351F82310331D89
:1008F00000930CF0FF034D4076685EF82310C9F3B7
:1009000007434E40C8F3072150F823305BF821100D
:1009100008F0FF0859404E4082493B0EC7F3074795
:1009200051F82310009B4E401B1D009319685EF880
:10093000283050F827705940C9F307235BF823305B
:100940007B405940774B4FEA1C6753F8273059409A
:10095000009B1B1DBAF1000F3FF72EAFDFF8C0C19F
:1009600004F0FF0880CB5CF828C0C6F3074887EA8C
:100970000C07C5F3072C86465BF82CC050F82800FE
:100980009A468CEA000C87EA0C0766484FEA116C1D
:10099000D3F8008050F82C00EBB24740604806F0D6
:1009A000FF0C50F8230088EA0008C6F307205BF824
:1009B0002030C1F307405EF82000434088EA030876
:1009C0005848230E50F82300554B88EA00095AF87E
:1009D000040F53F82C30C4F3074C5840C1F30723DD
:1009E0005EF82CC05BF8233001F0FF0883EA0C03AB
:1009F00058404C4B4FEA156C494953F82C3058403D
:100A00000AF1040351F8281053F804CB8CEA010CC6
:100A1000C4F30721C5F307445BF821105EF82440B6
:100A200061408CEA010C3F49340E51F8241010CB80
:100A30008CEA010C3C4951FA87F52D78C0F3074642
:100A40006C40C9F307258E5D4D5D2D0285EA064594
:100A50006C4001EB1C652D7884EA056420CB51FACB
:100A600089F63678CCF307487540C0F3072611F8AD
:100A700008808E5D9A46360286EA0846754001EB8C
:100A800017661B68367885EA066551FA80F636786F
:100A9000C7F307487340CCF3072611F808808E5D32
:100AA000360286EA0846734001EB1966367883EA17
:100AB000066651FA8CFC9CF800C0DAF80430C7F3E3
:100AC000072783EA0C03C9F3074CCF5D11F80CC06C
:100AD00001EB1060210A007814705170210C9170A4
:100AE000210ED1701571290A5171290C9171290EAD
:100AF000D1711672310A51723F02310C87EA0C47EC
:100B000091727B40310E83EA0060D1721073010A4A
:100B10005173010C9173000ED073BDE8F88F000083
:100B2000484A02004856020048490200002807D0FF
:100B300040F217115FF0000200F8012B491EFBD2B2
:100B400070474FF48C71F9F712BB00002DE9F04F9C
:100B5000C7B0054616460F466846FFF7F2FF05F197
:100B600008043246394668466C6000F055F84690F5
:100B7000F0BB00982860DDE9001000EB011101C90D
:100B800001C401C901C401C944F8080B51F81C098A
:100B900044F8040C2A6828E01E48002500F5905906
:100BA00000F5B05A00F5D05C00F5F05B08C950FACA
:100BB00083F637786D1C59F82760C3F3072710F8C0
:100BC00007805AF828707E40C3F3074700EB136391
:100BD000C75D93F800805CF827705BF828305F40B1
:100BE0007E4040C4042DE1DB2039521E002A00E083
:100BF00008E0D1DC08682060486860608868A06010
:100C0000C868E0606846FFF791FF469847B0BDE8C6
:100C1000F08F000048490200F0B5802A07D0C02AB2
:100C200007D0B2F5807F0BD06FF01F00F0BD0A2314
:100C300000E00C23036000F10803002443600AE095
:100C40000E23F7E701EB8405EE782D6866F31F6548
:100C500043F82450641CB4EB521FF3D3544A016888
:100C6000A2F508500A2904D00C292BD00E2928D12E
:100C700056E0002453F80C5B52F824104D4002CB90
:100C8000C1F30726C1F30747865DC75D86EA0726DD
:100C9000754000EB1166367885EA064550FA81F614
:100CA0003678641C85EA06651D6053F80C6C6E404E
:100CB0005E6053F8085C75406940C3E902510A2C34
:100CC000D8D373E05FF000041D6852F824104D4043
:100CD0005969C1F30726C1F30747865DC75D86EAF8
:100CE0000726754000EB1166367885EA064550FA0E
:100CF00081F63678641C85EA06659D615E686E4003
:100D0000DE619D6875401D62DE686E405E621D6931
:100D100075406940C3E90A511833082CD4D345E023
:100D20005FF000051C6852F825104C40D969C1F3EA
:100D30000726C1F30747865DC75D86EA072674402C
:100D400000EB1166367884EA064450FA81F636786C
:100D500084EA06661E625C6874405C629E68664057
:100D60009E62DC687440DC6250FA84F73F781E694A
:100D7000C4F3074C7E40C4F3072710F80CC0C75DCE
:100D800000EB14643F0287EA0C4724787E4086EA31
:100D900004641C635E696D1C66405E639C697440FC
:100DA0006140C3E90E412033072DBBD30020F0BDC5
:100DB000486B020070B54843044601F0B5FA0500DF
:100DC00002D02146F9F7D3F9284670BD01F05AB98F
:100DD00010B50349034800F0E3F8002010BD0000FF
:100DE000CD0D0200B50D02000020704710B50400C3
:100DF0000AD004F12000FFF799FE40F23F100021D5
:100E000004F8011B401EFBD210BD4FF4A071F9F78E
:100E1000AEB908B50023009300F001F808BD2DE934
:100E2000F04190B09846169F154604460E46B2F51E
:100E3000806F04D96FF0350010B0BDE8F081B7F5D0
:100E4000807F02D96FF03700F6E730216846F9F766
:100E50008EF9E1692069884201DC606938B13A465F
:100E60004146204600F038F80028E5D109E047B1B6
:100E70003A4641466846FBF765FD69462046FCF761
:100E80003DFF04F12008F5B11020211811F8012DC3
:100E9000521C12F0FF020A7002D1401E0028F4DC3E
:100EA0000CAB224601214046FFF76AFA102D01D90A
:100EB000102700E02F463A460CA93046F9F73EF9D4
:100EC0003E44ED1BDFE769462046FCF717FF20692B
:100ED000401C20610020AFE7F0B50F4685694FF454
:100EE000C071E1B0164604468D4203D8C5F5C07006
:100EF000B04203D26FF0370061B0F0BD6846F9F739
:100F000036F9D4E94E302A466946984710B16FF059
:100F10003300F1E7A5693FB136B10DEB050032466C
:100F20003946F9F70BF9354469462A460846FBF776
:100F300009FD69462046FCF7E1FE01202061002002
:100F4000DAE77CB53025069CCDE9004500F001F8D4
:100F50007CBD2DE9F04788B00D46DDE910890446D7
:100F60009A46164620216846F9F701F904F1200057
:100F70000746FFF7E6FD42F21070C4E90690C4E9A7
:100F80004E564FF4807269463846FFF745FE42469A
:100F900051462046FFF7A0FF08B0BDE8F0870000EB
:100FA000024AC2E90001002070470000A41D002091
:100FB00010B50446002902D0F9F7D9F8207810BD01
:100FC00010B50446FEF724FE014684EA010081EADA
:100FD000306080EA344080EA342010BDF8B50F4616
:100FE000017814460546012901D1687830B120887E
:100FF000821C9A422DD8012902D006E00720F8BDB4
:1010000069780144891C994223D8181A801E86B237
:10101000ADF800602188B81C084469467DDF0028CF
:10102000EDD12878022805D1BDF80010B14201D8D1
:1010300009210AE00821012805D16878B04202D8C8
:10104000ADF8000001E0ADF80060BDF80000FE283A
:1010500001D90C20F8BD2288401CB8542088401CBF
:1010600080B2208039542088401C2080BDF80010B8
:10107000084420800020F8BD10B5F8F716F908B133
:10108000002010BD112010BD10B531B1B2FBF3F43A
:1010900003FB14241CB1092010BD0E2010BD0160FB
:1010A0000021416081608281C381084610BD70B516
:1010B0000C460546F8F7AEF8002802D021882868CB
:1010C000084470BD10B50A8849888A4203D1F8F7F0
:1010D000E3F8012010BD002010BD70B50C46054698
:1010E000F8F7BDF8002802D061882868084470BD70
:1010F00010B50A8849888A4203D1F8F7A7F8012079
:1011000010BD002010BD01F01F0301229A40D24300
:10111000490900EB8100114600F01EB84A0950F859
:10112000220001F01F0201219140084000D001205F
:10113000704701F01F0301229A40490900EB81002A
:10114000114600F019B8012100F011B808B56A463F
:10115000F8F7F7F8009808BD08B56A46F8F7D7F829
:10116000009808BD08B56A46F8F7EBF808BD08B561
:101170006A46F8F7BFF808BD08B56A46F8F7BAF846
:10118000009808BD08B56A46F8F7E8F8009808BD69
:10119000C20800F007030120895C984008407047AE
:1011A00010B5C20800F00703885C01249C4020436E
:1011B000885410BD00B52C4995B048604FF6FF70BB
:1011C0004880FEF7A1F82948FDF7D4F908B1FAF7ED
:1011D00069FEFDF743F908B1FAF764FEFDF756F929
:1011E0000028FBD12248FDF779FC08B1FAF75AFE36
:1011F000FCF7AAFFFBF7F4F91EA30DF1400C0FCB8F
:101200008CE80F0040221F496846F8F797FF0E222E
:1012100010A90DF11200F8F791FF6846FEF704F8E7
:10122000FDF790F8002101A8FDF7B4F80A2812D0C4
:1012300008B1FAF737FE0C4800900C489DF80630CC
:10124000BDF8042000781049FCF7FAFE15B05DF8EF
:1012500004EBFCF773BF4FF47A70ADF80400002084
:101260008DF80600E7E70000801D0020882F002091
:10127000911402001000016E6F7264696373656DF2
:101280006900000010480200DBBA010010B50446F6
:10129000FCF716FF2146074800F0D4F808B1FAF72A
:1012A00001FE204601F082FD2046BDE81040FDF71A
:1012B000F3B80000882F0020FCF732BF70B55F4BF9
:1012C0000D4604000FCB8CB00DF1100C4FF0000652
:1012D0008CE80F008DF820607ED0002D7CD04FF67A
:1012E000FF70A4F864006868A066A868E0662146FC
:1012F00004A862DF002870D120788DF826004FF412
:10130000EA40ADF82400A21C09A90120A8DF0028AA
:1013100063D14B481022067068462968F8F70EFF23
:10132000BDF90400231D010241EA2020ADF80400AC
:1013300028686A46008A010241EA1020ADF82800B8
:101340003E4821465038FCF7FFF9002872D13B484F
:1013500004F10C0321464A38226FFCF7F5F9002806
:1013600068D1364804F114030AAA21464438FCF730
:10137000EBF900285ED131482A6804F11C032146AC
:101380003E381232FCF7E0F9002853D12B482A6886
:1013900004F12403214638381332FCF7D5F900282C
:1013A00048D1264804F12C0321463238626FFCF7FD
:1013B000CBF900283ED1214804F1340308AA214684
:1013C0002C38FCF7C1F9002834D11C4804F13C0347
:1013D00008AA2146263801E02EE02BE0FCF7B4F9FC
:1013E000002827D1154804F1440308AA21462038D3
:1013F000FCF7AAF900281DD1104804F14C0308AAF3
:1014000021461A38FCF7A0F9002813D10B482A68A6
:1014100004F15403214614381432FCF795F90028DE
:1014200008D106482A6804F15C0321460E381532BB
:10143000FCF78AF90CB070BD0E20FBE77044020087
:10144000401C002010B538B131B10A88102A0AD0EA
:1014500004DC012A17D110E00E2010BD112A04D09F
:10146000512A10D106E0898801E04FF6FF71A0F8FB
:10147000641008E001F066FD03E0B0F86400034981
:1014800066DF0028E9D1002010BD0000441C0020C8
:1014900030B5204C8DB00546052938D2DFE801F083
:1014A00003080F183000616F012008700DB030BDC7
:1014B0002846FDF703FD0120FCF7D2F9F6E708A95D
:1014C0002846FDF7D9FA08A92846FDF725FDEDE7DE
:1014D00069462846FDF788FB0F482021018000213E
:1014E0004180C0F804D008384088A0F57F41FF391A
:1014F000DCD0A18FB4F86400074AACDF20B9D5E78F
:101500002846FDF76BFEF9E7FAF7CCFCCEE707209B
:10151000FAE70000882F0020881D002010B560B178
:10152000C160172120F8021B20F8021B1B2100F8C4
:10153000021BFEF78BFD002010BD0E2010BD000029
:101540002DE9FC4786880C46002E4AD101880127E8
:101550000025102908D0112920D0DFF8EC903A2975
:1015600020D0552965D13EE0C07B04F10608012852
:1015700002D12088A8F80000B8F80010B8F80200DE
:10158000814256D93046A5DF10B1112803D050E072
:1015900088F805704DE088F804704DE0A01DFEF756
:1015A00055FD46E02246408934F8061F814200D8A6
:1015B00008466080172800D217206080D06870B17C
:1015C000607960B1D9E90010CDE90010ADF8026092
:1015D0006088ADF80400D368694610469847657185
:1015E0002571BDE8FC87C08804F10608172800D2E1
:1015F0001720B8F80010814200D80846A8F8020069
:1016000088F804502846B8F80010B5DF98F80500AF
:1016100078B9E06868B1D9E90210CDE90010ADF8F9
:101620000260B8F80200ADF80400E268204669469E
:101630009047A07A0028D4D02846E188A5DF00286A
:10164000CFD1A572E772CCE71044020000F18040D0
:101650000068002800D00120704708B500F18040E4
:10166000002101600068009008BD2DE9FF4F87B0A0
:101670000446DDE91758DDE91976DDE915A9DDF83D
:1016800050B0FCF71BFB00281AD1099948F2105002
:1016900011B90A99002913D10FB9002E10D1BBF14D
:1016A000000F02D1BAF1000F0AD1B9F1000F01D138
:1016B000002D05D1B8F1000F05D125B148F2135026
:1016C0000BB0BDE8F08FCDF800B0CDE90358CDE9FF
:1016D0000576CDE901A960680DF1200C9CE80E00AB
:1016E000C5682046A847EBE770B5044616460D00CE
:1016F00048F2105014D0002E12D02046FCF7DEFA2B
:1017000018B1A0F5054102390AD10649C4E900150E
:101710006A68204631469047002801D000212160A8
:1017200070BD00004145414410B50446FCF7C6FABF
:10173000002805D160688168204688470021216023
:1017400010BD2DE9F84F9846DDE90DB7DDF828A06A
:1017500091460E004FF00004054601D025B109E086
:1017600048F21050BDE8F88F706800F0DDFD04000D
:101770000CD005464A46314600F054F8060008D021
:1017800014B1204600F07EFC3046EBE748F21550DD
:10179000E8E74146284600F077F80600F0D15146C8
:1017A000284600F05BF80646A0F50540033801D056
:1017B000002EE5D10097DDE90B125B46284600F0CC
:1017C00007F80600DCD0284600F070F8D8E70000E3
:1017D0002DE9F8431E4690460F460446089DFCF747
:1017E0007DFA002817D1C7B148F21350002E12D04D
:1017F000002D10D00095606833464246056A394690
:101800002046A847002806D1204600F04FF80028BF
:1018100001D103492160BDE8F88348F21050FAE78E
:101820005345416370B516460D460446FCF756FA1B
:1018300018B1A0F50541023909D14DB16560AA681A
:10184000204631469047002801D10349216070BDF0
:1018500048F2105070BD00006341455370B50D460D
:101860000446FCF73BFA00280AD1606842692AB1B5
:101870003DB129462046BDE87040104748F203506C
:1018800070BD48F2105070BD70B50D460446FCF7AF
:1018900025FA002809D135B1606829460269204639
:1018A000BDE87040104748F2105070BD10B50446B6
:1018B000FCF714FAA0F50541023908D0002805D13B
:1018C0006068C168204688470021216010BD024A37
:1018D00021689142F4D010BD5345416310B51C46B8
:1018E000184608310832F8F7BDFC2021204600F0E8
:1018F0002CFA002010BD70B501F108000C46154609
:101900000646202100F0FAFA002810D114F8080F3A
:10191000314600F0F8002070E07F00F07F0040F0DA
:101920004000E07705F10800F8F77AFD002070BD6F
:1019300010B542680830936892799847002010BD2E
:1019400010B50C4641688A798B6800F10801204681
:101950009847002010BD00002DE9F0410E460746D3
:1019600014461D461146304600F0BEF9002810D13D
:101970002946304600F0B8F900280AD11A46214617
:101980003846FFF7B8FF002803D103492160891FBB
:101990002960BDE8F08100007652464D70B51646CC
:1019A0000C46054600F0A0F900280ED1AA79194688
:1019B000304600F0A6F9002807D131462046FFF74F
:1019C000B7FF002801D10149216070BD7052464D1A
:1019D00070B50D4614460346094900F079F9002810
:1019E0000DD1586821468279284600F095F90028E3
:1019F00005D12946BDE870401846FFF7A1BF70BD6C
:101A00007052464D2DE9F0410C4680461E46154663
:101A100012492046069F00F05BF900280CD10F49BF
:101A20002846891F00F054F9002805D160686968CC
:101A3000884203D048F24150BDE8F08142793946EE
:101A4000304600F069F90028F6D133462A4621468F
:101A50004046BDE8F041FFF741BF00007652464DD9
:101A60002DE9FF4FA9B05FEA010838A94FF0400007
:101A700091E86008DDF8ECA02790DDF8DC901868AC
:101A80001F464FF0000448F21051259028D02B9AA1
:101A9000F2B110B3369818B35FEA090148F2115059
:101AA00018D00DB1002E15D05FEA0B0102D05FEA0D
:101AB0000A010FD000203860299898B128903C98EE
:101AC000D8B1369905AACDE90221CDF8109036E0BB
:101AD00048F213502DB0BDE8F08F48F21450F9E7EA
:101AE0000846F7E7D8F8100000F01EFC040001D00B
:101AF0002894E4E748F21550ECE735B9D8F80C60C3
:101B000005A83146F8F733FB05AD3699CDF80C90B2
:101B10000095CDE9016127AB15AA4146299800F04F
:101B200020F8050005D014B1204600F0ABFA284695
:101B3000D0E715AB05A8CDE90203279A0492CDE9B9
:101B400000BA4146259B2B9A2898FEF7D5F8050048
:101B5000E9D114B1204600F095FA259838600020AC
:101B6000B8E72DE9F05F1F46DDE90AA9DDF834B0DA
:101B700090460E004FF0000401D020B108E048F27A
:101B80001050BDE8F09F306900F0CEFB04000DD08E
:101B900005464B465246314600F03AF8060008D05A
:101BA00014B1204600F06EFA3046EAE748F21550CC
:101BB000E7E75A4628460C9900F052F80600EFD1A4
:101BC0003A464146284600F007F8054614B120463B
:101BD00000F058FA2846D4E770B515460E4604467C
:101BE00002F07EFA002807D13EB160682968C26819
:101BF000914205D248F2145070BD48F2135070BDA6
:101C000083682A4631462046BDE8704018470000E8
:101C10002DE9F0411E4617460D46044600F0A2F895
:101C200098B1ACB148F21050002D0CD0002F0AD062
:101C30008EB165602B6820463246394698470028A9
:101C400001D106492160BDE8F0814FF40540FAE773
:101C500048F20150F7E748F21150F4E711BADEBA42
:101C600070B515460E46044602F03AFA00280BD12C
:101C700046B155B160682A46314643682046BDE802
:101C80007040184748F2105070BD48F2115070BDB6
:101C90002DE9F0410B480C4D0C4F401BC6080120AC
:101CA0003870002406E000BF55F834008047002853
:101CB00005D1641CB442F7D3022038700020BDE87F
:101CC000F0810000C06C0200B06C02004C1C0020CF
:101CD00028B10068884205D048F24050704748F269
:101CE000105070470020704728B139B10022C1E977
:101CF00000201046704748F21050704748F21350C9
:101D0000704720B1914205D048F21150704748F217
:101D1000105070470020704730B149B108689042B8
:101D200005D248F21450704748F2135070470A60C9
:101D3000002070470244521E04E000BF11F8013B2E
:101D400002F801398242F9D270470144491E05E088
:101D500002780B7800F8013B01F801298142F7D2A3
:101D60007047000003480078022801D00020704727
:101D7000012070474C1C002005480178022904D03E
:101D80000078012801D00020704701207047000032
:101D90004C1C002038B5041D002000F0FBF8002882
:101DA0000ED12046FFF731F800200346024600908E
:101DB00004492046FFF7C5F8BDE8384001F0C9BC2A
:101DC00038BD000089DF010010B511461A46001D1C
:101DD000FFF782F8BDE8104001F0BBBC10B5001D54
:101DE000FFF704F800F032F9002010BD10B5001D17
:101DF000FFF70FF8BDE8104001F0ABBC2DE9F04152
:101E00000F46064600F0DEFC18B148F21950BDE856
:101E1000F081FFF7B1FF40B10F4C104D606838B151
:101E2000A068A84204D10020F1E74FF40540EEE796
:101E300048F21750002EEAD1002FE8D10649084891
:101E40000C316060FFF7A6FF0028E0D1A560626852
:101E500004491160DBE70000501C00206572E54B6F
:101E6000342000206169614D70B514460D46064668
:101E700000F0A8FC10B148F2195070BD04B13DB19A
:101E80000B480C4A8168914205D048F2025070BD5F
:101E900048F2105070BD16B148F2175070BD23467D
:101EA0002A464068BDE8704001490C31FFF78CBFFD
:101EB000501C00206572E54B70B50D4C0D4A48F280
:101EC0000251A068904204D160680B4B02689A42AC
:101ED00001D0084670BD00210160A160FFF77EFFC0
:101EE0000546206808B100F0CDF8284670BD000016
:101EF000501C00206572E54B6169614D0122FDF7C0
:101F0000EBBD000070B50B4C207808B185250FE0C3
:101F10000020A06060602061E060074800F072FC73
:101F2000054600F0F5FB08B900F056FC01202070D2
:101F3000284670BD78210020F5D8010038B500256D
:101F40008DF800506846FAF7EFF8074CE068401E3D
:101F5000E060E06810B900F065FCA5709DF8000035
:101F6000FAF706F938BD00007821002070B50C465C
:101F700006460CE0402C01D2254600E04025E9B29F
:101F8000304600F033F80028F9D1641B2E44002CB1
:101F9000F0D170BD38B5124C0025217809B18520EB
:101FA00038BD00B90F480088A4F8010000208DF862
:101FB00000006846FAF7B8F800F0AAFB38B90A49F9
:101FC000601C00F067FD0500EAD100F091FD0120E2
:101FD00020709DF80000FAF7CBF8284638BD0000C5
:101FE000601C0020D84402005D2A02002DE9F8435D
:101FF0000F468046002542F2070600BF8DF80050CC
:102000006846FAF791F800F083FB58B19DF800009C
:10201000FAF7AEF83946404631DF0446B0420DD1FA
:1020200005240DE03A464146074800F056FA0446BA
:1020300000F05EFD9DF80000FAF79AF8022CDDD062
:102040002046BDE8F8830000C06C020038B50024CB
:102050008DF800406846FAF767F800F059FB18B9A8
:1020600000F056FD00F05EFD9DF80000FAF780F8E4
:10207000024800F051FA0248047038BDC06C0200FA
:10208000601C00200749097800290AD0002808D0E0
:10209000054A00218242084601D1FAF7DFBCFDF76C
:1020A00093BD7047781D0020682F00202DE9F04176
:1020B0001F46164604000D4616D02068B8B1C6B1BA
:1020C00060680268501E284215D172432046F9F715
:1020D000F8FC80B120683B463246D0F810C0294653
:1020E0002046BDE8F04160470E20BDE8F0810820A1
:1020F000FBE70920F9E71020F7E720B119B10160EB
:102100000B68114618470E20704700000448012153
:102110004174007A08B10020704701207047000028
:102120009C300020012801D0032808D10449002256
:1021300001284A7400D00020087401F0E5B8704707
:102140009C30002070B50246022801D0032A45D1F8
:10215000234C207A002841D0012833D0022831D1E5
:1021600020480023022A006802D0032A2AD11BE05B
:10217000E360017911B1012924D10DE0D0E90565B1
:10218000711B4FF48056B14200D33146294481611E
:102190004569A9420ED015E00169491C01614269F7
:1021A00091420FD1237213E0E168491CE1600829D4
:1021B00008D9E3602372022A0AD00D21FDF754F9F1
:1021C00001F048F8607C28B1BDE8704000F0A6BA84
:1021D0000021F3E7BDE8704001F096B870BD000043
:1021E0009C300020901D00202DE9F8431D46089FDB
:1021F0001646884604000DD066B1206860B135B13E
:1022000060684068B5FBF0F100FB115030B1092067
:10221000BDE8F8830E20FBE70820F9E74046F9F710
:102220004AFC90B13046F9F746FC70B12A46414667
:102230002046F9F746FC40B1009720682B4632460D
:10224000C76841462046B847E2E71020E0E770B58E
:1022500041EA4201DDE904564FF0A04441EA83011E
:1022600041EA052104EB800041EA0641C0F800176D
:1022700070BD70B541EA4201DDE904564FF0A0445B
:1022800041EA830141EA052104EB800041EA06416D
:10229000C0F8001770BD4FF0A04202EB8000D0F8EC
:1022A000002722F44032C0F80027D0F8002742EA85
:1022B0000141C0F80017704701224FF0A04382404F
:1022C00011B1C3F808257047C3F80C25704700000A
:1022D00018B5084B6C4601441B68009306E000BF2C
:1022E00054F82030D3F81035401C08C28142F7D88A
:1022F00018BD0000DC440200034908B50844002171
:1023000001600068009008BD00600040024940582C
:10231000012800D0002070470060004000210846DE
:10232000FFF76CBDFFF7C8BD1CB50024CDE9004028
:1023300001A9684600F004F800B1009400981CBDA3
:102340002DE9F04105461B480C46007868B148F27B
:102350000E10002D07D0002C05D0206808B12028D1
:1023600006D948F20710BDE8F08148F20810FAE7F4
:102370000121FDF70BFC104A0F49383248F20416D0
:1023800051F8201052F8207089B90846FDF71CFC5E
:10239000084A0146121D106810F0010F07D020F006
:1023A000010010600548002638442860216030464E
:1023B000D9E70000781D0020BC470200682F0020EC
:1023C000064910B500204870091D0860BFF35F8FF3
:1023D0000349044800F0CEF9002010BD981D0020EC
:1023E00098480200B030002010B500F091F908B113
:1023F00041DF10BD20BF40BF20BF10BD01680A688B
:1024000049688068884201D9491C00E00021914256
:1024100001D101207047002070478068884201D9AF
:10242000481C7047002070472DE9F84304464FF0E0
:1024300000080E468DF800806846F9F775FE2046C4
:10244000FFF7DCFF07000AD0207C40B14FF0040802
:102450009DF80000F9F78CFE4046BDE8F88320683F
:10246000456841682046FFF7D8FF2168486037B1CA
:10247000206801682046FFF7D0FF21680860E26805
:10248000012A14D0022A16D0042A19D0082A1CD0F6
:102490006068314605FB0200F7F750FE204600F069
:1024A000D7FF21688A688242D2D28860D0E761680B
:1024B00030784855F2E76168308821F81500EDE77B
:1024C0006168306841F82500E8E7D6E900016268F4
:1024D00002EBC502C2E90001E0E7F8B507464FF09C
:1024E000000415000E46204615D08DF80000684601
:1024F000F9F71AFE384600F0ABFFA84205D32A468A
:102500003146384600F050FF00E005249DF80000F9
:10251000F9F72EFE2046F8BD38B5054600248DF8A3
:1025200000406846F9F700FE286804604460846053
:102530009DF80000F9F71CFE38BD0000024A10604B
:10254000101D0160704700002C7600400301034815
:102550001844C0F81425C0F81015704700700040EA
:1025600002494058002800D0012070470070004008
:10257000034908B50844002202600068009008BDC5
:102580000070004020B103490968016000207047D5
:102590000E2070471C49020060DF002802D1024A69
:1025A0000121117070470000A31D002030B51448B0
:1025B00091B00078002820D05FF03405ADF840508D
:1025C00010A903A861DF30B1052816D011B0BDE80D
:1025D0003040F9F767BC03AC0A49684600F0CAF816
:1025E00007E000BFD0E9002120469047684600F090
:1025F000D8F802980028E1D0F4E711B030BD00000F
:10260000A31D002020490200F8B5134C2078C0B16A
:102610000120A07001F03AF9112814D0022001F035
:102620004DF900258DF800506846F9F77DFD11DF62
:10263000064625709DF80000F9F79AFD2EB1304648
:10264000F8BD0820F8BD0020F8BDA57001F056FACD
:10265000032001F033F9F6E7A01D00207CB5204CE3
:10266000207808B108207CBD0120A070002001F076
:102670000DF9112819D0002001F020F91948002681
:10268000006801908DF800606846F9F74DFD164925
:1026900001A810DF05000AD0002020709DF800007E
:1026A000F9F766FD2DB128467CBD00207CBD0120D8
:1026B000F3E7A67066700721162001F075F808B1DF
:1026C000F9F7F0FB0721152001F06EF808B1F9F7D2
:1026D000E9FB01F02FFA012001F0F0F8E5E7000036
:1026E000A01D0020B448020075BE01000EB50749C8
:1026F000684600F03FF805E0D0E9001088476846DA
:1027000000F04FF802980028F6D10EBDD048020024
:102710000148007870470000A01D0020054881781E
:1027200019B1007818B1FFF76FBF08207047FFF7A5
:1027300095BF0000A01D00201FB568464BDF30B1DB
:10274000052814D004B0BDE81040F9F7ABBB084928
:1027500001A800F00FF806E0D0E9002100989047AA
:1027600001A800F01EF803980028E6D0F4E71FBD8A
:102770003C490200016009684160AFF3008010B578
:10278000D0E900215368994201D1002104E0D1E948
:102790000034A34202D01946816010BD0831416067
:1027A000F0E7816800290BD0026892680A448260D1
:1027B00041684B689A4203D108314160FFF7DFBF9F
:1027C0007047000003496846884201D201207047E3
:1027D00000207047C038002008480068012110F030
:1027E000010F08D14FF0E020E02280F80024C0F86B
:1027F0008012C0F8001102480160704700E100E05B
:10280000180500400649024600200B790BB18520CF
:1028100070470A6001220A7100224A717047000065
:10282000641C002004490120086004480168C1F3C9
:1028300000410029FAD170470C0000401804004004
:10284000002802D00149800108477047E94402008E
:102850002DE9F0418846054600F0CEFC234E0028C5
:1028600028461AD0FAF768FF304490F848008009EB
:10287000032802D001280ED007E04FF0A040D0F886
:102880001005E84010F0010F05D003212846BDE8EF
:10289000F041FFF700BD0221F8E700F0B9FC002885
:1028A00022D02846FAF748FF04464FF4807000EB28
:1028B00084000F4F81B207EB8400D0F8102542F05E
:1028C0000102C0F810250846FFF716FDB8F1000F09
:1028D0000AD02846FAF730FF56F82000002803D027
:1028E0000120A040C7F80403BDE8F081DC210020EE
:1028F000006000402DE9FC41DFF8BC80044608EB95
:102900000400002790F930001346C0170E46401C03
:1029100001D008274CE0B0781946C0F340022046A9
:10292000FAF7E6FE0546401C41D0B078410719D4BD
:10293000C0070AD04FF0A04000EB8401D1F8000797
:1029400020F00200C1F8000707E00021737820465C
:1029500000910A460191FFF78CFC1749204654313B
:10296000FEF71EFCB078800718D51448317800EBCC
:102970008500D0F81025124B1A40C0F810254FF4EE
:10298000F8524FF4403302EA042203EA01410A43B9
:10299000D0F810150A43C0F8102509E008EB05002F
:1029A000327810F8481F41EA8211017000E00427D4
:1029B0003846BDE8FC810000DC21002000600040BA
:1029C000FFE0FCFF4FF0A041D1F81015C14011F01D
:1029D000010000D00120704770B5184D95F85800DF
:1029E00008B1082070BD0020411E2A18401CC0B24A
:1029F00082F830102028F8D300242046FAF76AFE27
:102A0000641CE4B20C2CF8D300240D49E0206C6562
:102A100081F8000401264020891FC1F88002C1F816
:102A200000014FF4BE70FFF767FC0649F007C1F8DC
:102A3000040385F85860204670BD0000DC210020AA
:102A400006E000E000600040034890F858000028CD
:102A500000D0012070470000DC21002001B582B0C9
:102A600000208DF800006846F9F75EFBFFF750FE86
:102A700048B902A90648FFF7D7FC0548FFF7BEFC96
:102A800008B100F045F89DF80000F9F771FB0EBDA4
:102A9000C06C0200124A13780BB185207047516058
:102AA0000178C90704D00F490B6843F001030B609C
:102AB0000D49D1F8003223F00103C1F8003240780B
:102AC0000A49400181F8000401234FF0E020590336
:102AD000C0F88012C0F80011137000207047000089
:102AE0006C1C002004D5004000D000400DE000E048
:102AF000064908B5002204480A60096800910121CE
:102B0000C0F80413016008BD00D0004000D10040AF
:102B100003490120C1F80803091D0860704700003F
:102B200000D0004007490120C1F80803091D0860D2
:102B300041034FF0E0220020C2F8801102490870E2
:102B40007047000000D000406C1C00202DE9F041CF
:102B5000254C064612200D46C4F808032348017C84
:102B6000022918D0027C01464FF4807891F82E108B
:102B7000012A12D00222C4F80423012707744660F8
:102B800005810022C26021B3458390F82D103046A4
:102B9000FFF7D4FC25E0122002E0C2682AB102202F
:102BA000C4F804031120BDE8F081C660058361B953
:102BB00047463846FFF7D4FC0028FAD03846FFF7DE
:102BC000D7FC29463046FFF7B9FC0220C4F80403BD
:102BD00007E029463046FFF7B1FC4046FFF7C8FC46
:102BE00027600020DFE7000000700040382200204E
:102BF00070B505462A480C46017C09B1112070BD0C
:102C00002179284E09B1012901D10021316000EB61
:102C100045010A7F1AB910F82D2F521C0270E07975
:102C20000877207A487721786278302301F0030111
:102C300003EA02121143A2784FF4E06303EA02228E
:102C40001143E2784FF4805303EA023211432279B0
:102C50004FF4E02303EA0242114362794FF48013F8
:102C600003EA02521143A2791B0103EA02620E4BEE
:102C70002846114303EB0012C2F81815227AE179B5
:102C8000FFF764FC227AE1792846FFF75FFC2079A0
:102C900008B1012801D101203060002070BD000082
:102CA0003822002000750040007000402DE9F041FE
:102CB0001E4C054694F82C0010B10820BDE8F081A8
:102CC00044F8101B1A4928780860091D68780860C4
:102CD000E878A07701272777002020706077606070
:102CE000144EE0776FF00040C6F808034FF482708E
:102CF000FFF73EFCB015FFF73BFCA8780E494001FA
:102D000081F800048020C91FC1F88002C1F80001C9
:102D10000220C6F80403A07F10B10120C6F8040306
:102D20000348F03807600020C8E700003822002080
:102D3000F07500400070004007E000E00248007CB1
:102D4000002800D0012070473822002008490020C8
:102D50000A7C012A01D00820704791F82E30054ADC
:102D600001210BB111607047024A121DFAE7000001
:102D7000382200200070004070B515460A4604460F
:102D800000F108011046F7F751FB6068C068286041
:102D9000002070BD10B50830F7F762FB002010BDB1
:102DA00010B50830F7F7A6FD002010BD2DE9FE4351
:102DB0000026044600960196FCF7F4F805462188A3
:102DC0002248234F102933D0112935D14FF6FF71F6
:102DD00041800024E846E0B2FCF700FA08B1F9F7B8
:102DE00061F805EB841090F82A0038B35FF0000119
:102DF00008F80410641C052CEDD301216846FBF78C
:102E0000DBFA08B1F9F74EF8FBF730F9ADF8080036
:102E1000FBF77AF98DF80A00012102A8FBF7BAFA4C
:102E200008B1F9F73FF8786F0178012908D008E078
:102E3000A1884180386F0670BDE8FE830121D7E785
:102E400006700020FAF70CFDF6E70000801D002058
:102E5000882F002028B1012806D0022807D1F9F7D1
:102E600049BE0020F9F734BE0220F9F74BBE704787
:102E70002DE9F04190B006003ED000293CD000245E
:102E80000394049405940694887B2C4F01F1080563
:102E90004FF00208042832D006282DD1242107A89B
:102EA000F7F765F9264803A9806C019007A80290FE
:102EB0007C70ADF810408DF80C808DF81240ADF8A4
:102EC00014406889ADF81600B6F86400B0DF08B1A8
:102ED000F8F7E8FFB6F84C10B6F8640001AAADDFC9
:102EE00008B1F8F7DFFFBDF804000090B46E2A883F
:102EF000029B79883046A04710B0BDE8F0810F49A9
:102F00002888891CFCF76CFE08B1F8F7CBFF01207C
:102F10007870ADF810408DF80C808DF81240ADF847
:102F200014406889ADF816000694B6F8640003A949
:102F3000B0DF0028E0D0F8F7B5FFDDE7401C002047
:102F4000204402007FB550B149B18C798B1D00221D
:102F5000012C06D0022C15D0082004B070BD0E2024
:102F6000FBE7ADF800200D89044669462846FCF7CA
:102F700037FE0028F1D1E36E2A46BDF80010204646
:102F8000984732E01B7A012B08D0022B06D0042B85
:102F90001AD0062B18D0052B19D026E00546ADF81F
:102FA000042001F10804088901A9FCF719FE002892
:102FB000D3D160890090AE6E228804F10C03BDF875
:102FC00004102846B04710E0FFF752FF0DE00092D2
:102FD00001920220029203928DF80000ADF80420C5
:102FE00088886946B0DF0028B7D10020B5E7000027
:102FF00048B1064A0168914205D140680449401829
:1030000002D0012800D0032070470000DEC0ADDEF2
:1030100002FEE10E8A7D022A04D90289CB881A4475
:10302000D21C02814289C988511AC91E4181704748
:103030002DE9F0410D460221904600F58056298089
:1030400000F10804144F1BE031462046FCF738FE1F
:1030500040B1B8F1000F02D0012288F80020022808
:1030600016D004E0A0687969884200D97861288880
:1030700061880844C01C2880608804EB80040C34FC
:1030800031462046FCF72FFE0028DDD1BDE8F08157
:103090004FF480602880F9E7481D002008B5002122
:1030A000009101460823024A0248FFF79DF808BD37
:1030B00098470200B81D002008B500200090044881
:1030C0000823044A01680448FFF78EF808BD000091
:1030D000701D002090470200B81D00202DE9F05F10
:1030E0000025DFF80891DFF808B12C464FF00A08F8
:1030F000AA462F46D9F80C0000EB07363046FFF7FA
:1031000077FF78B3012847D0032862D100204FF41D
:10311000806200BF56F82010491C0ED004EB8401D9
:103120000BEB8102A8F10100566003221FFA80F820
:103130000BF82120641CA4B24BE0401C9042E9D360
:103140002C48016879B104EB840102200BF82100BE
:103150000BEB81014E6008812548B4304480641C2B
:10316000A4B205E007E00221066081804FF0010A69
:1031700045F001052DE004EB840100220BF821202D
:103180000BEB810101F110024E6030460831FFF770
:103190004FFF45F00205CDE7BAF1000F0CD0022039
:1031A00004EB8401134A0BF821000BEB8101126838
:1031B0004A60641C0881A4B20E480022011D06600A
:1031C0003046FFF735FF0B48808802280CD00820D6
:1031D00005437F1CBFB20A2F8CD3B8F1020F00D277
:1031E0000025E8B2BDE8F09F0420F1E7B81D0020FB
:1031F000A02E0020701D00200449084490F93000E2
:10320000082801DB0120704700207047DC210020E6
:103210000449084490F93000082801D20120704781
:1032200000207047DC2100200146054810B50068E9
:10323000FDF73DFF04461C21F6F799FF204610BD1F
:1032400088470200014602480068FDF751BF0000B0
:1032500088470200034802490068FDF733BF0000B9
:10326000941D002050480200F0B5254D254E85B034
:1032700004460027686828B9214930680831FDF7FD
:103280002CFF686001460078072817D2DFE800F0BD
:10329000160408080E0E12002046FCF79FFD02E0FF
:1032A000204600F0DBFF040028D008E02046FAF7B3
:1032B00077FDF8E72046FCF71FFBF4E70F24142105
:1032C0006846F6F754FFA4F5E8501D3800D10024F5
:1032D000019469466868FCF77DF86846FCF7B4F825
:1032E00007496F60002408313068FDF7EBFE0448A1
:1032F00001210C30FDF746FF0028BBD105B0F0BD21
:10330000481D0020884702002DE9F041234C00258C
:10331000234E207A012730B92248311D0068FDF77D
:10332000DCFE306038B1022020723168087928B1A3
:1033300001281ED116E06560BDE8F081D1E90503E2
:10334000C01A4FF48052904200D31046B7EB900F52
:1033500001D2820800E001220869C96818441944B2
:1033600029DF03E0D1E90301084428DF58B111281F
:1033700012D003213068FCF777F825726560BDE84C
:10338000F041FFF767BF207C0028D5D1BDE8F041B0
:1033900000210220FEF7D6BE2772CDE79C30002028
:1033A000901D0020504802002DE9F04104460068BD
:1033B0001746884605684068854201D8461B02E0EA
:1033C000A068461B761CE2686068B74205FB0201F4
:1033D0000CD87A434046F6F7B1FEA168E819884256
:1033E00000D9002021680860BDE8F08102FB06F5E5
:1033F0002A464046F6F7A2FEE268BE1B724308EB7F
:1034000005006168F6F79AFE20680660ECE70000A8
:1034100010B501210448FDF7A5FE002803D1BDE841
:103420001040FFF721BF10BD541D002010B5074C00
:10343000201DFDF788FE002806D1607C002803D1FE
:10344000BDE81040FFF760BF10BD00009C300020B9
:1034500001680A684968914201D3881A70478068F8
:10346000801A0844401C704710B510461A46F6F7FB
:1034700065FE002010BD0168C07809BA21F0FF0187
:10348000084370470168C07809BA21F0FF0108437A
:1034900070472DE9F04188B00D465FEA000827D05B
:1034A000002602EB8514009601960296039694F886
:1034B000260030281ED092F8410150B192F84D01FB
:1034C00038B192F84C01884203D192F84701FBF7DA
:1034D00037FD94F827001234ADF80A000394ADF8D4
:1034E00004606946404600F01FFA08B0BDE8F0816C
:1034F0000E20FAE70846FBF773FA07BA0E20ADF87C
:103500000A0030208DF810002846FBF77FFB8DF86D
:103510001100CDF812706069CDF81600A069CDF8E1
:103520001A0004A80390DAE71FB570B16AB100234E
:1035300002930193ADF80A1000930392ADF80430A2
:10354000694600F0F1F904B010BD0E20FBE7000061
:103550002DE9F04707461E481C46154600780E46E2
:1035600070B185B17CB1DFF86C804FF00009A088A4
:1035700009282BD200EB800118F8210010BB19E0BC
:103580000220BDE8F0870520FBE720681FB1818895
:103590003A8891420ED11EB101883288914209D1F8
:1035A00080682860206868600A48B43000892881F3
:1035B0000020E6E7A088214600F05EF80028E4D16C
:1035C000C4F80090A088401CA080D0E70A20D8E76B
:1035D000681D0020A02E0020F8B505464068244F45
:1035E0000C46002648B32349CA68824225D8096997
:1035F000814222D3FCF702FDF8B12889398988423B
:103600001BD1D5E900018A68904216D10020A7F1AC
:10361000B40200BF00EB800302EB83035B688B42C4
:1036200005D203F580538B4201D9208011E0401C64
:1036300080B20928EED30020F8BD268000960AE06B
:10364000009829688068884205D1009868603889A8
:1036500028810120F8BD2088694600F00DF8002877
:10366000EED12088401C80B220800928E6D3E2E712
:10367000542F0020B81D002070B50E4600EB8001CD
:10368000134800EB81004468306804F5805518B198
:10369000418800EB810411E0083410E029462046FF
:1036A000FCF70EFB20B1012805D0022807D10DE060
:1036B0000120346070BD608804EB80040C3429461E
:1036C0002046FCF710FB0028E8D170BD002070BD3B
:1036D000A02E002038B50C4600210091014604239D
:1036E000074A0848FEF780FD08B10E2038BD064A9B
:1036F00004EB840102EB810101200874002038BD35
:103700008C470200B81D0020A02E002048F2115165
:1037100010F5A24F1AD009DC10F5C34F10D010F5E8
:10372000C24F0BD010F5C14F05D10CE010F1220FA4
:1037300004D0002801D048F2165070470846704760
:1037400048F21550704748F20350704748F217503E
:10375000704710F1380F07D010F1360F07D000284E
:1037600001D048F21650704748F21150704748F2A5
:1037700014507047084670470178002911D14068FD
:103780004FF41671008810FB01F0C11700EB915047
:10379000801200EB40004FF4877101EB40000149BB
:1037A00048807047E81C002070B50D460446F8F7C5
:1037B000F5F870B12846F8F703F968B16807000E0C
:1037C000002C0CDA04F00F0101F1E02181F8140D56
:1037D00009E042F2010070BD42F2020070BD04F146
:1037E000E02484F80004002070BD000038B50021FA
:1037F000012548B101280CD0032809D1FEF7ECFFC0
:10380000BDE83840FEF79ABB4FF0E020C0F8805189
:1038100038BD8DF800106846F8F786FC064C207815
:1038200008B9FEF76FFBE068401CE060A5709DF8EA
:103830000000F8F79DFC38BD7821002038B5114C08
:1038400058B103281CD100208DF800006846F8F715
:103850006BFC2178012909D00EE0207801280FD1D6
:10386000FFF756F9BDE83840FFF75CB90649601C20
:10387000FFF710F9FFF73CF99DF80000F8F778FC26
:1038800038BD0000601C00205D2A02003EB50446E1
:1038900009496846FEF76EFF08E000BFD0E9002145
:1038A0002046904730B16846FEF77BFF029800281B
:1038B000F4D13EBD11203EBDB84802003EB50446DD
:1038C00008496846FEF756FF07E000BFD0E900212F
:1038D000204690476846FEF764FF02980028F5D11D
:1038E0003EBD0000C448020070B5002405462346D2
:1038F0000DE000BF85EA0300461E8643C6F3C010F4
:103900004042C0B2CE5C8443064034435B1C9342C9
:10391000F0D3204670BD000002498969002900D01B
:10392000084770472C1F002038B131B101220A70BE
:103930008A7100220A81FAF7EDBE0E20704740B16D
:1039400039B102220A7001228A7100220A81FAF733
:10395000E1BE0E20704700002DE9F0410746806A65
:1039600014468846C8B3002531E000BFB96A05EBAC
:10397000450001EB8006B088801CFE2802D90C208F
:10398000BDE8F0812288401C08F802002088162239
:10399000401C80B2208008F800202088401C80B2A3
:1039A000208000EB0801308800F0A4FA2188084448
:1039B00080B22080B28842B1B16871B14044F6F75C
:1039C000BDFB2088B188084420806D1CEDB297F8BB
:1039D0002C00A842CAD80020D2E7FFE70720CFE793
:1039E00030B518A289B01CCA04AD85E81C0018A225
:1039F00001AD1CCA85E81C00184B002203EB8010A7
:103A000090F8283013B190F929200AE0002301AC86
:103A1000E5568D4202DB04A9CA5602E05B1C092B65
:103A2000F6D390F82610123029B1102903D020299E
:103A300004D0302900D1427009B030BD0720F8F71A
:103A400031FAF9E7CFD9E3E8EDF2F7F9FB0000002E
:103A5000D8ECF0F4F8FC000304000000B02B0020C8
:103A6000F0B50368426803F07F41C2F3074441EABE
:103A700004448168C1F3072544EA0527C468C1F3FB
:103A80000746E5B22F4302F07F4545EA0645C4F3F9
:103A9000072645EA0626DDB22E4301F07F45C4F332
:103AA000074C45EA0C45C3F3072C45EA0C2502F008
:103AB000FF0C04F07F44C3F3074344EA0343C2F31B
:103AC000072243EA0222C9B245EA0C050A43C0E9CB
:103AD0000252C0E90076F0BD0178042901D9042121
:103AE00001707047002805D103490120487000206B
:103AF000F9F7ECBE704700007821002010B51620C1
:103B0000F7F74CFF48B10A4882684FF4800152B180
:103B1000016821F48001016010BDBDE8104042F24F
:103B20000100F8F7BFB94FF0E020C0F8801110BDD8
:103B30009423002010B51620F7F730FF80B10F480E
:103B400090F800044009F7F73BFF60B10C48826829
:103B50004FF480016AB1016841F48001016010BD39
:103B600042F2010001E042F20200BDE81040F8F725
:103B700099B94FF0E020C0F8001110BD16E000E048
:103B80009423002010B5044600680A4900F014F898
:103B900020600849606800F00FF860600549A0687F
:103BA00000F00AF8A0600349E06800F005F8E06062
:103BB00010BD0000EE4402002DE9F04F91B0020E5E
:103BC0008DF83420020C8DF83820020A8DF8400060
:103BD0008DF83C200DA80A904FF000080FA808901F
:103BE0004FF480700DF1380B0DF1400A0B91C14676
:103BF00047464646454604900B98445D0A98294638
:103C00000078FCF7B5FB28EA0001204041EA0008F3
:103C10009BF800002946FCF7ABFB29EA0001204095
:103C200041EA0009089829460078FCF7A1FB874380
:103C3000204007439AF800002946FCF799FB864389
:103C40000440049826436D1C8542D5D30A9981F817
:103C500000808BF80090089807708AF800609DF843
:103C600034009DF83810000640EA01409DF83C10F1
:103C700040EA01209DF8401011B00843BDE8F08FE4
:103C800030B500EB4002C2EB401287B0154810215E
:103C900000EB82040020059120616061A061FF2299
:103CA000E061E276A26E0DF1080C130EA377120C00
:103CB000E27704F11003CDE9000305AD04F1200221
:103CC0008CE826002346012207490848FDF739FD04
:103CD00008B1F8F7E7F820340FCC84E80F0007B0FC
:103CE00030BD0000CC250020B44402006028002034
:103CF00010B50446082902D00020F8F7D3F8D4E91B
:103D00000010BDE8104008472DE9F84F1D4C002574
:103D10006846D4E901A6FAF717F9002738B300235B
:103D2000009A61681CE0D1F800C00846944503D9A8
:103D3000ACEB02020A6015E0A2EB0C0263440760E0
:103D4000D0F80CC0C1698146BCF1000F08D006EB69
:103D5000030828F07F48C0E9018CC9F81C500546CB
:103D60000029E0D128466160FCF778F903E0284695
:103D7000FCF774F910B15046F9F736FEE770BDE86C
:103D8000F88F0000A81C00200D4B10B5596831B108
:103D900002680C68A24204D8A21A0A60C161586085
:103DA00010BD0B4603E00B46C969121B21B10C681C
:103DB0009442F8D3A41A0C600260C161D86110BDAE
:103DC000A81C00202DE9F041144E77683D462C4692
:103DD00003E0844204D02546E469002CF9D11BE0BD
:103DE000D4B1A5420BD1F869706040B90C490120EB
:103DF00088600021B160F0702F20FEF721FD21685E
:103E0000E069E86110B1026811440160706887429E
:103E100002D00120BDE8F0810020FBE7A81C0020B3
:103E2000001001407CB5064600240D468DF8004088
:103E30006846F8F779F901A800F0D2F870B105707A
:103E4000094946609DF8040048709DF80000F8F7A5
:103E50008FF91420F7F706FB20467CBD04249DF85B
:103E60000000F8F785F9F7E7882200202DE9FC41EA
:103E70001D4D6C68002C35D01C4800270068A968CF
:103E8000B846401A20F07F462068B04215D8361A4E
:103E900007442046E469017C69B180F810804169DB
:103EA000009180690190124A08216846F8F706F8E7
:103EB00008B1F7F7F7FF002CE6D12978687881423E
:103EC00006D1401CC0B26870022801D185F801807B
:103ED000054869780C3040F82170BDE8FC41142099
:103EE000F7F7C0BABDE8FC81A81C0020041501400A
:103EF000F13C02000870000A487002207047000080
:103F000010B514210448F6F732F904480068FDF7AB
:103F1000B3F8002010BD00009C3000205048020083
:103F200008B568464CDF00980249820880010A7192
:103F3000487108BD302D002010B5064C2078FBF7E5
:103F4000A3F9616808440449606000BAC1F80A0036
:103F500010BD00003C1D0020302D0020F8B50546A6
:103F600080B2FBF79FFF040013D0154E207A002784
:103F7000317B88420ED2A8B204F10A0175DF28B164
:103F8000112806D0BDE8F840FFF7C6BC207A401CD7
:103F90002072F8BD2772307C38B1A8B23B2176DFA1
:103FA00018B1082801D0FFF7B7FC71690029F0D0DB
:103FB0008DF80070ADF8025068468847F8BD0000E3
:103FC0002C1F002008B56846FAF7A0F9BDF80000DC
:103FD000024902128A70C87008BD0000302D00200E
:103FE0000A494A788B78521CD2B2934200D10022FF
:103FF0000B78934201D1002070470270487800EBA3
:10400000400001EBC000001D704700008822002026
:104010002DE9FC411646DDE90854CDE900541F4660
:104020008046022200F00CF8002807D1CDE90054A8
:104030003B4610223146404600F002F8BDE8FC81C4
:104040002DE9FC5F0026DDE90C4B994692468E4631
:1040500080462788354630E0D8F80400002200EB7F
:10406000850069460068019001A864DF002830D10E
:104070009DF8000050451FD10EB1002100E0022143
:10408000228808441118594522D846B9521C90B2CA
:10409000208009F800E02088401C2080012621882B
:1040A00001A801EB0902694664DF002811D12088CC
:1040B0009DF80010084420806D1CB8F80000A8424C
:1040C000CADC56B12088C01B401E80B2FF2802D92E
:1040D0000C20BDE8FC9F09F807000020F9E700006C
:1040E00030B100680549884205D048F20250704757
:1040F00048F20150704700207047000011BADEBA44
:10410000002070472DE9F84F114D884681461E4624
:1041100017466946DDF828A02868FCF7C8FF0400A8
:1041200013D01C21F6F723F800202071C4F800906A
:10413000C4E90486C4E902A769462868FCF7D8FFE9
:10414000FFF774F90020BDE8F88F0420FBE70000BA
:1041500050480200020E0A70020C4A70020A8A706D
:10416000C8707047020E0A70020C4A70020A8A7008
:10417000C87070472DE9FC470646364898461446F5
:1041800000780D464FF0000978B37DB32888A0F57C
:104190007F41FF3931D0688848B36868FBF72EFF4C
:1041A00068B374B32088ADF80000678801A8FFF7F2
:1041B0003BF804002FD084F800804FF0000A84F808
:1041C00016A0BDF80000A082686820612148012186
:1041D0000C38FCF7BBFFE060288820816888A0804D
:1041E000E780B8F1030F1DD020E001E003E004E018
:1041F0000220BDE8FC870520FBE70420F9E7032047
:10420000F7E7FFE72889694687B2384600F0ACF83F
:104210000028EED1CAE7BDF80010384600F098F843
:104220000820E6E70420A0753068A061A4F80A9091
:1042300001A8FFF707F846B1C6F804A0E1680648F0
:10424000316086F80AA000893081FFF7E1F800208C
:10425000CFE70000681D0020542F00202DE9F8430F
:104260000D46898A364A01EB810102EB810630B1A5
:1042700029463046FEF7CEFE0120BDE8F88331899D
:104280007068002400EB8107A97D2E484FF00E08CE
:1042900007294DD2DFE801F00C2C1523043F49001B
:1042A0004460A969016028492648FFF795F930B1B3
:1042B0000220A875042339462A1D009423E00A2011
:1042C000DBE728692A4608B1032000E00120907549
:1042D000042305F10C0207F10801009413E001200A
:1042E000A8750094E88807F10C0183002A690AE0A8
:1042F00028782A4603280CD006209075042305F15F
:104300000802391D00941148FDF76EFFA8B144461C
:104310000FE00520F1E70621A9750B4940680988DF
:10432000FFF7D8F9040004D107E041F61D5400E07E
:104330000F2429463046FEF76DFE20469DE700001B
:10434000A02E0020502D0020481D0020B81D002068
:1043500001EB8102034901EB82014A89101AC01E58
:1043600048817047A02E002070B5C01C82B240F278
:10437000FE30824201D3092070BD114B00204FF462
:10438000806500BF00EB800413F8246096B903EB4E
:1043900084063489768914443444A4B2AC4209D2E8
:1043A000088000EB800003EB8000418911444181CB
:1043B000002070BD401C80B20928E3D3072070BDE7
:1043C000A02E002070B5002404E00D5D165D754040
:1043D0000555641C9C42F8D370BD111213140D0EC8
:1043E0000F1000008C1E0020AC1E0020D81E0020E4
:1043F0000D0003007DCB01000E0003007DCB01000A
:104400000F0003007DCB0100100003007DCB0100F5
:10441000770A000000000000770A0000000000009A
:104420000175350F0F0002754F01010003752F0252
:10443000020004752F01010005752F0101000675AA
:104440005F01110007752F0110000875350120006C
:104450000975350110000A753F0022000B752A010D
:1044600001000C752F010100220000000000000077
:1044700095E2EDEB1BA0398ADF4BD38E0000C8A379
:104480002800280000202000351D0200952D020084
:10449000A12D0200792D0200200000003001000053
:1044A000000000000200800031C2010063C2010070
:1044B000A5C101000400800024010000A5C2010084
:1044C00023C30100F3C2010000000000000000004F
:1044D00041C301006FC2010001070000000000504D
:1044E00003000000682200200738FDD87047637C75
:1044F000777BF26B6FC53001672BFED7AB76CA8234
:10450000C97DFA5947F0ADD4A2AF9CA472C0B7FDE3
:104510009326363FF7CC34A5E5F171D8311504C7A1
:1045200023C31896059A071280E2EB27B275098318
:104530002C1A1B6E5AA0523BD6B329E32F8453D1B9
:1045400000ED20FCB15B6ACBBE394A4C58CFD0EFAE
:10455000AAFB434D338545F9027F503C9FA851A3E8
:10456000408F929D38F5BCB6DA2110FFF3D2CD0C06
:1045700013EC5F974417C4A77E3D645D1973608197
:104580004FDC222A908846EEB814DE5E0BDBE03268
:104590003A0A4906245CC2D3AC629195E479E7C833
:1045A000376D8DD54EA96C56F4EA657AAE08BA78A7
:1045B000252E1CA6B4C6E8DD741F4BBD8B8A703E49
:1045C000B5664803F60E613557B986C11D9EE1F800
:1045D000981169D98E949B1E87E9CE5528DF8CA14E
:1045E000890DBFE6426841992D0FB054BB168D016D
:1045F000020408102040801B3652096AD53036A5C7
:1046000038BF40A39E81F3D7FB7CE339829B2FFF09
:1046100087348E4344C4DEE9CB547B9432A6C22354
:104620003DEE4C950B42FAC34E082EA16628D924C4
:10463000B2765BA2496D8BD12572F8F664866898D4
:1046400016D4A45CCC5D65B6926C704850FDEDB993
:10465000DA5E154657A78D9D8490D8AB008CBCD3ED
:104660000AF7E45805B8B34506D02C1E8FCA3F0F91
:1046700002C1AFBD0301138A6B3A9111414F67DC50
:10468000EA97F2CFCEF0B4E67396AC7422E7AD357C
:1046900085E2F937E81C75DF6E47F11A711D29C5EF
:1046A000896FB7620EAA18BE1BFC563E4BC6D27964
:1046B000209ADBC0FE78CD5AF41FDDA8338807C7E7
:1046C00031B11210592780EC5F60517FA919B54AAA
:1046D0000D2DE57A9F93C99CEFA0E03B4DAE2AF5E6
:1046E000B0C8EBBB3C83539961172B047EBA77D6D5
:1046F00026E169146355210C7D00000010000000C4
:104700007DCF0100B5CE010000750000AAFE0100BA
:10471000E023002000240020000000000000000032
:104720000000000000000000000000002024002025
:104730000100070100000000020000090000000065
:10474000040038138C250020000000001000000039
:10475000050037131C1D00200000000004000000AD
:1047600000003713000000000000000040000000BF
:1047700001003713141D0020000000000700000096
:104780002200000000000000402D00200000FFFF7C
:10479000DEC0ADDEFF011EF1DEC0ADDEFE011EF1AA
:1047A0002000000040000000200000000001000088
:1047B0000001000028050000740D0000000000004A
:1047C00000000000000000000100000001000000E7
:1047D00001000000010000000000000000000000D7
:1047E00001000000010000000100000001000000C5
:1047F00001000000000000000000000000000000B8
:104800002000000020000000200000002000000028
:104810000000000000000000000000000000000098
:104820000000000000000000000000000000000088
:10483000000000000000100E000001000000000059
:104840000000000000000000000000000000000068
:1048500000300020001000000400000001000000F3
:10486000A9FD0100013F0200693402000541020078
:1048700099DF01007537020001410200A9FF010024
:104880000000000000000000000000000000000028
:10489000000000000000000080480200984802006C
:1048A00004000000046D02000C6D02000000000016
:1048B0000000000001000007A4480200B448020004
:1048C00008000000DC480200EC480200080000007C
:1048D000EC480200FC480200080000002C6D0200B9
:1048E000446D020000000000000000001C6D02008A
:1048F0002C6D02000000000000000000D46C0200DB
:10490000DC6C0200DC6C0200F46C0200F46C02004F
:10491000FC6C0200FC6C0200046D0200181C0020FC
:10492000FC4802001C490200080000000C6D020057
:104930001C6D020000000000000000002C49020075
:104940003C49020008000000637C777BF26B6FC576
:104950003001672BFED7AB76CA82C97DFA5947F082
:10496000ADD4A2AF9CA472C0B7FD9326363FF7CC5E
:1049700034A5E5F171D8311504C723C31896059AFB
:10498000071280E2EB27B27509832C1A1B6E5AA01E
:10499000523BD6B329E32F8453D100ED20FCB15B09
:1049A0006ACBBE394A4C58CFD0EFAAFB434D338572
:1049B00045F9027F503C9FA851A3408F929D38F546
:1049C000BCB6DA2110FFF3D2CD0C13EC5F9744177D
:1049D000C4A77E3D645D197360814FDC222A9088F4
:1049E00046EEB814DE5E0BDBE0323A0A4906245C80
:1049F000C2D3AC629195E479E7C8376D8DD54EA9E5
:104A00006C56F4EA657AAE08BA78252E1CA6B4C6B0
:104A1000E8DD741F4BBD8B8A703EB5664803F60E09
:104A2000613557B986C11D9EE1F8981169D98E94F8
:104A30009B1E87E9CE5528DF8CA1890DBFE6426811
:104A400041992D0FB054BB16C66363A5F87C7C84D6
:104A5000EE777799F67B7B8DFFF2F20DD66B6BBD0F
:104A6000DE6F6FB191C5C554603030500201010353
:104A7000CE6767A9562B2B7DE7FEFE19B5D7D76207
:104A80004DABABE6EC76769A8FCACA451F82829D03
:104A900089C9C940FA7D7D87EFFAFA15B25959EBF9
:104AA0008E4747C9FBF0F00B41ADADECB3D4D467F2
:104AB0005FA2A2FD45AFAFEA239C9CBF53A4A4F71D
:104AC000E47272969BC0C05B75B7B7C2E1FDFD1C76
:104AD0003D9393AE4C26266A6C36365A7E3F3F4154
:104AE000F5F7F70283CCCC4F6834345C51A5A5F4BC
:104AF000D1E5E534F9F1F108E2717193ABD8D873DF
:104B0000623131532A15153F0804040C95C7C7526A
:104B1000462323659DC3C35E30181828379696A197
:104B20000A05050F2F9A9AB50E07070924121236A7
:104B30001B80809BDFE2E23DCDEBEB264E27276911
:104B40007FB2B2CDEA75759F1209091B1D83839E42
:104B5000582C2C74341A1A2E361B1B2DDC6E6EB298
:104B6000B45A5AEE5BA0A0FBA45252F6763B3B4DE2
:104B7000B7D6D6617DB3B3CE5229297BDDE3E33EC0
:104B80005E2F2F7113848497A65353F5B9D1D16842
:104B900000000000C1EDED2C40202060E3FCFC1F74
:104BA00079B1B1C8B65B5BEDD46A6ABE8DCBCB463A
:104BB00067BEBED97239394B944A4ADE984C4CD400
:104BC000B05858E885CFCF4ABBD0D06BC5EFEF2A9D
:104BD0004FAAAAE5EDFBFB16864343C59A4D4DD778
:104BE00066333355118585948A4545CFE9F9F91027
:104BF00004020206FE7F7F81A05050F0783C3C44C6
:104C0000259F9FBA4BA8A8E3A25151F35DA3A3FE31
:104C1000804040C0058F8F8A3F9292AD219D9DBC00
:104C200070383848F1F5F50463BCBCDF77B6B6C11F
:104C3000AFDADA754221216320101030E5FFFF1A48
:104C4000FDF3F30EBFD2D26D81CDCD4C180C0C14F8
:104C500026131335C3ECEC2FBE5F5FE1359797A2A7
:104C6000884444CC2E17173993C4C45755A7A7F2CC
:104C7000FC7E7E827A3D3D47C86464ACBA5D5DE7E8
:104C80003219192BE6737395C06060A01981819861
:104C90009E4F4FD1A3DCDC7F44222266542A2A7E19
:104CA0003B9090AB0B8888838C4646CAC7EEEE29B2
:104CB0006BB8B8D32814143CA7DEDE79BC5E5EE284
:104CC000160B0B1DADDBDB76DBE0E03B64323256CE
:104CD000743A3A4E140A0A1E924949DB0C06060A37
:104CE0004824246CB85C5CE49FC2C25DBDD3D36E23
:104CF00043ACACEFC46262A6399191A8319595A4FA
:104D0000D3E4E437F279798BD5E7E7328BC8C8432F
:104D10006E373759DA6D6DB7018D8D8CB1D5D5648D
:104D20009C4E4ED249A9A9E0D86C6CB4AC5656FA48
:104D3000F3F4F407CFEAEA25CA6565AFF47A7A8E10
:104D400047AEAEE9100808186FBABAD5F07878887F
:104D50004A25256F5C2E2E72381C1C2457A6A6F1FE
:104D600073B4B4C797C6C651CBE8E823A1DDDD7C98
:104D7000E874749C3E1F1F21964B4BDD61BDBDDC6A
:104D80000D8B8B860F8A8A85E07070907C3E3E4248
:104D900071B5B5C4CC6666AA904848D80603030529
:104DA000F7F6F6011C0E0E12C26161A36A35355F7B
:104DB000AE5757F969B9B9D01786869199C1C158CC
:104DC0003A1D1D27279E9EB9D9E1E138EBF8F8136B
:104DD0002B9898B322111133D26969BBA9D9D97024
:104DE000078E8E89339494A72D9B9BB63C1E1E2262
:104DF00015878792C9E9E92087CECE49AA5555FF84
:104E000050282878A5DFDF7A038C8C8F59A1A1F870
:104E1000098989801A0D0D1765BFBFDAD7E6E6311B
:104E2000844242C6D06868B8824141C3299999B08A
:104E30005A2D2D771E0F0F117BB0B0CBA85454FC08
:104E40006DBBBBD62C16163AA5C6636384F87C7C72
:104E500099EE77778DF67B7B0DFFF2F2BDD66B6B0B
:104E6000B1DE6F6F5491C5C550603030030201014F
:104E7000A9CE67677D562B2B19E7FEFE62B5D7D703
:104E8000E64DABAB9AEC7676458FCACA9D1F8282FF
:104E90004089C9C987FA7D7D15EFFAFAEBB25959F5
:104EA000C98E47470BFBF0F0EC41ADAD67B3D4D4EE
:104EB000FD5FA2A2EA45AFAFBF239C9CF753A4A419
:104EC00096E472725B9BC0C0C275B7B71CE1FDFD72
:104ED000AE3D93936A4C26265A6C3636417E3F3F50
:104EE00002F5F7F74F83CCCC5C683434F451A5A5B8
:104EF00034D1E5E508F9F1F193E2717173ABD8D8DB
:104F0000536231313F2A15150C0804045295C7C766
:104F1000654623235E9DC3C328301818A137969693
:104F20000F0A0505B52F9A9A090E070736241212A3
:104F30009B1B80803DDFE2E226CDEBEB694E27270D
:104F4000CD7FB2B29FEA75751B1209099E1D83833E
:104F500074582C2C2E341A1A2D361B1BB2DC6E6E94
:104F6000EEB45A5AFB5BA0A0F6A452524D763B3BDE
:104F700061B7D6D6CE7DB3B37B5229293EDDE3E3BC
:104F8000715E2F2F97138484F5A6535368B9D1D13E
:104F9000000000002CC1EDED604020201FE3FCFC70
:104FA000C879B1B1EDB65B5BBED46A6A468DCBCB36
:104FB000D967BEBE4B723939DE944A4AD4984C4CFC
:104FC000E8B058584A85CFCF6BBBD0D02AC5EFEF99
:104FD000E54FAAAA16EDFBFBC5864343D79A4D4D74
:104FE0005566333394118585CF8A454510E9F9F923
:104FF0000604020281FE7F7FF0A0505044783C3CC2
:10500000BA259F9FE34BA8A8F3A25151FE5DA3A32D
:10501000C08040408A058F8FAD3F9292BC219D9DFC
:105020004870383804F1F5F5DF63BCBCC177B6B61B
:1050300075AFDADA63422121302010101AE5FFFF44
:105040000EFDF3F36DBFD2D24C81CDCD14180C0CF4
:10505000352613132FC3ECECE1BE5F5FA2359797A3
:10506000CC884444392E17175793C4C4F255A7A7C8
:1050700082FC7E7E477A3D3DACC86464E7BA5D5DE4
:105080002B32191995E67373A0C06060981981815D
:10509000D19E4F4F7FA3DCDC664422227E542A2A15
:1050A000AB3B9090830B8888CA8C464629C7EEEEAE
:1050B000D36BB8B83C28141479A7DEDEE2BC5E5E80
:1050C0001D160B0B76ADDBDB3BDBE0E056643232CA
:1050D0004E743A3A1E140A0ADB9249490A0C060633
:1050E0006C482424E4B85C5C5D9FC2C26EBDD3D31F
:1050F000EF43ACACA6C46262A8399191A4319595F6
:1051000037D3E4E48BF2797932D5E7E7438BC8C82B
:10511000596E3737B7DA6D6D8C018D8D64B1D5D589
:10512000D29C4E4EE049A9A9B4D86C6CFAAC565644
:1051300007F3F4F425CFEAEAAFCA65658EF47A7A0C
:10514000E947AEAE18100808D56FBABA88F078787B
:105150006F4A2525725C2E2E24381C1CF157A6A6FA
:10516000C773B4B45197C6C623CBE8E87CA1DDDD94
:105170009CE87474213E1F1FDD964B4BDC61BDBD66
:10518000860D8B8B850F8A8A90E07070427C3E3E44
:10519000C471B5B5AACC6666D89048480506030325
:1051A00001F7F6F6121C0E0EA3C261615F6A353577
:1051B000F9AE5757D069B9B9911786865899C1C1C8
:1051C000273A1D1DB9279E9E38D9E1E113EBF8F867
:1051D000B32B989833221111BBD2696970A9D9D920
:1051E00089078E8EA7339494B62D9B9B223C1E1E5E
:1051F0009215878720C9E9E94987CECEFFAA555580
:10520000785028287AA5DFDF8F038C8CF859A1A16C
:1052100080098989171A0D0DDA65BFBF31D7E6E617
:10522000C6844242B8D06868C3824141B029999986
:10523000775A2D2D111E0F0FCB7BB0B0FCA8545404
:10524000D66DBBBB3A2C161663A5C6637C84F87C6E
:105250007799EE777B8DF67BF20DFFF26BBDD66B07
:105260006FB1DE6FC55491C530506030010302014B
:1052700067A9CE672B7D562BFE19E7FED762B5D7FF
:10528000ABE64DAB769AEC76CA458FCA829D1F82FB
:10529000C94089C97D87FA7DFA15EFFA59EBB259F1
:1052A00047C98E47F00BFBF0ADEC41ADD467B3D4EA
:1052B000A2FD5FA2AFEA45AF9CBF239CA4F753A415
:1052C0007296E472C05B9BC0B7C275B7FD1CE1FD6E
:1052D00093AE3D93266A4C26365A6C363F417E3F4C
:1052E000F702F5F7CC4F83CC345C6834A5F451A5B4
:1052F000E534D1E5F108F9F17193E271D873ABD8D7
:1053000031536231153F2A15040C0804C75295C762
:1053100023654623C35E9DC31828301896A137968F
:10532000050F0A059AB52F9A07090E07123624129F
:10533000809B1B80E23DDFE2EB26CDEB27694E2709
:10534000B2CD7FB2759FEA75091B1209839E1D833A
:105350002C74582C1A2E341A1B2D361B6EB2DC6E90
:105360005AEEB45AA0FB5BA052F6A4523B4D763BDA
:10537000D661B7D6B3CE7DB3297B5229E33EDDE3B8
:105380002F715E2F8497138453F5A653D168B9D13A
:1053900000000000ED2CC1ED20604020FC1FE3FC6C
:1053A000B1C879B15BEDB65B6ABED46ACB468DCB32
:1053B000BED967BE394B72394ADE944A4CD4984CF8
:1053C00058E8B058CF4A85CFD06BBBD0EF2AC5EF95
:1053D000AAE54FAAFB16EDFB43C586434DD79A4D70
:1053E000335566338594118545CF8A45F910E9F91F
:1053F000020604027F81FE7F50F0A0503C44783CBE
:105400009FBA259FA8E34BA851F3A251A3FE5DA329
:1054100040C080408F8A058F92AD3F929DBC219DF8
:1054200038487038F504F1F5BCDF63BCB6C177B617
:10543000DA75AFDA2163422110302010FF1AE5FF40
:10544000F30EFDF3D26DBFD2CD4C81CD0C14180CF0
:1054500013352613EC2FC3EC5FE1BE5F97A235979F
:1054600044CC884417392E17C45793C4A7F255A7C4
:105470007E82FC7E3D477A3D64ACC8645DE7BA5DE0
:10548000192B32197395E67360A0C0608198198159
:105490004FD19E4FDC7FA3DC226644222A7E542A11
:1054A00090AB3B9088830B8846CA8C46EE29C7EEAA
:1054B000B8D36BB8143C2814DE79A7DE5EE2BC5E7C
:1054C0000B1D160BDB76ADDBE03BDBE032566432C6
:1054D0003A4E743A0A1E140A49DB9249060A0C062F
:1054E000246C48245CE4B85CC25D9FC2D36EBDD31B
:1054F000ACEF43AC62A6C46291A8399195A43195F2
:10550000E437D3E4798BF279E732D5E7C8438BC827
:1055100037596E376DB7DA6D8D8C018DD564B1D585
:105520004ED29C4EA9E049A96CB4D86C56FAAC5640
:10553000F407F3F4EA25CFEA65AFCA657A8EF47A08
:10554000AEE947AE08181008BAD56FBA7888F07877
:10555000256F4A252E725C2E1C24381CA6F157A6F6
:10556000B4C773B4C65197C6E823CBE8DD7CA1DD90
:10557000749CE8741F213E1F4BDD964BBDDC61BD62
:105580008B860D8B8A850F8A7090E0703E427C3E40
:10559000B5C471B566AACC6648D890480305060321
:1055A000F601F7F60E121C0E61A3C261355F6A3573
:1055B00057F9AE57B9D069B986911786C15899C1C4
:1055C0001D273A1D9EB9279EE138D9E1F813EBF863
:1055D00098B32B981133221169BBD269D970A9D91C
:1055E0008E89078E94A733949BB62D9B1E223C1E5A
:1055F00087921587E920C9E9CE4987CE55FFAA557C
:1056000028785028DF7AA5DF8C8F038CA1F859A168
:10561000898009890D171A0DBFDA65BFE631D7E613
:1056200042C6844268B8D06841C3824199B0299982
:105630002D775A2D0F111E0FB0CB7BB054FCA85400
:10564000BBD66DBB163A2C166363A5C67C7C84F86A
:10565000777799EE7B7B8DF6F2F20DFF6B6BBDD603
:105660006F6FB1DEC5C55491303050600101030247
:105670006767A9CE2B2B7D56FEFE19E7D7D762B5FB
:10568000ABABE64D76769AECCACA458F82829D1FF7
:10569000C9C940897D7D87FAFAFA15EF5959EBB2ED
:1056A0004747C98EF0F00BFBADADEC41D4D467B3E6
:1056B000A2A2FD5FAFAFEA459C9CBF23A4A4F75311
:1056C000727296E4C0C05B9BB7B7C275FDFD1CE16A
:1056D0009393AE3D26266A4C36365A6C3F3F417E48
:1056E000F7F702F5CCCC4F8334345C68A5A5F451B0
:1056F000E5E534D1F1F108F9717193E2D8D873ABD3
:105700003131536215153F2A04040C08C7C752955E
:1057100023236546C3C35E9D181828309696A1378B
:1057200005050F0A9A9AB52F0707090E121236249B
:1057300080809B1BE2E23DDFEBEB26CD2727694E05
:10574000B2B2CD7F75759FEA09091B1283839E1D36
:105750002C2C74581A1A2E341B1B2D366E6EB2DC8C
:105760005A5AEEB4A0A0FB5B5252F6A43B3B4D76D6
:10577000D6D661B7B3B3CE7D29297B52E3E33EDDB4
:105780002F2F715E848497135353F5A6D1D168B936
:1057900000000000EDED2CC120206040FCFC1FE368
:1057A000B1B1C8795B5BEDB66A6ABED4CBCB468D2E
:1057B000BEBED96739394B724A4ADE944C4CD498F4
:1057C0005858E8B0CFCF4A85D0D06BBBEFEF2AC591
:1057D000AAAAE54FFBFB16ED4343C5864D4DD79A6C
:1057E00033335566858594114545CF8AF9F910E91B
:1057F000020206047F7F81FE5050F0A03C3C4478BA
:105800009F9FBA25A8A8E34B5151F3A2A3A3FE5D25
:105810004040C0808F8F8A059292AD3F9D9DBC21F4
:1058200038384870F5F504F1BCBCDF63B6B6C17713
:10583000DADA75AF2121634210103020FFFF1AE53C
:10584000F3F30EFDD2D26DBFCDCD4C810C0C1418EC
:1058500013133526ECEC2FC35F5FE1BE9797A2359B
:105860004444CC881717392EC4C45793A7A7F255C0
:105870007E7E82FC3D3D477A6464ACC85D5DE7BADC
:1058800019192B32737395E66060A0C08181981955
:105890004F4FD19EDCDC7FA3222266442A2A7E540D
:1058A0009090AB3B8888830B4646CA8CEEEE29C7A6
:1058B000B8B8D36B14143C28DEDE79A75E5EE2BC78
:1058C0000B0B1D16DBDB76ADE0E03BDB32325664C2
:1058D0003A3A4E740A0A1E144949DB9206060A0C2B
:1058E00024246C485C5CE4B8C2C25D9FD3D36EBD17
:1058F000ACACEF436262A6C49191A8399595A431EE
:10590000E4E437D379798BF2E7E732D5C8C8438B23
:105910003737596E6D6DB7DA8D8D8C01D5D564B181
:105920004E4ED29CA9A9E0496C6CB4D85656FAAC3C
:10593000F4F407F3EAEA25CF6565AFCA7A7A8EF404
:10594000AEAEE94708081810BABAD56F787888F073
:1059500025256F4A2E2E725C1C1C2438A6A6F157F2
:10596000B4B4C773C6C65197E8E823CBDDDD7CA18C
:1059700074749CE81F1F213E4B4BDD96BDBDDC615E
:105980008B8B860D8A8A850F707090E03E3E427C3C
:10599000B5B5C4716666AACC4848D890030305061D
:1059A000F6F601F70E0E121C6161A3C235355F6A6F
:1059B0005757F9AEB9B9D06986869117C1C15899C0
:1059C0001D1D273A9E9EB927E1E138D9F8F813EB5F
:1059D0009898B32B111133226969BBD2D9D970A918
:1059E0008E8E89079494A7339B9BB62D1E1E223C56
:1059F00087879215E9E920C9CECE49875555FFAA78
:105A000028287850DFDF7AA58C8C8F03A1A1F85964
:105A1000898980090D0D171ABFBFDA65E6E631D70F
:105A20004242C6846868B8D04141C3829999B0297E
:105A30002D2D775A0F0F111EB0B0CB7B5454FCA8FC
:105A4000BBBBD66D16163A2C52096AD53036A5382E
:105A5000BF40A39E81F3D7FB7CE339829B2FFF8756
:105A6000348E4344C4DEE9CB547B9432A6C2233D3A
:105A7000EE4C950B42FAC34E082EA16628D924B2EB
:105A8000765BA2496D8BD12572F8F664866898160C
:105A9000D4A45CCC5D65B6926C704850FDEDB9DA6B
:105AA0005E154657A78D9D8490D8AB008CBCD30A59
:105AB000F7E45805B8B34506D02C1E8FCA3F0F0235
:105AC000C1AFBD0301138A6B3A9111414F67DCEA04
:105AD00097F2CFCEF0B4E67396AC7422E7AD35857D
:105AE000E2F937E81C75DF6E47F11A711D29C58987
:105AF0006FB7620EAA18BE1BFC563E4BC6D2792069
:105B00009ADBC0FE78CD5AF41FDDA8338807C73171
:105B1000B11210592780EC5F60517FA919B54A0D69
:105B20002DE57A9F93C99CEFA0E03B4DAE2AF5B0DE
:105B3000C8EBBB3C83539961172B047EBA77D626FA
:105B4000E169146355210C7D51F4A7507E416553E2
:105B50001A17A4C33A275E963BAB6BCB1F9D45F14A
:105B6000ACFA58AB4BE303932030FA55AD766DF6A3
:105B700088CC7691F5024C254FE5D7FCC52ACBD7CA
:105B800026354480B562A38FDEB15A4925BA1B671A
:105B900045EA0E985DFEC0E1C32F7502814CF012FC
:105BA0008D4697A36BD3F9C6038F5FE715929C953B
:105BB000BF6D7AEB955259DAD4BE832D587421D338
:105BC00049E069298EC9C84475C2896AF48E79781A
:105BD00099583E6B27B971DDBEE14FB6F088AD171D
:105BE000C920AC667DCE3AB463DF4A18E51A31822B
:105BF0009751336062537F45B16477E0BB6BAE84ED
:105C0000FE81A01CF9082B94704868588F45FD1937
:105C100094DE6C87527BF8B7AB73D323724B02E2EE
:105C2000E31F8F576655AB2AB2EB28072FB5C20387
:105C300086C57B9AD33708A5302887F223BFA5B243
:105C400002036ABAED16825C8ACF1C2BA779B49244
:105C5000F307F2F04E69E2A165DAF4CD0605BED590
:105C6000D134621FC4A6FE8A342E539DA2F355A0E0
:105C7000058AE132A4F6EB750B83EC394060EFAA9C
:105C80005E719F06BD6E10513E218AF996DD063D7C
:105C9000DD3E05AE4DE6BD4691548DB571C45D0542
:105CA0000406D46F605015FF1998FB24D6BDE99700
:105CB000894043CC67D99E77B0E842BD07898B887D
:105CC000E7195B3879C8EEDBA17C0A477C420FE913
:105CD000F8841EC90000000009808683322BED483D
:105CE0001E1170AC6C5A724EFD0EFFFB0F853856BC
:105CF0003DAED51E362D39270A0FD964685CA62122
:105D00009B5B54D124362E3A0C0A67B19357E70FA8
:105D1000B4EE96D21B9B919E80C0C54F61DC20A241
:105D20005A774B691C121A16E293BA0AC0A02AE5E8
:105D30003C22E043121B171D0E090D0BF28BC7AD61
:105D40002DB6A8B9141EA9C857F11985AF75074C0F
:105D5000EE99DDBBA37F60FDF701269F5C72F5BC69
:105D600044663BC55BFB7E348B432976CB23C6DC84
:105D7000B6EDFC68B8E4F163D731DCCA4263851044
:105D80001397224084C61120854A247DD2BB3DF85A
:105D9000AEF93211C729A16D1D9E2F4BDCB230F335
:105DA0000D8652EC77C1E3D02BB3166CA970B9996C
:105DB000119448FA47E96422A8FC8CC4A0F03F1A69
:105DC000567D2CD8223390EF87494EC7D938D1C1A0
:105DD0008CCAA2FE98D40B36A6F581CFA57ADE2810
:105DE000DAB78E263FADBFA42C3A9DE45078920DD1
:105DF0006A5FCC9B547E4662F68D13C290D8B8E899
:105E00002E39F75E82C3AFF59F5D80BE69D0937C6B
:105E10006FD52DA9CF2512B3C8AC993B10187DA71B
:105E2000E89C636EDB3BBB7BCD2678096E5918F48A
:105E3000EC9AB701834F9AA8E6956E65AAFFE67EB5
:105E400021BCCF08EF15E8E6BAE79BD94A6F36CEFA
:105E5000EA9F09D429B07CD631A4B2AF2A3F2331BE
:105E6000C6A5943035A266C0744EBC37FC82CAA663
:105E7000E090D0B033A7D815F104984A41ECDAF796
:105E80007FCD500E1791F62F764DD68D43EFB04D46
:105E9000CCAA4D54E49604DF9ED1B5E34C6A881B2E
:105EA000C12C1FB84665517F9D5EEA04018C355DAB
:105EB000FA877473FB0B412EB3671D5A92DBD252E3
:105EC000E91056336DD647139AD7618C37A10C7AF7
:105ED00059F8148EEB133C89CEA927EEB761C9356A
:105EE000E11CE5ED7A47B13C9CD2DF5955F2733F96
:105EF0001814CE7973C737BF53F7CDEA5FFDAA5B9D
:105F0000DF3D6F147844DB86CAAFF381B968C43EC5
:105F10003824342CC2A3405F161DC372BCE2250C8A
:105F2000283C498BFF0D954139A80171080CB3DE5F
:105F3000D8B4E49C6456C1907BCB8461D532B670F2
:105F4000486C5C74D0B857425051F4A7537E4165F9
:105F5000C31A17A4963A275ECB3BAB6BF11F9D4546
:105F6000ABACFA58934BE303552030FAF6AD766D9F
:105F70009188CC7625F5024CFC4FE5D7D7C52ACBC6
:105F8000802635448FB562A349DEB15A6725BA1B16
:105F90009845EA0EE15DFEC002C32F7512814CF0F8
:105FA000A38D4697C66BD3F9E7038F5F9515929C37
:105FB000EBBF6D7ADA9552592DD4BE83D358742134
:105FC0002949E069448EC9C86A75C28978F48E7916
:105FD0006B99583EDD27B971B6BEE14F17F088AD19
:105FE00066C920ACB47DCE3A1863DF4A82E51A3127
:105FF000609751334562537FE0B1647784BB6BAEE9
:106000001CFE81A094F9082B58704868198F45FD33
:106010008794DE6CB7527BF823AB73D3E2724B02EA
:1060200057E31F8F2A6655AB07B2EB28032FB5C283
:106030009A86C57BA5D33708F2302887B223BFA53F
:10604000BA02036A5CED16822B8ACF1C92A779B440
:10605000F0F307F2A14E69E2CD65DAF4D50605BE8C
:106060001FD134628AC4A6FE9D342E53A0A2F355DC
:1060700032058AE175A4F6EB390B83ECAA4060EF98
:10608000065E719F51BD6E10F93E218A3D96DD0678
:10609000AEDD3E05464DE6BDB591548D0571C45D3E
:1060A0006F0406D4FF605015241998FB97D6BDE9FC
:1060B000CC8940437767D99EBDB0E8428807898B79
:1060C00038E7195BDB79C8EE47A17C0AE97C420F0F
:1060D000C9F8841E000000008309808648322BED39
:1060E000AC1E11704E6C5A72FBFD0EFF560F8538B8
:1060F0001E3DAED527362D39640A0FD921685CA61E
:10610000D19B5B543A24362EB10C0A670F9357E7A4
:10611000D2B4EE969E1B9B914F80C0C5A261DC203D
:10612000695A774B161C121A0AE293BAE5C0A02AE4
:10613000433C22E01D121B170B0E090DADF28BC75D
:10614000B92DB6A8C8141EA98557F1194CAF75070B
:10615000BBEE99DDFDA37F609FF70126BC5C72F565
:10616000C544663B345BFB7E768B4329DCCB23C680
:1061700068B6EDFC63B8E4F1CAD731DC1042638540
:10618000401397222084C6117D854A24F8D2BB3D56
:1061900011AEF9326DC729A14B1D9E2FF3DCB23031
:1061A000EC0D8652D077C1E36C2BB31699A970B968
:1061B000FA1194482247E964C4A8FC8C1AA0F03F65
:1061C000D8567D2CEF223390C787494EC1D938D19C
:1061D000FE8CCAA23698D40BCFA6F58128A57ADE0C
:1061E00026DAB78EA43FADBFE42C3A9D0D507892CD
:1061F0009B6A5FCC62547E46C2F68D13E890D8B895
:106200005E2E39F7F582C3AFBE9F5D807C69D09367
:10621000A96FD52DB3CF25123BC8AC99A710187D17
:106220006EE89C637BDB3BBB09CD2678F46E591886
:1062300001EC9AB7A8834F9A65E6956E7EAAFFE6B1
:106240000821BCCFE6EF15E8D9BAE79BCE4A6F36F6
:10625000D4EA9F09D629B07CAF31A4B2312A3F23BA
:1062600030C6A594C035A26637744EBCA6FC82CA5F
:10627000B0E090D01533A7D84AF10498F741ECDA92
:106280000E7FCD502F1791F68D764DD64D43EFB042
:1062900054CCAA4DDFE49604E39ED1B51B4C6A882A
:1062A000B8C12C1F7F466551049D5EEA5D018C35A7
:1062B00073FA87742EFB0B415AB3671D5292DBD2DF
:1062C00033E91056136DD6478C9AD7617A37A10CF3
:1062D0008E59F81489EB133CEECEA92735B761C966
:1062E000EDE11CE53C7A47B1599CD2DF3F55F27392
:1062F000791814CEBF73C737EA53F7CD5B5FFDAA99
:1063000014DF3D6F867844DB81CAAFF33EB968C4C1
:106310002C3824345FC2A34072161DC30CBCE22586
:106320008B283C4941FF0D957139A801DE080CB35B
:106330009CD8B4E4906456C1617BCB8470D532B6EE
:1063400074486C5C42D0B857A75051F465537E41F5
:10635000A4C31A175E963A276BCB3BAB45F11F9D42
:1063600058ABACFA03934BE3FA5520306DF6AD769B
:10637000769188CC4C25F502D7FC4FE5CBD7C52AC2
:1063800044802635A38FB5625A49DEB11B6725BA12
:106390000E9845EAC0E15DFE7502C32FF012814CF4
:1063A00097A38D46F9C66BD35FE7038F9C95159233
:1063B0007AEBBF6D59DA9552832DD4BE21D3587430
:1063C000692949E0C8448EC9896A75C27978F48E12
:1063D0003E6B995871DD27B94FB6BEE1AD17F08815
:1063E000AC66C9203AB47DCE4A1863DF3182E51A23
:1063F000336097517F45625377E0B164AE84BB6BE5
:10640000A01CFE812B94F90868587048FD198F452F
:106410006C8794DEF8B7527BD323AB7302E2724BE6
:106420008F57E31FAB2A66552807B2EBC2032FB57F
:106430007B9A86C508A5D33787F23028A5B223BF3B
:106440006ABA0203825CED161C2B8ACFB492A7793C
:10645000F2F0F307E2A14E69F4CD65DABED5060588
:10646000621FD134FE8AC4A6539D342E55A0A2F3D8
:10647000E132058AEB75A4F6EC390B83EFAA406094
:106480009F065E711051BD6E8AF93E21063D96DD74
:1064900005AEDD3EBD464DE68DB591545D0571C43A
:1064A000D46F040615FF6050FB241998E997D6BDF8
:1064B00043CC89409E7767D942BDB0E88B88078975
:1064C0005B38E719EEDB79C80A47A17C0FE97C420B
:1064D0001EC9F8840000000086830980ED48322B35
:1064E00070AC1E11724E6C5AFFFBFD0E38560F85B4
:1064F000D51E3DAE3927362DD9640A0FA621685C1A
:1065000054D19B5B2E3A243667B10C0AE70F9357A0
:1065100096D2B4EE919E1B9BC54F80C020A261DC39
:106520004B695A771A161C12BA0AE2932AE5C0A0E0
:10653000E0433C22171D121B0D0B0E09C7ADF28B59
:10654000A8B92DB6A9C8141E198557F1074CAF7507
:10655000DDBBEE9960FDA37F269FF701F5BC5C7261
:106560003BC544667E345BFB29768B43C6DCCB237C
:10657000FC68B6EDF163B8E4DCCAD731851042633C
:1065800022401397112084C6247D854A3DF8D2BB52
:106590003211AEF9A16DC7292F4B1D9E30F3DCB22D
:1065A00052EC0D86E3D077C1166C2BB3B999A97064
:1065B00048FA1194642247E98CC4A8FC3F1AA0F061
:1065C0002CD8567D90EF22334EC78749D1C1D93898
:1065D000A2FE8CCA0B3698D481CFA6F5DE28A57A08
:1065E0008E26DAB7BFA43FAD9DE42C3A920D5078C9
:1065F000CC9B6A5F4662547E13C2F68DB8E890D891
:10660000F75E2E39AFF582C380BE9F5D937C69D063
:106610002DA96FD512B3CF25993BC8AC7DA7101813
:10662000636EE89CBB7BDB3B7809CD2618F46E5982
:10663000B701EC9A9AA8834F6E65E695E67EAAFFAD
:10664000CF0821BCE8E6EF159BD9BAE736CE4A6FF2
:1066500009D4EA9F7CD629B0B2AF31A423312A3FB6
:106660009430C6A566C035A2BC37744ECAA6FC825B
:10667000D0B0E090D81533A7984AF104DAF741EC8E
:10668000500E7FCDF62F1791D68D764DB04D43EF3E
:106690004D54CCAA04DFE496B5E39ED1881B4C6A26
:1066A0001FB8C12C517F4665EA049D5E355D018CA3
:1066B0007473FA87412EFB0B1D5AB367D25292DBDB
:1066C0005633E91047136DD6618C9AD70C7A37A1EF
:1066D000148E59F83C89EB1327EECEA9C935B76162
:1066E000E5EDE11CB13C7A47DF599CD2733F55F28E
:1066F000CE79181437BF73C7CDEA53F7AA5B5FFD95
:106700006F14DF3DDB867844F381CAAFC43EB968BD
:10671000342C3824405FC2A3C372161D250CBCE282
:10672000498B283C9541FF0D017139A8B3DE080C57
:10673000E49CD8B4C190645684617BCBB670D532EA
:106740005C74486C5742D0B8F4A750514165537EF1
:1067500017A4C31A275E963AAB6BCB3B9D45F11F3E
:10676000FA58ABACE303934B30FA5520766DF6AD97
:10677000CC769188024C25F5E5D7FC4F2ACBD7C5BE
:106780003544802662A38FB5B15A49DEBA1B67250E
:10679000EA0E9845FEC0E15D2F7502C34CF01281F0
:1067A0004697A38DD3F9C66B8F5FE703929C95152F
:1067B0006D7AEBBF5259DA95BE832DD47421D3582C
:1067C000E0692949C9C8448EC2896A758E7978F40E
:1067D000583E6B99B971DD27E14FB6BE88AD17F011
:1067E00020AC66C9CE3AB47DDF4A18631A3182E51F
:1067F00051336097537F45626477E0B16BAE84BBE1
:1068000081A01CFE082B94F94868587045FD198F2B
:10681000DE6C87947BF8B75273D323AB4B02E272E2
:106820001F8F57E355AB2A66EB2807B2B5C2032F7B
:10683000C57B9A863708A5D32887F230BFA5B22337
:10684000036ABA0216825CEDCF1C2B8A79B492A738
:1068500007F2F0F369E2A14EDAF4CD6505BED50684
:1068600034621FD1A6FE8AC42E539D34F355A0A2D4
:106870008AE13205F6EB75A483EC390B60EFAA4090
:10688000719F065E6E1051BD218AF93EDD063D9670
:106890003E05AEDDE6BD464D548DB591C45D057136
:1068A00006D46F045015FF6098FB2419BDE997D6F4
:1068B0004043CC89D99E7767E842BDB0898B880771
:1068C000195B38E7C8EEDB797C0A47A1420FE97C07
:1068D000841EC9F800000000808683092BED483231
:1068E0001170AC1E5A724E6C0EFFFBFD8538560FB0
:1068F000AED51E3D2D3927360FD9640A5CA6216816
:106900005B54D19B362E3A240A67B10C57E70F939C
:10691000EE96D2B49B919E1BC0C54F80DC20A26135
:10692000774B695A121A161C93BA0AE2A02AE5C0DC
:1069300022E0433C1B171D12090D0B0E8BC7ADF255
:10694000B6A8B92D1EA9C814F119855775074CAF03
:1069500099DDBBEE7F60FDA301269FF772F5BC5C5D
:10696000663BC544FB7E345B4329768B23C6DCCB78
:10697000EDFC68B6E4F163B831DCCAD76385104238
:1069800097224013C61120844A247D85BB3DF8D24E
:10699000F93211AE29A16DC79E2F4B1DB230F3DC29
:1069A0008652EC0DC1E3D077B3166C2B70B999A960
:1069B0009448FA11E9642247FC8CC4A8F03F1AA05D
:1069C0007D2CD8563390EF22494EC78738D1C1D994
:1069D000CAA2FE8CD40B3698F581CFA67ADE28A504
:1069E000B78E26DAADBFA43F3A9DE42C78920D50C5
:1069F0005FCC9B6A7E4662548D13C2F6D8B8E8908D
:106A000039F75E2EC3AFF5825D80BE9FD0937C695F
:106A1000D52DA96F2512B3CFAC993BC8187DA7100F
:106A20009C636EE83BBB7BDB267809CD5918F46E7E
:106A30009AB701EC4F9AA883956E65E6FFE67EAAA9
:106A4000BCCF082115E8E6EFE79BD9BA6F36CE4AEE
:106A50009F09D4EAB07CD629A4B2AF313F23312AB2
:106A6000A59430C6A266C0354EBC377482CAA6FC57
:106A700090D0B0E0A7D8153304984AF1ECDAF7418A
:106A8000CD500E7F91F62F174DD68D76EFB04D433A
:106A9000AA4D54CC9604DFE4D1B5E39E6A881B4C22
:106AA0002C1FB8C165517F465EEA049D8C355D019F
:106AB000877473FA0B412EFB671D5AB3DBD25292D7
:106AC000105633E9D647136DD7618C9AA10C7A37EB
:106AD000F8148E59133C89EBA927EECE61C935B75E
:106AE0001CE5EDE147B13C7AD2DF599CF2733F558A
:106AF00014CE7918C737BF73F7CDEA53FDAA5B5F91
:106B00003D6F14DF44DB8678AFF381CA68C43EB9B9
:106B100024342C38A3405FC21DC37216E2250CBC7E
:106B20003C498B280D9541FFA80171390CB3DE0853
:106B3000B4E49CD856C19064CB84617B32B670D5E6
:106B40006C5C7448B85742D001000000020000009D
:106B500004000000080000001000000020000000F9
:106B600040000000800000001B0000003600000014
:106B7000090000000000000000000000000000000C
:106B80000000000000000000000000000000000005
:106B9000982F8A4291443771CFFBC0B5A5DBB5E988
:106BA0005BC25639F111F159A4823F92D55E1CABFC
:106BB00098AA07D8015B8312BE853124C37D0C558A
:106BC000745DBE72FEB1DE80A706DC9B74F19BC1D2
:106BD000C1699BE48647BEEFC69DC10FCCA10C24C2
:106BE0006F2CE92DAA84744ADCA9B05CDA88F976A6
:106BF00052513E986DC631A8C82703B0C77F59BF10
:106C0000F30BE0C64791A7D55163CA06672929143B
:106C1000850AB72738211B2EFC6D2C4D130D3853D8
:106C200054730A65BB0A6A762EC9C281852C72929A
:106C3000A1E8BFA24B661AA8708B4BC2A3516CC7C8
:106C400019E892D1240699D685350EF470A06A1001
:106C500016C1A419086C371E4C774827B5BCB03450
:106C6000B30C1C394AAAD84E4FCA9C5BF36F2E68EE
:106C7000EE828F746F63A5781478C8840802C78C7D
:106C8000FAFFBE90EB6C50A4F7A3F9BEF27871C680
:106C9000446D0200181C0020B40100000CA2010089
:106CA000986D0200CC1D0020F42200008CB9010078
:106CB000D10D0200E90D02001D2302002523020070
:106CC000D02100208C2100204000000001000000A5
:106CD0000000000039C8010000000000411502005A
:106CE0007C1E0020CDC60100000000003DC7010051
:106CF000000000008D1202000000000071C60100BB
:106D0000000000000D21020000000000E53A020032
:106D1000000000004521020000000000AD25020037
:106D2000000000003927020000000000ED370200DB
:106D3000000000003D380200000000002521020094
:106D400000000000120D120304259DCE0113C01F88
:106D500003772040A3E80313A02333201F5ABF0862
:106D6000011243FFFF1206120712081209320A131A
:106D70004C241B208C041ACC04130C251B204C041F
:106D8000016C5AFF94011C14ADA1012429F8019B48
:086D900090D0EE612A79187120
:040000050001920163
:00000001FF
